:100000000C94A8180C94A7DF0C947CDF0C9451DF9F
:100010000C9426DF0C94FBDE0C94D0DE0C94A5DE51
:100020000C947ADE0C94D9180C94D9180C94D91825
:100030000C94D9180C94D9180C94D9180C94B3F6C4
:100040000C94D9180C94D9180C94D9180C94D9186C
:100050000C94D9180C94D9180C94D9180D94671BCA
:100060000C94D9180C940DE30C94E3E20C94D91879
:100070000C94D9180C94D9180C94D9180C94D9183C
:100080000C94D9180C94D9180C94D9180C94D9182C
:100090000C9439E50C94AFE40C94F1E40C9458F80A
:1000A0000C94D9180C94D9180C94D9180C94D9180C
:1000B0000C94D9180C94D9180C94D9180C94D918FC
:1000C0000C94D9180C94D9180C94D9180C94B9E242
:1000D0000C948FE20C94D9180C9465E20C943BE2DA
:1000E0000C94D91807634236B79BD8A71A396856BB
:1000F00018AEBAAB558C1D3CB7CC5763BD6DEDFD4A
:10010000753EF6177231BF000000803F0800000006
:10011000BE922449123EABAAAA2ABECDCCCC4C3EFC
:1001200000000080BEABAAAAAA3E00000000BF00EB
:100130000000803F0000000000084178D3BB4387E7
:10014000D1133D190E3CC3BD4282AD2B3E68EC82FB
:1001500076BED98FE1A93E4C80EFFFBE01C4FF7F80
:100160003F00000000000C9413660D94610F0C9486
:10017000B3930C944F930C9495620C9401DB0C9404
:10018000EEB30C944EC30C94D0580C94D2260C941D
:10019000CA600C94969B0C94074E0C94E1180C9436
:1001A0001C650C94858D0D94AA0A0C94EE330C9466
:1001B00051910C94EA940C9460390C944A660C9416
:1001C000FA8B0D94800E0C94E5650C942E970C948C
:1001D000B1190C947BD80C9492E10C9437280C94B0
:1001E0001F9E0C94FC640C9420630C94123E0C949F
:1001F00099EE0C941BA80D94840F0C94F5590C9453
:10020000AA8D0D948C0F0C9438750C94A1190D9433
:100210009E0F0D94780B0C94492A0C9404A60C9410
:10022000BCEE0C948E7A0D94C8150C940ACD0C94E7
:1002300022C40C94EE400C9439DA0C9486B40C94DD
:10024000B3A40C94ECD90C9461960C9495DC0C94AA
:10025000661F0C9435630C9444620C9497610C9463
:100260009E8C0C946EED0D94D3000C9414640C943D
:10027000A41A0C9424EF0C94012B0C9411DC0C9414
:1002800047250C94BE760C948E250C948DD90C9435
:10029000F6B60C94536F0C9457CC0C94F08D0C94D0
:1002A000FBD90C94E6DA0C94501E0C94832C0D941C
:1002B0001E240C949D190C942C650C94AA6E0C941D
:1002C0006C280C944D1A0C9467380C944C2C0C949C
:1002D0002BDB0C9443A70C94F9A60C9416AC0C944D
:1002E000A8E00C94F88D0C94B61B0C942D290D9459
:1002F000C10F0C94ED2B0C9435D80C94E4240C9481
:100300008BDB0C944B290D949C0A0C94AD340C940B
:1003100000290C94A3D60C94D4650C947CD80C942E
:1003200018B60C94B6250D94A30A0C94F0180C94EE
:10033000E7190C9445A70C94791B0C94B5190C94EF
:10034000029A0D94F30F0C94FD2B0C94332A0C9409
:10035000D4330C94D9F10C94058D0C94D9230C94BE
:10036000904D0C9431DC0C9439EA0C9427A30C9436
:10037000192B0C9464380C94781C0C9453200C9416
:10038000EADA0C94866F0C94298D0C94F9CC0C94B9
:10039000CF260C9461380C94F48D0C9469280D943C
:1003A0005E0B0C9482270C9482620C94ED640C9486
:1003B000FA640D94660F0C94C6650C94B1620C94AB
:1003C000A3390D94AF0E0C94B9B50C940A1A0C9481
:1003D0008F8C0D94B4000C944A1A0C945C1A0C94F3
:1003E000EB540C9456C90C94D8C30C94F1220C9481
:1003F000BC600C94B38C0C9433A80C941A750C94B8
:1004000001F60C9433390C9483CF0C94672C0C9424
:10041000D2D80C9429EB0C94FF8C0C948DF50C9491
:1004200007960C94A5190D94870A0C9453B60D9455
:10043000100C0D94940F0C9484610C944AB40D9498
:10044000B20F0C94F2270C94BDA30C94F78B0D946F
:10045000590F0C944BEE0C94BB640C94D5350C9452
:1004600015660C94C6270C945E380C9450640C945A
:10047000374D0C9473390C94C9340C9483DA0C9472
:10048000C6AC0C94C1680C94F6230C94E6D80C947A
:1004900098C40C94B9650C94BB740C9446910C945C
:1004A000DC730D94790A0C9416250D94A10E0C940E
:1004B0007AD80D94970E0C9417AC0C94CA1F0C9418
:1004C000FADA0C94268D0C94621C0C946F260C9412
:1004D00062740C9421910C94ED740D94700F0D9432
:1004E000BC1C0C9410750C9494EA0C946B8D0C94B9
:1004F00026290C944CA60C94331A0C94A29D0C94AF
:10050000FF330C94C7AC0C94C3330C9449DC0C94AB
:1005100061620D94CB0F0C94E0280C9403370C947B
:1005200081B30C94A9190C94E0650D94D50F0C942B
:10053000DB8C0C94EA230C94FA8D0C94FC8D0C94B7
:1005400045390C9431640C945E250C94F28D0D9415
:10055000490C0C94C5960C94D2380C94F8280C9441
:1005600031B60C9422BD0C94D1640C94FDC30C9450
:10057000F1190C9471DA0C94D4740C94E8A60D94CF
:10058000B7150C946A960C947B920C94FE8D0C9487
:100590008FA60C94C9B60C940CDB0C94D5260C9445
:1005A00037DB0C943B3D0C942E640C9486390C94F0
:1005B000AD390C94887A0C946F370C94E0330C941A
:1005C000DC230C9414AC0C945CC40C94041A0C94AE
:1005D000B5DB0C9453EB0C94E7230C94CD250C94D1
:1005E000FECC0C9409260C94F9270C94018C0C94E5
:1005F00023B70C9414DB0D94A5000C94028E0C947C
:1006000034200C94028D0D948C000C94201A0C94C0
:1006100047DA0C94491A0C94F68D0C949F650C944F
:100620005E340C94ADA60C94A3230D946E0E0C9422
:1006300064EE0C948CDB0C948ADA0D94DF0F0C942E
:10064000796E0C9472ED0C94B6230C940D1A0C94E4
:100650004E390C943C290C94F6260C9499390C9440
:100660003C390C9430340C94E2DB0C94C7190D9493
:1006700093000D94A80F0C948D1A0C94EA900C948E
:10068000AEDB0C94F2EE0C9476370C94C8AC0C9460
:100690003FA70C94DD2A0C9406370C94B9DA0D941C
:1006A000A50E0D947C0E0C94DAED0C9437C40C94CA
:1006B000BD940D948E0A0C9446210C9480AC0D943C
:1006C0007A0F0C9446950C9451EA0C941D2A0C94C4
:1006D00015AC0C94E9280C942B2B0C94345F0C94DF
:1006E000081A0C94802B0C94AD190C948ADB0C9492
:1006F000E7180C942D990D94E90F0C947DD80C9467
:10070000C91B0D94A90E0C944BC40D94780E0C9437
:1007100040340C94BC760C94C18C0D946F0B0C94EB
:100720002FA70C94D0DA0C943F8D0C94D88C0C9499
:1007300028260C94008E0C944E650D94830E0C9418
:100740009BDB0D948F0B0C94E3AB0D94890E0C94F2
:1007500024750C94282A0C94621F0C94F3650D9454
:10076000740E0C94196F0C940AB20D94FE0B0C9439
:10077000BFB30C9415DB0C9474C40C949D730C944F
:100780008A1D0D94930E0D94EA000C9476910C94AE
:1007900047A70C94DB620C944CF20C94F5B90C94C2
:1007A000539C0C9451F50D94C5150D94800A0C942E
:1007B000555A0D949B0E0C940E980C94FC8C0C9432
:1007C00027740C9498B40C947F7A0C94B6C30C9450
:1007D0008F230C9420DD0C9440D90C9464E80C9485
:1007E000F4D40C943BAE0C9495650C946EA80C94C8
:1007F00053340C94CD230C940C370C94C2760D9486
:10080000AE0E0C943F260C9476650C9461A70D9463
:10081000B6150C9407290C94641F0C949C740C94CA
:100820008A5B0C94F4D80C9433290C946AA60C942B
:10083000B8960C9446640C94B71A0C94AE3B0C9486
:100840004D620C9411950C94BF620C9461650C94EC
:1008500000200D94B30E0C94C3D80C94AF390C94B3
:1008600035DB0C94DB180C9425A80D948D0E0C949C
:100870001DA10C942E230C94559D0C94F9630C949B
:100880006A660C946C380C9418DA0C94348D0C94C1
:10089000422A0C94095A0C94383D0C940AEB0C949F
:1008A00042CC0C94048E4E414E494E495459494E07
:1008B00046CDCCCC3D0AD7233C17B7D13877CC2BCB
:1008C000329595E6241FB14F0A000020410000C870
:1008D0004200401C4620BCBE4CCA1B0E5AAEC59DF1
:1008E000746364696E6F70737578585B00556E6BD6
:1008F0006E6F776E207375666669782000556E6B33
:100900006E6F776E20636D642000636C7243747247
:100910003A2000454F46002F00496E3A200025003E
:10092000C2B04320483D00204448543232207479FC
:1009300070652E20543D00494E3A00204E6F2065D0
:100940006D69742064617461210020436F756E7459
:10095000657220747970652E2076616C3D00494E79
:100960003A0020436F756E74657220747970652E3D
:1009700020494E434F525245435420496E7465728C
:1009800072757074206E756D626572212121004947
:1009900052513A002D3E00200023002D3E00200041
:1009A00050656E6465643A2023003D00494E3A006C
:1009B0003D004C454741435920494E3A0020666F5F
:1009C0007220286D73293A004354524C3A205363E5
:1009D000686564756C6520636D642000206D73200C
:1009E0003A0041726D656420666F72200020446990
:1009F0007361726D6564002074696D653A004354DB
:100A0000524C3A205265733A002054533A00205415
:100A10003A00544845524D3A00436C65616E696E28
:100A20006720616C61726D20003D0050696E3A0074
:100A30004354524C3A20436F6D6D616E6420626C7A
:100A40006F636B65642062792064726976657220D9
:100A50006F72206368616E6E656C2066726F7A6576
:100A60006E004354524C3A204F4E3A416C726561CD
:100A70006479204163746976650A004354524C3AA4
:100A80002048414C543A416C726561647920496E4A
:100A90006163746976650A004354524C3A20584F9A
:100AA0004E3A2044697361626C65640A0043545293
:100AB0004C3A20584F4E3A416C726561647920413E
:100AC00063746976650A004354524C3A20584F4685
:100AD0004620736B69707065642E205072657620B5
:100AE000636D643A004354524C3A205475726E65FB
:100AF00064206F66662066726F6D3A004354524CF4
:100B00003A20526573746F7265642066726F6D3A35
:100B1000004354524C3A2049676E6F7265642C2032
:100B20006368616E6E656C20636D643D002045787E
:100B300065633A004354524C3A20416374697665C8
:100B40003A004354524C3A2048414C543A416C725A
:100B50006561647920496E6163746976650A004352
:100B600054524C3A20584F4E3A2044697361626C9B
:100B700065640A004354524C3A20584F4E3A416C37
:100B80007265616479204163746976650A00435433
:100B9000524C3A20584F464620736B69707065641A
:100BA0002E205072657620636D643A004354524C97
:100BB0003A205475726E6564206F66662066726FA7
:100BC0006D3A004354524C3A20526573746F72650B
:100BD000642066726F6D3A004354524C3A204E6F57
:100BE0007420656E6F756768206D656D6F72792012
:100BF000666F722067726F7570206F7065726174B6
:100C0000696F6E00496E76616C696420617267007D
:100C1000496E76616C696420617267004354524C7E
:100C20003A20556E6B6E6F776E20737566666978C5
:100C300000536B697070656420686F6D696520731F
:100C400074756666002000205375623D002049746B
:100C5000656D3D004354524C3A2052414D3D004396
:100C600054524C3A204F75744F664D656D6F7279D2
:100C70003A2000282D292000282B292000207661E9
:100C80006C7565206973200020756E6B6E6F776ED2
:100C90000A005D3D005B0020696E76616C6964004E
:100CA00020004143544956453A00206F6B003A00FA
:100CB000206661696C6564003A00526574727969F6
:100CC0006E6720564354454D5020434D440A005210
:100CD00065747279696E6720564320434D440A005B
:100CE0005265747279696E67206D6F6462757320E6
:100CF000434D440A005265747279696E6720434D12
:100D0000440A00206572726F723D004D423A2070B5
:100D10006F6C6C696E6720002056616C3A20004D44
:100D2000423A20004D423A204E6F74207375707025
:100D30006F727465642072656720747970650A004B
:100D40004D423A20706F6C6C696E672064696D6DFE
:100D5000657220004D423A20496C6C6567616C20D9
:100D6000617267756D656E74730A00206572726FCB
:100D7000723D004D423A20706F6C6C696E67205076
:100D80004920002D004D423A2050492056616C20E8
:100D90003A004D423A20706F6C6C696E6720504982
:100DA00020004D423A20706F6C6C696E6720464D92
:100DB000206661756C742000206572726F723D0050
:100DC0004D423A20706F6C6C696E6720002D004DAB
:100DD000423A20464D2056616C203A004D423A205E
:100DE000706F6C6C696E6720464D20004354524C06
:100DF0002F706F6C6C3A204F75744F664D656D6F38
:100E000072793A2000207365632072656D61696EA6
:100E1000696E6700537461747573206465666665F6
:100E20007265640A002D3E005075623A20002D3E26
:100E3000005075623A20002D3E005075623A200045
:100E40000000000000636D640000736574000076AC
:100E5000616C000064656C00004853560000524706
:100E600042000066616E00006D6F6465006374721D
:100E70006C006875650000736174000074656D70C6
:100E80000072617700002D3E005075623A20002DFF
:100E90003E005075623A200053454E44535441542D
:100EA00055533A20556E6B6E6F776E20636D6420DC
:100EB0000A000000000000000000004F4E0000008B
:100EC000000000004F46460000000000005245535D
:100ED000540000000000544F47474C4500000048B4
:100EE000414C540000000000584F4E00000000002C
:100EF00000584F46460000000000494E435245410D
:100F0000534500444543524541534500454E4142F7
:100F10004C4500000044495341424C450000554EA9
:100F2000465245455A4500465245455A450000003F
:100F30004155544F000000000046414E5F4F4E4C5B
:100F400059004849474800000000004D45444955B4
:100F50004D0000004C4F5700000000000048454184
:100F6000540000000000434F4F4C000000000044BC
:100F7000525900000000000053544F500000000080
:100F80000052474200000000000048535600000095
:100F9000000000206661696C65643A004D6F646210
:100FA0007573206F7020004D423A206F6B003D003A
:100FB0004D423A205643230020636D643D003D00BE
:100FC0004D423A2056435F6865617423004D423AB2
:100FD000204E6F7420737570706F72746564207228
:100FE000656720747970650A002056616C3A307824
:100FF0000020543A00205265673A3078004D423A5A
:1010000020416464723A00444D5800000000000022
:10101000444D58524742570000444D5852474200F1
:10102000000050574D0000000000004D4255534451
:10103000494D0000544845524D4F00000052454C68
:1010400041590000000047524F5550000000005623
:101050004354454D500000004D4255535643000047
:10106000004143484149455200005350494C4544D2
:101070000000004D4F544F52000000005049440002
:1010800000000000004D4255530000000000554193
:101090005254425244470052454C415950574D001A
:1010A000444D5852474257570056454E545300003E
:1010B0000000454C455641544F5200434F554E5445
:1010C0004552000048554D0000000000004D4552BB
:1010D00043555259000020002D3E00436F6E766547
:1010E0007274696E6720002D3E0057726F6E672024
:1010F00041737369676E6D656E7420005247427864
:101100003A200020764C6576656C3A0020436F6E7D
:1011100076563A0020436F6E76533A0020486F743B
:101120003A00436F6C643A0020436F6E76657274C8
:10113000656420563A00436F6E766572746564206C
:10114000533A002D3E0057726F6E672041737369EA
:10115000676E6D656E7420002D3E0057726F6E676E
:101160002041737369676E6D656E74200000000026
:101170000000000000004F4E000000000000004F83
:101180004646000000000000524553540000000095
:1011900000544F47474C4500000048414C54000064
:1011A000000000584F4E000000000000584F464617
:1011B0000000000000494E4352454153450044455C
:1011C00043524541534500454E41424C45000000C5
:1011D00044495341424C450000554E465245455AFC
:1011E0004500465245455A450000004155544F00C0
:1011F0000000000046414E5F4F4E4C5900484947A1
:101200004800000000004D454449554D0000004C89
:101210004F57000000000000484541540000000006
:1012200000434F4F4C0000000000445259000000A2
:1012300000000053544F500000000000524742008D
:10124000000000000048535600000000000020533A
:101250007566663A002041543A00206973200044C4
:10126000656C6574696E6720636F6E662E205241EF
:101270004D207761733A0053746F70706564006E2F
:101280006F7468696E6720746F2073746F70005399
:10129000746F7070696E67206368616E6E656C73E1
:1012A000202E2E2E0043616E206E6F7420636C65BD
:1012B000616E202D206C6F636B6564004D5154543A
:1012C0003A20436F6D706C6574652E2052656D6FAA
:1012D000766520746F706963200024636F6D6D61A3
:1012E0006E64004D5154543A20436C65616E5570E4
:1012F0002072657461696E656420746F7069632023
:1013000000220022004F75744F664D656D6F727933
:1013100021005D20003A5B004D5154543A005D00BD
:10132000456D7074793A205B000A003A004D4143E4
:101330003A00476F7420495020616464726573738A
:101340003A00276970205B69705B2C646E735B2CBC
:1013500067775B2C7375626E65745D5D5D5D2720DC
:101360002D20736574207374617469632049500A79
:10137000004661696C656420746F20636F6E6669F6
:10138000677572652045746865726E657420757343
:10139000696E6720444843502E20596F7520636161
:1013A0006E20736574206970206D616E75616C6C60
:1013B000792100204D41534B3A002047573A0020F5
:1013C000444E533A004C6F616465642066726F6DE1
:1013D00020666C6173682049503A000A7573657322
:1013E00020444843500A005374617274696E672048
:1013F0006C616E004D5154543A2074727969796E63
:1014000067206E656E78742062726F6B6572004D36
:101410005154543A20546F6F206D616E7920636F80
:101420006E6E656374696F6E206572726F72732E73
:101430002052657374617274204C414E00207472A6
:101440007920616761696E20696E2035207365635C
:101450006F6E6473004D5154543A206661696C6537
:10146000642C2072633D004D5154543A2041776101
:101470006974696E6720666F722072657461696E47
:10148000656420746F7069637300636F6E6E65636B
:101490007465642061732000202E2E2E0020757349
:1014A00065723A003A000A4D5154543A204174741E
:1014B000656D7074696E6720636F6E6E65637469C5
:1014C0006F6E20746F2000646973636F6E6E656366
:1014D000746564005573696E67204D5154542070D3
:1014E000617373776F72642066726F6D20636F6EC5
:1014F00066696700446576696365204E616D653A8B
:10150000004D5154543A204174206C65617374202D
:10151000646576696365206E616D6520616E642027
:1015200062726F6B6572204950206D757374206212
:101530006520636F6E6669677572656400246E6FFF
:10154000646573004F4E2C4F46462C48414C542C3A
:10155000524553542C584F4E2C584F46462C544FFE
:1015600047474C450024666F726D617400656E7567
:101570006D0024646174617479706500687376002D
:10158000636F6C6F7200302D32353500696E746593
:1015900067657200666C6F617400332E302E310007
:1015A00024686F6D696500757074696D652C66726D
:1015B00065656865617000653231353431615F326F
:1015C0003032342D30382D3232004C69676874481F
:1015D00075622000246E616D6500526562696E64FB
:1015E00020737563636573732E20495020616464B2
:1015F000726573733A004572726F723A2072656257
:10160000696E64206661696C0052656E6577656419
:1016100020737563636573732E2049502061646481
:10162000726573733A004572726F723A2072656E1A
:1016300065776564206661696C000A4E6F206C698D
:101640006E6B00436F6E74696E75652077697468A0
:101650002070726576696F75736C79206C6F616448
:10166000656420636F6E666967003330732045459B
:1016700050524F4D206973206E6F742072656C6FED
:10168000616465642E205265626F6F74004D515421
:10169000543A20416363657074696E6720636F6DAF
:1016A0006D616E64732E2E2E0A004E6F204D5154C4
:1016B0005420636F6E66696775726564004C6F6174
:1016C00064696E6720636F6E6669672066726F6D0E
:1016D00020706F7274616C2064697361626C656400
:1016E0002E2075736520676574204F4E20746F201F
:1016F000656E61626C6500436F6E66696720697331
:101700002076616C696400436F6E74696E75652044
:10171000776974682070726576696F75736C79206B
:101720006C6F6164656420636F6E66696700536502
:10173000747570204F5441004D5154543A207365D4
:10174000742066697273742062726F6B65720043F5
:10175000757272656E74204C414E20636F6E6669BF
:10176000672869702C646E732C67772C7375626EB2
:101770006574293A000A557365207468657365209D
:10178000636F6D6D616E64733A202768656C7027B6
:10179000202D207468697320746578740A276D6140
:1017A000632064653A61643A62653A65663A6665E3
:1017B0003A3030272073657420616E642073746F33
:1017C0007265204D41432D616464726573732069B5
:1017D0006E20454550524F4D0A276970205B697055
:1017E0005B2C646E735B2C67775B2C7375626E6524
:1017F000745D5D5D5D27202D2073657420737461B9
:101800007469632049500A277361766527202D206B
:10181000736176652063757272656E7420636F6E96
:1018200066696720696E204E5652414D3B204F4EEF
:101830007C4F4646202D20656E61626C652F646981
:101840007361626C65206175746F736176650A27D8
:1018500067657427205B636F6E66696720616464E7
:10186000725D27202D2067657420636F6E6669673F
:101870002066726F6D207072652D636F6E6669678A
:10188000757265642055524C20616E642073746FCC
:10189000726520616464722C204F4E7C4F46462056
:1018A0002D20656E61626C652F64697361626C6581
:1018B00020646F776E6C6F6164206F6E207374614B
:1018C000727475700A276C6F616427202D206C6F0D
:1018D000616420636F6E6669672066726F6D204E6B
:1018E0005652414D0A2770776427202D2064656683
:1018F000696E6520616E642073746F7265204D514E
:1019000054542070617373776F72640A276F746127
:1019100070776427202D20646566696E6520616E8E
:10192000642073746F7265204854545020415049AC
:101930002070617373776F72640A276C6F67205B26
:1019400073657269616C5F6C6F676C6576656C5D01
:10195000205B7564705F6C6F676C6576656C5D2786
:10196000202D20646566696E65206C6F67206C654C
:1019700076656C2028302E2E37290A276B696C6C0F
:1019800027202D2074657374207761746368646FF9
:10199000670A27636C65617227202D20636C65617F
:1019A0007220454550524F4D0A2773656172636836
:1019B00027202D2073656172636820312D7769724D
:1019C00065206465760A277265626F6F7427202D23
:1019D000207265626F6F7420636F6E74726F6C6CCF
:1019E000657200536F6674207265626F6F74696E02
:1019F000672E2E2E00206E6577002069732000313F
:101A000057543A003157543A2053656172636869FC
:101A10006E67206465760052414D3D000A312D7796
:101A200069726520000A6D71747420000A6D6F641C
:101A3000627573207632000A6D6F6462757320766A
:101A40003120282B29000A696E7075747320000AF2
:101A50006974656D7320000A436F6E6669677572FD
:101A600065643A00496E697469616C697A696E6788
:101A700020496E70757473003157543A2073657441
:101A80007570207265736F6C7574696F6E200031AC
:101A900057543A204453323438322D313030206E8E
:101AA0006F742070726573656E74003157543A20FC
:101AB0004453323438322D31303020493243207291
:101AC0006573746F726564003157543A20427573C0
:101AD000207265736574206572726F72003157549D
:101AE0003A2042757320526573657420646F6E6589
:101AF000003157543A204453323438322D3130308B
:101B00002070726573656E742C2072657365740045
:101B10004572726F7220312D7720696E69740031C1
:101B200057543A204453323438325F3130305F49B1
:101B300032435F544F5F31575F425249444745201B
:101B4000696E697400444D584F75742E2046726555
:101B5000653A00444D58696E20427566666572208C
:101B6000616C6C6F632065727200496E69742069E4
:101B70006E2063683A003B003D0050696E3A003BBE
:101B8000003D4C4F5700546865726D6F3A004F6EC0
:101B90006520776972652052656164790A00467232
:101BA00065653A00444D58206F75742073746172F6
:101BB0007465642E204368616E6E656C733A200014
:101BC000444D5820696E20737461727465642E20D0
:101BD0004368616E6E656C733A0042726F6B65723A
:101BE0007320636F6E666967757265643A00417051
:101BF000706C79696E6720636F6E666967004C6F01
:101C00006164656420455441473A004E6F20737407
:101C10006F72656420636F6E666967004C6F616404
:101C200065642066726F6D20454550524F4D006CC3
:101C30006F6164206661696C6564004A534F4E2091
:101C40006465746563746564004C6F6164696E6794
:101C500020436F6E6669672066726F6D2045455040
:101C6000524F4D00436F6E666967206175746F73E4
:101C70006176653A000A5379736C6F672064656218
:101C80007567206C6576656C3A0053657269616CA6
:101C9000206465627567206C6576656C3A005361F7
:101CA0007665640A005365742064796E616D6963BA
:101CB0002049500A004F54412050617373776F726E
:101CC0006420757064617465640A004E6F20495029
:101CD0002061647265737300205361766564004C03
:101CE0006F6164696E67204854545020636F6E665C
:101CF0006967206F6E20737461727475703A0000AA
:101D000000000000000000004F4E00000000000036
:101D1000004F4646000000000000524553540000AA
:101D2000000000544F47474C4500000048414C54C8
:101D30000000000000584F4E000000000000584F07
:101D400046460000000000494E43524541534500BD
:101D5000444543524541534500454E41424C4500A0
:101D6000000044495341424C450000554E465245FF
:101D7000455A4500465245455A45000000415554D4
:101D80004F000000000046414E5F4F4E4C59004846
:101D900049474800000000004D454449554D0000AA
:101DA000004C4F570000000000004845415400001F
:101DB000000000434F4F4C00000000004452590007
:101DC000000000000053544F500000000000524734
:101DD00042000000000000485356000000000000D0
:101DE000636F756C64206E6F742070617273653AF6
:101DF0002000557064617465640A00454550524F77
:101E00004D20636C65617265640A004D5154542025
:101E100050617373776F7264207570646174656468
:101E20000A002B002D00455461673A200047657475
:101E300020455441473A2000485454502F312E3108
:101E40000025733A2025730D0A0020485454502F62
:101E5000312E310D0A486F73743A2025730D0A41F3
:101E600063636570743A202A2F2A0D0A436F6E6EE1
:101E7000656374696F6E3A20636C6F73650D0A0059
:101E800025730020000D0A00474554006661696C07
:101E9000656420746F20636F6E6E6563740A00451D
:101EA00052524F523A2053657276657220726574B1
:101EB00075726E65642000436F6E666967206E6F91
:101EC00074206368616E6765640A00446F6E652EF6
:101ED0000A00436F6E6669672070617273696E678E
:101EE000206661696C65640A004765742061626FF1
:101EF0007274656400676F7420436F6E6669670A69
:101F0000006874747020726574636F646520006685
:101F10007265652000436F6E666967205552493AC5
:101F200020687474703A2F2F002044656661756CC8
:101F30007420636F6E6669672073657276657220C0
:101F4000757365643A20006C617A79686F6D652EEF
:101F50007275000A282D2943414E000A282D294D6B
:101F6000455243555259000A282B294D554C544986
:101F700056454E54000A282B2950574D5F52454C68
:101F80004159000A282D294D444E53000A282D2975
:101F900055415254425249444745000A282D29537D
:101FA00059534C4F47000A282B29504944000A280E
:101FB0002D294D43503233303137000A282D294125
:101FC00052544E4554000A282D294F5441000A28E6
:101FD0002B29535049204C4544000A282B294D4FAA
:101FE000544F5220435452000A282B294143204881
:101FF00041494552206F6E2053657269616C320011
:102000000A282B29434353383131202620484443A2
:1020100031303830000A282B29524553544152544C
:102020005F4C414E5F4F4E5F4D5154545F4552528D
:102030004F5253000A282D294841524452455345D6
:10204000542C207573696E6720736F6674000A28BC
:102050002B29434F554E544552000A282B294448FA
:1020600054000A282B294453323438322D31303071
:10207000000A282B294F57495245000A282D294983
:10208000504D4F44425553000A282B294D4F44428E
:102090005553203078303620617420536572696161
:1020A0006C332073706565643A39363030000A2825
:1020B0002B294144414652554954204C4544000A7D
:1020C000282B29444D58000A282B2957697A6E6518
:1020D0007435313030000A282B294672656552610B
:1020E0006D207072696E74696E67000A282B29571B
:1020F00041544348444F47000A282B29434F4E542C
:10210000524F4C4C494E4F000A4669726D776172CE
:1021100065204D414320416464726573732064659A
:102120003A61643A62653A65663A66653A30370004
:102130006C617A79686F6D652E7275000A436F6EF7
:10214000666967207365727665723A0032303131A4
:1021500030334C0020432B2B2076657273696F6EF1
:102160003A00653231353431615F323032342D30EE
:10217000382D3232000A4C617A79686F6D652E72A3
:1021800075204C6967687448756220636F6E74725D
:102190006F6C6C65722000204F464600204F4E0049
:1021A0002042595041535300536176656420746F47
:1021B00020454550524F4D00536176696E6720634C
:1021C0006F6E66696720746F20454550524F4D2EE3
:1021D0002E004343533831313A20416C72656164BB
:1021E0007920696E697469616C697A65640043433A
:1021F000533831313A20496E6974206572726F72BA
:1022000020004343533831313A20496E6974004805
:102210004443313038303A20416C72656164792032
:10222000696E697469616C697A6564004465766990
:1022300063652053657269616C204E756D626572CD
:102240003D00204465766963652049443D3078004F
:102250004D616E7566616374757265722049443DA7
:10226000307800484443313038303A20496E697440
:102270002E2000432C2052483D0048444331303842
:10228000303A205374617475733D004844433130D3
:1022900038303A204E6F7420696E697469616C69D8
:1022A0007A6564004D7367496E76616C69640052AB
:1022B000656164526567496E76616C6964004D655D
:1022C00061734D6F6465496E76616C6964004D6140
:1022D00078526573697374616E63650048656174F3
:1022E00065724661756C74004865617465725375FA
:1022F00070706C79004343533831313A2045727223
:102300006F7220004343533831313A204661696C83
:10231000656420746F20676574204552524F525F88
:1023200049442072656769737465722E005D20628E
:102330006173656C696E655B005D2074564F435B2D
:102340000020434F325B006363733831313A2064BD
:10235000617461206E6F7420617661696C61626C7A
:102360006500636373383131206E6F7420696E6964
:102370007469616C697A656400203C3C0041433AB1
:10238000200041433A2053657269616C2075736582
:1023900064206279204143202D2064697361626C5E
:1023A000696E672073657269616C206C6F6767691D
:1023B0006E6720616E6420636D640041433A204F74
:1023C0007574206F66206D656D6F72790041433AB8
:1023D00020496E69743A200041433A2044652D49F2
:1023E0006E69743A20004552520041433A204F4BE7
:1023F00000203E3E200041433A200041433A205015
:102400006F6C6C696E670041433A20556E6D757450
:1024100065000000000000000000004F4E000000BA
:10242000000000004F4646000000000000524553E7
:10243000540000000000544F47474C45000000483E
:10244000414C540000000000584F4E0000000000B6
:1024500000584F46460000000000494E4352454197
:10246000534500444543524541534500454E414282
:102470004C4500000044495341424C450000554E34
:10248000465245455A4500465245455A45000000CA
:102490004155544F000000000046414E5F4F4E4CE6
:1024A00059004849474800000000004D454449553F
:1024B0004D0000004C4F570000000000004845410F
:1024C000540000000000434F4F4C00000000004447
:1024D000525900000000000053544F50000000000B
:1024E0000052474200000000000048535600000020
:1024F0000000007261770071756569740073776917
:102500006E67006C6F636B00556E6B6E6F776E203D
:102510007375666669782000556E6B6E6F776E20F6
:10252000636D642000436F756E7465723A200044D9
:102530004D582D4F757420496E69743A2000444DF2
:10254000582D4F75742073746F703A200041737367
:1025500069676E65643A00444D58206374726C3A42
:1025600020006931360001693332000275313600CE
:10257000037533320004693868000569386C000659
:10258000753868000775386C0008783130000931FB
:102590003030000A44656661756C74207365726939
:1025A000616C206D6F6465204E38312075736564F1
:1025B00000384531002600384E31000600384532DB
:1025C000002E00384E32000E00384F3100360038F1
:1025D0004F32003E00374531002400374532002C91
:1025E00000374F31003400374F32003C00374E3156
:1025F000000400374E32000C004D4255533A204D36
:102600006F646275732074656D706C617465206EA3
:102610006F7420666F756E643A20004D4255533AD0
:1026200020496E76616C69642074656D706C6174AC
:10263000652E002C002C002C002C004D4255533AE6
:1026400020636F6E666967206661696C65643A0035
:102650004D4255533A20636F6E666967206572720A
:102660006F72004D4255533A20636F6E6669672062
:102670006C6F6164656420004D4255533A204F757C
:1026800074206F66206D656D6F7279004D425553F1
:102690003A20506F6C6C696E67206572726F7220A1
:1026A000004D4255533A204E6F7420737570706F11
:1026B000727465642072656720747970650A004DD4
:1026C0004255533A206578656320004D4255534486
:1026D0003A2049676E6F726564202D2065717561BF
:1026E0006C20776974682073657474656420766102
:1026F0006C004D4255533A206578656320004D4289
:1027000055533A204164642040533A20004D4255CD
:1027100053443A204D61707065643A004D42555300
:10272000443A204E65737465644D61707065643A17
:10273000004C6173744B6E6F776E2076616C7565BB
:102740003A2000536561726368696E67207265673D
:102750003A2000206F7574206F662072616E676585
:10276000206275666665722C206665746368696EA2
:102770006700646566207265672320004D425553EB
:10278000443A20536561726368696E6720726567B9
:1027900023003A002066726F6D2074797065200006
:1027A0004D425553443A2020676F742000207661D3
:1027B0006C3A0020004D425553207265733A200058
:1027C0002076616C206E6F74206368616E6765644B
:1027D0002E20436F6E74696E7565004D4255533AF5
:1027E000003A20657175616C20746172676572745E
:1027F0002E003D004D4255533A002076616C206317
:1028000068616E6765642E004D4255533A00204E54
:102810006F773A00204C6173743A002023002070D7
:10282000726566657463682000205265672F636F68
:10283000696C206D75737420626520696E74002068
:10284000696E7465726E616C2073656E642065726A
:10285000726F72202D206E6F207265672F636F6913
:102860006C0020696E7465726E616C2073656E64B5
:10287000206572726F72202D206E6F2074656D70EE
:102880006C6174650020696E7465726E616C207392
:10289000656E64206572726F72202D206E6F2073DA
:1028A000746F7265004D425553443A20656E645012
:1028B0006F6C6C20004D425553443A20506F6C6C45
:1028C0002000206E6F7420666F756E64004D425557
:1028D000533A2020706172616D20002073656E6430
:1028E000696E672063616E63656C6C6564004D4260
:1028F00055533A2020706172616D20002073656E1F
:1029000064206572726F722E20004D4255533A203A
:1029100020004164642040563A20002056616C3A01
:1029200020004D425553443A207375666669783AE3
:1029300000206F722073756666697820004D4255DD
:10294000533A204E6F2074656D706C61746520661B
:102950006F7220004D6F746F723A2074696D656FED
:10296000757400556E6B6E6F776E20636D64004DED
:102970006F746F723A20466F726365642065786584
:10298000637574696F6E0056454E543A20636F6EDE
:10299000666967206661696C65640056454E543A05
:1029A00020696E69740056454E543A2044652D499D
:1029B0006E697400204F75743A00205265713A00B8
:1029C00056454E543A2000206D33002066726F6DDC
:1029D0002000204D6178207265713A002066616E9A
:1029E000253A002061637469766520563A005645A1
:1029F0004E543A20546F74616C20563A005049444A
:102A00003A20616C726561647920696E69746961EC
:102A10006C697A6564005049443A20496E76616C6D
:102A2000696420706172616D2061727261792E003B
:102A30002C002C002C002C005049443A20636F6E6F
:102A4000666967206661696C65643A005049443A7A
:102A500020636F6E666967206572726F72005049FD
:102A6000443A20636F6E666967206C6F61646564C9
:102A700020005049443A204F7574206F66206D65E0
:102A80006D6F7279005049443A2044652D496E6952
:102A9000742000203C414C4D3E0020443A00204927
:102AA0003A0020503A0020696E3A00207365743A6B
:102AB000005049443A20005049443A20496E76611A
:102AC0006C696420706172616D2061727261792E2F
:102AD00000536574206F757420746F200020504976
:102AE0004420616C61726D2E2000205049442061A9
:102AF0006C61726D3A20636C6F7365640050494479
:102B00003A20556E6B6E6F776E20737566666978C6
:102B100020005049443A20556E6B6E6F776E2063EB
:102B20006D64200020536574706F696E743A0050B4
:102B300049443A200020496E7075742076616C75A6
:102B4000653A005049443A200020696E69740020BB
:102B50000050574D2D4F75742023002073746F70F3
:102B600000200050574D2D4F75742023003D00501C
:102B7000696E3A0020696E69740052656C61792D46
:102B80004F75742023002073746F700052656C6160
:102B9000792D4F75742023003D3E003A0070756218
:102BA00020616374696F6E200069646C65006F66F4
:102BB000660068656174696E670066616E006472C4
:102BC00079696E6700636F6F6C696E670020697367
:102BD00020004F75742000556E6B6E6F776E2073FA
:102BE00075666669782000556E6B6E6F776E206330
:102BF0006D642000616374696F6E0072656C617949
:102C00004374723A200053686F770020636D643D0F
:102C1000002D000000000000636D64000073657407
:102C2000000076616C000064656C0000485356003B
:102C300000524742000066616E00006D6F646500DF
:102C40006374726C006875650000736174000074D1
:102C5000656D7000726177000020002E00696E00C3
:102C6000735F6F7574006D79686F6D6500435452C2
:102C70004C2F657865633A204F75744F664D656DCE
:102C80006F72793A2000202D3E20004D5154543A65
:102C90002000202D3E2000456D69743A203C002024
:102CA0002D3E20004974656D436D643A2000202D4F
:102CB0003E20004974656D3A20003157543A204255
:102CC0007573207265736574206572726F7200315E
:102CD00057543A2042757320526573657420646FAF
:102CE0006E65003157543A204453323438322070E4
:102CF000726573656E742C20726573657400493259
:102D00004320526573657400005EBCE2613FDD8361
:102D1000C29C7E20A3FD1F419DC3217FFCA2401EBB
:102D20005F01E3BD3E6082DC237D9FC1421CFEA0AB
:102D3000E1BF5D0380DE3C62BEE0025CDF81633D9B
:102D40007C22C09E1D43A1FF4618FAA427799BC58B
:102D500084DA3866E5BB5907DB856739BAE406587B
:102D60001947A5FB7826C49A653BD987045AB8E66B
:102D7000A7F91B45C6987A24F8A6441A99C7257B5B
:102D80003A6486D85B05E7B98CD2306EEDB3510F4B
:102D90004E10F2AC2F7193CD114FADF3702ECC923B
:102DA000D38D6F31B2EC0E50AFF1134DCE90722C2B
:102DB0006D33D18F0C52B0EE326C8ED0530DEFB11B
:102DC000F0AE4C1291CF2D73CA947628ABF517490B
:102DD0000856B4EA6937D58B5709EBB536688AD4FB
:102DE00095CB2977F4AA4816E9B7550B88D6346AEB
:102DF0002B7597C94A14F6A8742AC896154BA9F7DB
:102E0000B6E80A54D7896B35436F6E6E6563746597
:102E1000642E00436F6E6E2E2061626F7274656463
:102E2000003E3E2000496E76616C696420636F6DE0
:102E30006D616E6400000020002300260029002C34
:102E4000002F003200000100000301060109013ECD
:102E50003E3E004E6F204D414320636F6E666967B2
:102E6000757265643A20736574206669726D776166
:102E700072652773204D41430A00454550524F4D1E
:102E8000207369676E6174757265206F6B00496E9F
:102E9000697469616C697A696E6720454550524F63
:102EA0004D2E002072656164206572726F7220661B
:102EB0006F7220003E2000203C003157543A003110
:102EC00057543A206E6F7420696E697400315754FC
:102ED0003A20425553592074696D656F75740031FD
:102EE00057543A204453323438325F4552524F528D
:102EF0005F434F4E464947003157543A20312D77B2
:102F00006972652073686F727465640072656164CC
:102F1000790024737461746500757074696D65005F
:102F2000667265656865617000247374617473000E
:102F300020457870697265640A00202D746172679B
:102F40006574207A6F6E652D0020416C61726D2072
:102F5000457870697265640A0020636D643A0020E8
:102F60004375723A00205365743A002054696D65C8
:102F7000723A00204C6F636B733A0052414D3D0032
:102F800000002200250028002B002E003100340014
:102F900002010000050108010B0100000A0B0209F3
:102FA0000C0D0E08070304010000000000000000E3
:102FB0000000000000000000000000000000000011
:102FC00000000000000012111000000000000000CE
:102FD00000000000000000000000000000000000F1
:102FE00000002100240027002A002D0030003300BB
:102FF00001010000040107010A010102102020085C
:103000000810204010204080020102010804020143
:1030100001020408102040808040201008040201B2
:10302000800402018040201008040201080402010B
:103030000102040810204080010204081020408092
:1030400005050505070508080808020202020A0A24
:103050000808040404040101010101010101030342
:10306000030303030303040707070C0C0C0C0C0CED
:103070000C0C0202020206060606060606060B0BEA
:103080000B0B0B0B0B0B556E7370656369666965F3
:1030900064206572726F722E0047454E4552494357
:1030A0005F4552524F5200494E5445524E414C5F7B
:1030B0004552524F52004932435F4552524F5200DF
:1030C00049445F4552524F52005355434345535371
:1030D000004343533831313A200057726F6E6720F6
:1030E0007061796C6164004D5154543A20435452DC
:1030F0004C2F7478743A204F75744F664D656D6F20
:1031000072793A2000202D3E2041543A00436861F4
:103110006E20747970653A004E6F2073746F72651B
:10312000642076616C756573202D20646566617519
:103130006C743A2000536176656420455441473AE7
:103140000053657420455441473A200057016F02EF
:1031500011241FBECFEFD1E2DEBFCDBF00E00CBF18
:1031600019E0A0E0B2E0E4E2F5E702E00BBF02C044
:1031700007900D92AC3AB107D9F720E1ACEAB9E07B
:1031800001C01D92AF3AB207E1F718E1C7EAD8E1F2
:1031900000E006C021970109802FFE010F945632EE
:1031A000C63AD10780E00807A9F70F94C61C0D9412
:1031B000803A0C940000E5E0F1E080818F79808313
:1031C0000895E5E0F1E080818066808308958FE0D6
:1031D00090E09093AC0A8093AB0A88EC90E008955D
:1031E000FC01848195810895DC011896ED91FC9194
:1031F000309739F080858F70823019F486819781FD
:10320000089590E080E00895FC01A681B7811097B1
:1032100021F118969C9118979F708EEF890F82303C
:1032200010F091111AC019964D935D936D937C9394
:103230001C97A681B78118969C911897907F9260F1
:1032400018969C930680F781E02D8085982F907FBB
:10325000903619F48F70806A80870895FC0123816D
:1032600030E090E080E0FC01EE0FFF1FE951F64FE7
:10327000A081B181A217B30761F4880F991F880F4D
:10328000991FFC01ED52F64F408351836283738393
:103290000895A081B181AB2B19F420813181EDCF4C
:1032A000019685309105F9F60895FC01238130E0FF
:1032B00090E080E0FC01EE0FFF1FE951F64F4081E6
:1032C00051814217530761F4880F991F880F991F86
:1032D000FC01ED52F64F60817181828193810895E6
:1032E00040815181452B89F431832083880F991FB8
:1032F000880F991FFC01ED52F64F10821182128245
:10330000138260E070E0CB0108950196853091054D
:1033100089F6F7CF880F991F880F991FFC01E55494
:10332000F64F80819181A281B3810196A11DB11DCB
:1033300080839183A283B383089585E090E00C9409
:103340008A1984E090E00C948A1983E090E00C9450
:103350008A1982E090E00C948A1981E090E00C9444
:103360008A1990E080E00C948A19CF93DF93EC01E6
:10337000E881F9810484F585E02D199529893A8938
:103380002F5F3F4F3A8B298BDF91CF910895CF93D9
:10339000DF93EC018E8581110DC081E090E04989B9
:1033A0005A892C853D854217530708F080E0DF914C
:1033B000CF910895E881F9810484F585E02DCE014F
:1033C00019958F3F910549F780E090E0F0CFFC011F
:1033D000848595856817790708F4CB01928B818BDA
:1033E0000895CF93DF93FC012685222351F0EC0151
:1033F0000190F081E02D0190F081E02D6FEF1995A3
:103400001E86DF91CF910895FC01878590890895EC
:1034100081E0089590E080E00895DC011296ED913E
:10342000FC91309761F00280F381E02D309739F004
:10343000862F8295807F60856F70682B60870895E6
:10344000DC011296ED91FC91309751F00280F381EE
:10345000E02D309729F0808582958F7090E0089557
:1034600090E080E008950F931F93CF93DF9300D0F7
:1034700000D01F921F92CDB7DEB781E028960FB61D
:10348000F894DEBF0FBECDBFDF91CF911F910F919A
:103490000895089590E080E00895A89582E090E076
:1034A0000C9453AD62E27EE1811102C064E27EE1E0
:1034B0008AE09FE00C94EAE163EE79E18AE09FE024
:1034C0000E94EAE1F0E0E0E0199584EF91E00895D0
:1034D00080916A0A8823B1F0E0916B0AF0916C0A3E
:1034E000309731F0868197819093690A8093680ABA
:1034F00068E377E18AE09FE00E94EAE18AE09FE0EA
:103500000C947EE0089568E77CE0811102C063E7D7
:103510007CE087EB9FE00C94EAE1DC0155962C916E
:103520005597273781F4ED91FC91008CF18DE02DBA
:10353000199563E179E087EB9FE00E94EAE187EB70
:103540009FE00C947EE00895892B71F0FB0182814D
:1035500093810F947F016BE07EE18AE09FE00E94FF
:10356000EAE188EC90E0089590E080E0F2CF0F93DC
:103570001F93CF93DF93EB0102970CF4A0C00A8155
:103580001B8168E07DE1C8010F94A72A892B61F4B3
:103590000F94E5036F7E0F943F0488EC90E0DF9179
:1035A000CF911F910F91089561E17DE1C8010F94C2
:1035B000A72A892B21F40F94E5036061ECCF6FED0E
:1035C0007CE18AE09FE00E94EAE10F94E5036295C6
:1035D000617081E0682770E04AE050E08AE09FE097
:1035E0000E948BE18AE09FE00E947EE08091E60EDF
:1035F0009091E70E892B09F452C00A811B810F9428
:103600000001882309F44BC0F80101900020E9F77C
:103610003197E01BF10BB09708F041C0A091E60E86
:10362000B091E70E52961C921E92519754961C929E
:103630001E92539784E890E01D969C938E931C975E
:103640001E961C921E9782E755968C935597ED9186
:10365000FC9111970088F189E02D60E270E0CD01C6
:103660001995B8018091E60E9091E70E0E94D4E181
:103670008091E60E9091E70EDC01ED91FC910190B6
:10368000F081E02D60E019958091E60E9091E70EB3
:10369000DC01ED91FC910488F589E02D19956A8192
:1036A0007B818AE09FE00E94D4E168ED7CE18AE0C2
:1036B0009FE00E94EAE18AE09FE00E947EE0809124
:1036C000AB0A9091AC0A02973CF080EF9FEF909389
:1036D000AC0A8093AB0A61CF6BEC7CE182E19FE0A6
:1036E0000E94EAE182E19FE00E947EE084EF91E0A7
:1036F00056CFCF93DF93EB010297ACF168E07DE109
:103700008A819B810F94A72A892B29F40F94E503C2
:103710007E7F0F943F0461E17DE18A819B810F945C
:10372000A72A892B29F40F94E50371600F943F04B5
:1037300064E67CE18AE09FE00E94EAE10F94E50301
:10374000672F609561704AE050E070E08AE09FE08A
:103750000E948BE18AE09FE00E947EE088EC90E08E
:10376000DF91CF9108950E94C9ACF8CF892B71F0F9
:10377000FB01828193810F94E00165EB7CE18AE09B
:103780009FE00E94EAE188EC90E0089590E080E0FC
:10379000F2CFEF92FF920F931F93CF93DF93CDB7AA
:1037A000DEB72C970FB6F894DEBF0FBECDBF8C01ED
:1037B0007B0181E795E09A8389831B821C821D82AD
:1037C0001E8298878F8319861A861B861C86053071
:1037D0001105ECF0BE01695F7F4FF701808591858F
:1037E0000E9467A9892B99F0CE0107960F94AA022F
:1037F000BE01695F7F4FF701868197810E9467A9AB
:10380000892B61F0CE0107960F947C030EC0CE0188
:1038100001960F94AA020430110554F7CE010196C7
:103820000F947C0303301105A4F1BE01695F7F4F43
:10383000F701848195810E9467A9892B51F1CE01FE
:1038400007960F941303BE01695F7F4FF7018281D2
:1038500093810E9467A9892B19F1CE0107960F94D5
:1038600041026EE97CE18AE09FE00E94EAE180E0AB
:103870000F94A30488EC90E02C960FB6F894DEBF6A
:103880000FBECDBFDF91CF911F910F91FF90EF90B1
:103890000895CE0101960F941303023011059CF692
:1038A000CE0101960F94410201301105D1F6CE01EF
:1038B00001960F94410265EA7CE18AE09FE00E9454
:1038C000EAE1CFCFCF93C1E068EE73E080E090E013
:1038D0000F942A114AE050E06C2F8AE09FE00E948A
:1038E000A1E0CF5FC43181F784EF91E0CF910895DB
:1038F0000F931F93CF93DF938C01EB010297C4F0DA
:103900008A819B810F94592A8093310299270F94C1
:10391000AC040230110549F08C819D810F94592A25
:103920008093300299270F94B604C8ECD0E002C00F
:10393000C0E9D1E06AE87CE18AE09FE00E94EAE128
:103940004AE050E0609131028AE09FE00E94A1E0ED
:1039500065E77CE18AE09FE00E94EAE14AE050E00E
:10396000609130028AE09FE00E94A1E08AE09FE03F
:103970000E947EE0CE01DF91CF911F910F910895BB
:10398000DC011496ED91FC91309771F090859F7059
:10399000923039F0953041F4CF010F94F00090E06F
:1039A000089581E090E0089590E080E00895009708
:1039B00089F0FC0120852F70253061F40F945F00A1
:1039C000009741F0FC0120852F70243019F4818587
:1039D0009285089590E080E0089565E0FC01828181
:1039E00093810F945F00009749F0FC018085982F28
:1039F000907F21F082958F7090E0089590E080E0B4
:103A000008958F929F92AF92BF92CF92DF92EF92E2
:103A1000FF920F931F93CF93DF93E091AD0AF09144
:103A2000AE0A309709F467C0812EF02E932EC22E75
:103A3000A52ED42EB72EE62EBC01CF010E94ADFFDD
:103A4000EC01892B19F481E090E057C088858F70D4
:103A50008530C9F760E0CE010F945F008C0161E012
:103A6000CE010F945F00FC01C185D285D801199663
:103A70002D913C912130310561F13CF46F2DCE0147
:103A8000232B09F70E949CF7DECF2230310531F15C
:103A900027303105C1F6892BB1F280858F708530D2
:103AA00091F6C681D781209771F288858F70843016
:103AB00061F40F2D182D2C2D392D4D2D5A2D6E2DD5
:103AC0007B2D89859A850E94011D0A80DB81C02D8E
:103AD000EACF6F2DCE0103960E949CF76E2DCE018A
:103AE0000E949CF76D2DCE0101960E949CF76C2DD3
:103AF000CE010296C7CF90E080E0DF91CF911F9179
:103B00000F91FF90EF90DF90CF90BF90AF909F907C
:103B10008F9008952F923F924F925F926F927F9273
:103B20008F929F92AF92BF92CF92DF92EF92FF92CD
:103B30000F931F93CF93DF938091640A9091650A4E
:103B4000892B09F49AC02090630A312C359427946C
:103B500035942794EE24E394F12CD0E0C0E088243F
:103B60008394912C2C163D0609F487C0C090640AFA
:103B7000D090650A24010C2E02C0440C551C0A94F6
:103B8000E2F7052C000C66087708F7013197EC0D79
:103B9000FD1D5701A4E0AA0EB11CC70160E02091F1
:103BA0002E0230912F02AC012817390720F44091E2
:103BB0002E0250912F0220919E0A30919F0A240FCD
:103BC000351FD9012C9131913217C1F04091B309C1
:103BD0005091B4096091B5097091B60944295529ED
:103BE000662977294093B3095093B4096093B509C6
:103BF0007093B609DF0111972C9361E001968A1545
:103C00009B0569F66623B1F18091660A9091670A77
:103C1000009729F1FC0120852F70253001F56C2FCC
:103C20000F945F00FC0190859F709430C1F48185F2
:103C300092850097A1F0FE01EE0FFF1FEE0FFF1F10
:103C4000EC0DFD1D038110E0228130E0EC0CFD1C29
:103C5000D7014C9150E0608170E00E94011D80E02E
:103C60000E94789B6093B7097093B8098093B90953
:103C70009093BA092196750175CFDF91CF911F916D
:103C80000F91FF90EF90DF90CF90BF90AF909F90FB
:103C90008F907F906F905F904F903F902F900895FE
:103CA000CF92DF92EF92FF920F931F93CF93DF9308
:103CB000CDB7DEB769970FB6F894DEBF0FBECDBFA4
:103CC000E091A20AF091A30A309709F483C0809191
:103CD000AF0A9091B00A892B09F47CC08FEF8387DB
:103CE000148613821482158216821782108611861A
:103CF000128664E07AE18AE09FE00E94EAE18AE0CD
:103D00009FE00E947EE08E010F5E1F4FBE016E5E3F
:103D10007F4F8091A20A9091A30A0E9403FC18167B
:103D20000CF058C0A895DE0111969E012E5E3F4F03
:103D30007D01F90141919F01842F90E054E0959518
:103D400087955A95E1F7845E9B4FFC0180818C93A7
:103D5000E42FEF70F0E0E45EFB4F808111968C93CE
:103D600011971296A017B10721F7198AB701809110
:103D7000AF0A9091B00A0E94ADFF6C016FEF79E13C
:103D80008AE09FE00E94EAE1B7018AE09FE00E949A
:103D9000D4E1C114D104B9F0C6010E94C4AB7C01C6
:103DA000892B09F4B3CF6AEF79E18AE09FE00E94A2
:103DB000EAE1B7018AE09FE00E94D4E18AE09FE057
:103DC0000E947EE0A3CF65EF79E18AE09FE00E9448
:103DD000EAE1F4CF88EC90E069960FB6F894DEBF84
:103DE0000FBECDBFDF91CF911F910F91FF90EF904C
:103DF000DF90CF900895EF92FF920F931F93CF9390
:103E0000DF930097C1F0FC0120812223A1F08C01F7
:103E100085E4E82E8EE0F82EC1E0D0E0B701C801BD
:103E20000F94C52A892B49F02196F5E0EF0EF11C7D
:103E3000CE30D10599F7D0E0C0E0CE01DF91CF912F
:103E40001F910F91FF90EF900895CF92DF92EF9224
:103E5000FF920F931F93CF93DF93CDB7DEB7C1547B
:103E6000D1090FB6F894DEBF0FBECDBF6C01AB0118
:103E700030E020E060E4CE0101967C010E947DA844
:103E8000F70101900020E9F731978F010E191F0902
:103E9000A801B701C6010F94E336892B11F010E099
:103EA00000E0C801CF5BDF4F0FB6F894DEBF0FBE56
:103EB000CDBFDF91CF911F910F91FF90EF90DF90D9
:103EC000CF9008950D9425280D942528CF92DF9248
:103ED000EF92FF920F931F93CF93DF93CDB7DEB78F
:103EE000C054D1090FB6F894DEBF0FBECDBF80918C
:103EF000AB0A9091AC0A059709F449C061157105A8
:103F000009F445C069017A018B0140E450E0CE011B
:103F100001960F94F1366FE270E0CE0101960F9496
:103F2000B836892B41F4980143E050E060E4CE01BB
:103F300001960E947DA84FE350E0B601CE010196A4
:103F40000F94D3360E94CBFF882309F18091AB0AEE
:103F50009091AC0A0697D9F48091A60A811117C0F6
:103F6000B701CE0101960F94C71381E090E0C05CC9
:103F7000DF4F0FB6F894DEBF0FBECDBFDF91CF91FC
:103F80001F910F91FF90EF90DF90CF90089590E0F8
:103F900080E0EDCFCF92DF92EF92FF920F931F93CD
:103FA000CF93DF93CDB7DEB760970FB6F894DEBF3F
:103FB0000FBECDBF7C016B01CA01B9012AE0AE0181
:103FC0004F5F5F4F0F945E2BD701ED91FC910288FC
:103FD000F389E02D9801AE014F5F5F4FB601C70135
:103FE000199560960FB6F894DEBF0FBECDBFDF9176
:103FF000CF911F910F91FF90EF90DF90CF90089598
:10400000CF92DF92EF92FF920F931F93CF93DF93A4
:10401000CDB7DEB760970FB6F894DEBF0FBECDBF49
:104020007C016B01BA01A901CE0101960E94A5A9EC
:10403000D701ED91FC910288F389E02D9801AE0142
:104040004F5F5F4FB601C701199560960FB6F894A0
:10405000DEBF0FBECDBFDF91CF911F910F91FF90BB
:10406000EF90DF90CF9008951F93CF93DF93FC01E3
:10407000162FC389D489818992899C012F5F3F4F74
:10408000328B218BC80FD91FCE010F94B93118176D
:1040900021F0612FCE010F94C13181E090E0DF91DA
:1040A000CF911F910895FC018189928924853585DE
:1040B0008217930740F423893489820F931F0F944A
:1040C000B93190E008958FEF9FEF089565E771E2B1
:1040D0008AE09FE00E94EAE162E671E28AE09FE006
:1040E0000E94EAE164E571E28AE09FE00E94EAE171
:1040F0006CE471E28AE09FE00E94EAE18AE09FE0DE
:104100000E947EE06CE371E28AE09FE00E94EAE1B7
:1041100060E371E28AE09FE00E94EAE168E071E218
:104120008AE09FE00E94EAE168EF70E28AE09FE0A7
:104130000E94EAE16BEE70E28AE09FE00E94EAE111
:1041400066ED70E28AE09FE00E94EAE167EC70E2CF
:104150008AE09FE00E94EAE16FEB70E28AE09FE074
:104160000E94EAE16EEA70E28AE09FE00E94EAE1E2
:1041700068E870E28AE09FE00E94EAE16BE770E2A3
:104180008AE09FE00E94EAE161E770E28AE09FE056
:104190000E94EAE162E670E28AE09FE00E94EAE1C2
:1041A0006AE570E28AE09FE00E94EAE16EE470E274
:1041B0008AE09FE00E94EAE164E370E28AE09FE027
:1041C0000E94EAE165E170E28AE09FE00E94EAE194
:1041D00060E070E28AE09FE00E94EAE168EE7FE141
:1041E0008AE09FE00E94EAE16AED7FE18AE09FE0D9
:1041F0000E94EAE16EEC7FE18AE09FE00E94EAE142
:1042000066EC7FE18AE09FE00E94EAE16BEB7FE1F0
:104210008AE09FE00E94EAE16EEA7FE18AE09FE0A7
:104220000E94EAE166EA7FE18AE09FE00E94EAE11B
:104230006BE97FE18AE09FE00E94EAE16CE87FE1C0
:104240008AE09FE00E94EAE163E87FE18AE09FE084
:104250000E94EAE165E77FE18AE09FE00E94EAE1EF
:1042600067E67FE18AE09FE00E94EAE16BE57FE19B
:104270008AE09FE00E94EAE163E57FE18AE09FE057
:104280000E94EAE18AE09FE00C947EE00F931F9386
:10429000CF93DF9300D000D0CDB7DEB70E94662069
:1042A0006FE477E18AE09FE00E94EAE1CE010196A7
:1042B0000F94FE0CCE0101960E9411A901E715E0B2
:1042C0001A8309838091640D9091650DA091660D0C
:1042D000B091670D8B839C83AD83BE83CE01019625
:1042E0000E9411A91A8309831B821C821D821E82CF
:1042F00080E590E00F94CD0C44E050E0BE016D5F8E
:104300007F4F81E090E00E941AE90E9411EACE01FD
:1043100001960E9411A91A8309831B821C821D82A7
:104320001E8280E590E00F94CD0C44E050E0BE0189
:104330006D5F7F4F85E090E00E941AE90E9411EACC
:10434000CE0101960E9411A965E777E18AE09FE01E
:104350000E94EAE188EC90E026960FB6F894DEBF62
:104360000FBECDBFDF91CF911F910F910895CF93D5
:10437000DF9300D000D01F921F92CDB7DEB7FC01B3
:10438000628398E0DE01119601900D929A95E1F713
:1043900029813A814B815C816D817E818F819885F5
:1043A00028960FB6F894DEBF0FBECDBFDF91CF9138
:1043B0000895CF93DF9300D000D01F921F92CDB706
:1043C000DEB7FC01608398E0DE01119601900D924A
:1043D0009A95E1F729813A814B815C816D817E81DB
:1043E0008F81988528960FB6F894DEBF0FBECDBF9B
:1043F000DF91CF9108952F923F924F925F926F92EB
:104400007F928F929F92AF92BF92CF92DF92EF9264
:10441000FF920F931F93CF93DF93CDB7DEB7A09793
:104420000FB6F894DEBF0FBECDBF8C01662E6A01B9
:10443000DC018D919C911197892B09F46AC0159626
:10444000ED91FC91309709F464C080818071BFEFD9
:104450006B1361C0D1F481E0A0960FB6F894DEBF73
:104460000FBECDBFDF91CF911F910F91FF90EF90C5
:10447000DF90CF90BF90AF909F908F907F906F9084
:104480005F904F903F902F9008954330510519F35E
:10449000618062942FE0622260EA79E087EB9FE01E
:1044A0000E94EAE14AE050E0D80113966C9187EB54
:1044B0009FE00E94A1E06EE979E087EB9FE00E9417
:1044C000EAE1D8011596ED91FC9161816F704AE0A7
:1044D00050E087EB9FE00E94A1E06BE979E087EB79
:1044E0009FE00E94EAE14AE050E0662D87EB9FE002
:1044F0000E94A1E087EB9FE00E947EE0D801159624
:10450000ED91FC9181818F70681207C080818F7E50
:10451000808380E0A1CF8111FCCF198E1A8E1B8E73
:104520001C8E1D8E1E8E1F8E18A28A8D807F8A8FF4
:10453000D8011596ED91FC9181818F708615A9F1B6
:10454000B3E0CB16D10489F169E979E087EB9FE00C
:104550000E94EAE14AE050E0F801638187EB9FE0C6
:104560000E94A1E067E979E087EB9FE00E94EAE121
:10457000D8011596ED91FC9161816F704AE050E091
:1045800087EB9FE00E94A1E064E979E087EB9FE080
:104590000E94EAE14AE050E0662D87EB9FE00E942E
:1045A000A1E087EB9FE00E947EE0F801208131814D
:1045B000FCE0F61508F41DC1E62DF0E08827EC516B
:1045C000FD4D8F4F0D945632F1222E23B623CD236D
:1045D000D923B6238F23B623DC23E723A323EA239F
:1045E000F623D8011596ED90FC90F70181818F702C
:1045F000853009F4FEC050F48230C1F061E875E006
:10460000C9010E94ADFF2C01712C4BC08730D1F045
:104610008A30A1F76AE775E0C9010E94ADFF2C015D
:10462000D7017C9072FA772470F83BC064E775E09C
:10463000C9010E94ADFF2C01D7017C9070FA77244C
:1046400070F82FC063E775E0C9010E94ADFF2C012F
:10465000F701708071FA772470F823C066E875E07E
:10466000C9010E94ADFF2C01D8011596ED91FC9176
:10467000808180FB772470F8982F9E7F80FF916067
:1046800090834114510469F461E0CE0149960E947F
:10469000D921298B3A8B4B8B5C8B6D8B7E8B8F8BCF
:1046A000988FF801E080F1806CEB75E0C7010E9403
:1046B000ADFF1C0161EC75E0C7010E94ADFF5C011C
:1046C00066EC75E0C7010E94ADFF4C01A114B10476
:1046D00081F42114310469F460E0CE0149960E940E
:1046E000D92129833A834B835C836D837E838F83B7
:1046F0009887D8011596ED91FC914114510409F069
:104700007CC0898D811179C0B62DBF706B2E8181DF
:10471000807F682A618280818F7E80839CCE6BE857
:1047200075E0C9010E94ADFF2C01D8011596ED91ED
:10473000FC91808181FB772470F8982F9D7F81FF09
:1047400092609083AECF61E975E0C9010E94ADFF30
:104750002C01D8011596ED91FC91808182FB772484
:1047600070F8982F9B7F82FF9460EBCF61E875E033
:10477000C9010E94ADFF2C01892B09F045CF62E0F1
:10478000CE0149960E94D92129873A874B875C87B9
:104790006D877E878F87988B37CF67E975E0C90172
:1047A0000E94ADFF2C01D8011596ED91FC9170800F
:1047B00045CF6CE975E0F3CF62EA75E0C9010E946C
:1047C000ADFF2C01D8011596ED91FC9142CF68EA1E
:1047D00075E0F4CF6FEA75E0C9010E94ADFF2C01CE
:1047E000D8011596ED91FC9170801CCF65EB75E0BA
:1047F000F3CF712C512C412C54CF83E0C816D10437
:10480000C1F0962D9F70692E8181807F682A618218
:1048100080818F7E80836101E98CFA8C0B8D1C8DE9
:104820002D8D3E8D4F8D58A1672DC2010E945CAE2B
:1048300012CE81818F70861509F40DCE629490EFAF
:104840006922682A61828081806167CF7F928F921E
:104850009F92AF92BF92CF92DF92EF92FF920F930F
:104860001F93CF93DF93EC014B018091F1098F5F90
:104870008093F109AB016FEFCE010E94FB218A8189
:1048800081FB002700F91B819AEC910F903110F009
:104890008730E1F56AEC75E0888199810E94ADFF6F
:1048A0007C01009799F1FC0180858F70853071F54E
:1048B0008091C50F18131DC08091C60F8034C9F4B4
:1048C0008091C70F9091C80F5C01990FCC08DD084B
:1048D00060E0C7010F945F00FC0181859285A3858C
:1048E000B485A816B906CA06DB060CF05CC0712CAC
:1048F00037C01093C50F80E48093C60F812F0F94AB
:10490000F80F9093C80F8093C70FDECF212F30E0B0
:10491000F901E656F04D8491F901E650F04D1491FD
:10492000F901E05CFF4CF490FF2009F439C08111DB
:104930000F94500EEF2DF0E0EE0FFF1FEB5CF14DEA
:10494000A591B491EC911E2331E020E009F430E010
:10495000832F922F772473940817190609F0C7CF75
:10496000F3E08F16910409F47EC0ED81FE81E181B0
:10497000EF70E150EC3008F076C0F0E08827EC539F
:10498000FB4D8F4F0D945632E4243F2616254725C4
:104990003F265E253F268E25B625CD2509262826CD
:1049A00090E080E0D7CF61E0C7010F945F007724EB
:1049B0007394FC0181859285A385B4858A159B0536
:1049C000AC05BD056CF693CF0F942A139B01AC0187
:1049D00044275527ED81FE816281738190E080E05C
:1049E000AA24AA94BA2CC12CD12C18EEE12E13E0E3
:1049F000F12E00E010E00E94B19A8823A1F1088115
:104A0000198167E975E0C8010E94ADFF892B41F467
:104A10006CE975E0C8010E94ADFF892B09F4F6C06E
:104A2000A40163E0CE010E94FB211DC00F942A1354
:104A30009B01AC0144275527ED81FE816281738182
:104A400090E080E0AA24AA94BA2CC12CD12C1CE2BC
:104A5000E12EFF24F39400E010E00E94B19AA4013B
:104A600064E0811179C0ED81FE81808183FB99270B
:104A700090F9971509F4BDC1982F907E09F41EC1D5
:104A8000982F907E90528F71892B808339C10F941B
:104A90002A139B01AC0144275527ED81FE816281D9
:104AA000738190E080E0AA24AA94BA2CC12CD12C66
:104AB00016E9E12EF12C00E010E0CFCF0F942A137D
:104AC0009B01AC0144275527ED81FE8162817381F2
:104AD00090E080E0AA24AA94BA2CC12CD12C18EE24
:104AE000E12E13E0F12E00E010E00E94B19A88233D
:104AF00009F4B9CF0881198162EA75E0C8010E9402
:104B0000ADFF892B41F468EA75E0C8010E94ADFF52
:104B1000892B09F47BC0A40168E084CF0F942A1389
:104B20009B01AC0144275527ED81FE816281738191
:104B300090E080E0AA24AA94BA2CC12CD12C1CE2CB
:104B4000E12EFF24F39400E010E00E94B19AA4014A
:104B500069E0882309F487CFCE010E94FB210F94DE
:104B60002A13ED81FE81738362837DCF0F942A1314
:104B70009B01AC0144275527ED81FE816281738141
:104B800090E080E0AA24AA94BA2CC12CD12C16E97A
:104B9000E12EF12C00E010E0D8CF0F942A139B01F6
:104BA000AC0144275527ED81FE816281738190E03D
:104BB00080E0AA24AA94BA2CC12CD12C18EEE12EA4
:104BC00013E0F12E00E010E00E94B19A882309F46E
:104BD0004ACF088119816FEA75E0C8010E94ADFFD4
:104BE000892B39F465EB75E0C8010E94ADFF892B74
:104BF00019F0A4016BE016CF61E975E0C8010E94CD
:104C0000ADFFA40166E0892B09F40CCFA4016DE08F
:104C100009CF0F942A139B01AC0144275527ED813E
:104C2000FE816281738190E080E0AA24AA94BA2C6C
:104C3000C12CD12C1CE2E12EFF24F39400E010E003
:104C40000E94B19A882309F40ECFA4016CE084CFAE
:104C50000F942A139B01AC0144275527ED81FE8157
:104C60006281738190E080E0AA24AA94BA2CC12CBE
:104C7000D12C16E9E12EF12C00E010E0E1CF0F94E9
:104C80002A139B01AC0144275527ED81FE816281E7
:104C9000738190E080E0AA24AA94BA2CC12CD12C74
:104CA00018E5E12E12E0F12E00E010E00E94B19A2A
:104CB000882309F4D8CEA40160E0B4CE0F942A135F
:104CC000ED81FE8173836283E181EF70772009F4C7
:104CD0004EC0E23041F148F4EE2309F445C0ED81C5
:104CE000FE81808170FA83F9D0CEE530E1F0A40135
:104CF0006AE0E730A1F7CE010E94FB218111EFCFDE
:104D00008091F10981508093F109DF91CF911F913A
:104D10000F91FF90EF90DF90CF90BF90AF909F905A
:104D20008F907F900895088119816BE875E0C80124
:104D30000E94ADFF892BA9F462EA75E0C8010E94C8
:104D4000ADFF892B71F468EA75E0C8010E94ADFFE0
:104D5000892B39F463E775E0C8010E94ADFF892B08
:104D600019F0A40166E0C7CFA40161E0C4CFE1500F
:104D7000ED3008F0B4CFF0E08827EE53F94D8F4FB7
:104D80000D945632CF266F26D226D2266F26D526F0
:104D90006F26F626F626F626F626F626D226A40155
:104DA00062E0A9CFA40165E0A6CF088119816BE874
:104DB00075E0C8010E94ADFF892BA9F462EA75E095
:104DC000C8010E94ADFF892B71F468EA75E0C80143
:104DD0000E94ADFF892B39F463E775E0C8010E949A
:104DE000ADFF892B19F0A40167E085CFA40160E035
:104DF00082CF8F71806449CECF93DF9300D000D0F3
:104E00001F921F92CDB7DEB7FC019181907F9B600E
:104E10009183448355836683778388E0DE0111960E
:104E200001900D928A95E1F729813A814B815C814D
:104E30006D817E818F81988528960FB6F894DEBFAC
:104E40000FBECDBFDF91CF910895CF93DF9300D0F8
:104E500000D01F921F92CDB7DEB7FC019181907FE9
:104E60009A609183448355836683778388E0DE016B
:104E7000119601900D928A95E1F729813A814B8133
:104E80005C816D817E818F81988528960FB6F8941C
:104E9000DEBF0FBECDBFDF91CF910895CF93DF93DB
:104EA00000D000D01F921F92CDB7DEB7FC016F3F3C
:104EB000710519F014F06FEF70E077FD60E09181FB
:104EC000892F8F7081508230C8F4648388E0DE01BE
:104ED000119601900D928A95E1F729813A814B81D3
:104EE0005C816D817E818F81988528960FB6F894BC
:104EF000DEBF0FBECDBFDF91CF910895907F91604F
:104F00009183E3CFCF93DF93CDB7DEB760970FB632
:104F1000F894DEBF0FBECDBF19821A821B821C829D
:104F20001D821E821F8218868A81807F8A836FEF8E
:104F300070E0CE0101960E944E2760960FB6F8945D
:104F4000DEBF0FBECDBFDF91CF910895CF92DF922C
:104F5000EF92FF92DC01362F1196EC911197EF70D2
:104F6000EC3008F0B6C0F0E08827E654F84D8F4FDB
:104F70000D9456326C28F227F2276928692869288F
:104F80003728F92769286928C627C62714968D91DE
:104F90009D910D90BC91A02D662399F0B7FD9FC007
:104FA0008F3F9105A105B10529F024F08FEF90E026
:104FB000A0E0B0E02FEF30E0A901481B590BCA0177
:104FC0000CC0B7FD89C08F3F9105A105B10529F03F
:104FD00024F08FEF90E0A0E0B0E0FF90EF90DF9042
:104FE000CF90089514962C91822F90E06623A9F318
:104FF000E1CF1496CD90DD90ED90FC90179766234D
:1050000001F120E030E0A901C701B6010F9495300D
:1050100087FD65C020E030E04FE753E4C701B601EB
:105020000F949D3318160CF457C0A701960160E049
:1050300070E08FE793E40F9488320F946733CB01CD
:10504000CCCF20E030E0A901C701B6010F94953024
:1050500087FD42C020E030E04FE753E4C701B601CE
:105060000F949D331816DCF1C701B601E6CF1496F4
:105070006D917D918D919C9117973323B1F06D398E
:105080005FEF75078507950754F1611524E67207F0
:10509000810591050CF52CE93FEF4FEF5FEF0F9481
:1050A0000132C90181509F4F98CF6D394FEF74077E
:1050B000840794078CF0611554E675078105910506
:1050C00074F424E630E040E050E00F940132C9016E
:1050D00084CF8FEF9FEF81CF90E080E07ECF8FEF86
:1050E00090E07BCFCF93DF93EC01DB0189818F7060
:1050F0008630E1F128F481508230C8F080E014C09D
:10510000873009F18A508230C8F72FEF30E00F94D2
:105110006D3224E630E040E050E00F9401322C8301
:105120003D834E835F8381E0DF91CF9108952FEF20
:1051300030E00F946D3224E630E040E050E00F9410
:1051400001322C83F0CF2FEF30E00F946D3224E644
:1051500030E040E050E00F940132CA01B9010F94F1
:105160009C306C837D838E839F83DDCF2CE933E677
:105170000F946D3224E630E040E050E00F940132AD
:105180002C833D834E835F83B9CFDC011196EC9174
:105190001197EF70E150EB3008F039C0F0E088274C
:1051A000EB52F74D8F4F0D945632F828F828072907
:1051B000E028E028E928002900290029E028E02843
:1051C00014966D917D918D919C9117970F949C30C1
:1051D000089514966D917D918D919C91179724E679
:1051E00030E040E050E00F940132CA01B901EECF47
:1051F00014966C9170E090E080E00F949A300895DE
:1052000014966D917D918D919C911797089560E012
:1052100070E0CB010895DC011196EC911197EF70CD
:10522000E150EB3008F037C0F0E08827E55EF64D3E
:105230008F4F0D9456322D292D294B2926292629A9
:105240003C293329332933292629262914966D919F
:105250007D918D919C911797089514966C9170E0B3
:1052600090E080E0089514966D917D918D919C91D0
:1052700017970F946733089514966D917D918D91D2
:105280009C91179724E630E040E050E00F94013203
:10529000CA01B901089560E070E0CB0108958F92D2
:1052A0009F92AF92BF92CF92DF92EF920F931F9394
:1052B000CF93DF9300D000D01F921F92CDB7DEB7FF
:1052C000FC0109831A832B833C834D835E836F83A8
:1052D0007887828193810097A1F490E080E02896FE
:1052E0000FB6F894DEBF0FBECDBFDF91CF911F91F7
:1052F0000F91EF90DF90CF90BF90AF909F908F90E5
:1053000008958F010F94F000C82ED12C86E0C816A6
:10531000D10464F40F94A305BC01F8018281938148
:105320000F94B005FFEFCF1ADF0AF0CF65E0F80168
:10533000828193810F945F008C01892B71F28981A6
:10534000803158F6CE0101960E940B2916161706D9
:105350001806190644F4F8018085982F9D70A1F075
:105360008F70873089F0F80180858F7080876DEEAF
:1053700079E087EB9FE00E94EAE187EB9FE00E94E3
:105380007EE081E090E0ABCF0F942A134B015C01EB
:10539000CE0101960E940B29860E971EA81EB91EEB
:1053A000F80181869286A386B48682E0E11087E0C8
:1053B00099819295907F892BF801808762EE79E040
:1053C00087EB9FE00E94EAE1CE0101960E940B2943
:1053D000AB01BC012AE030E087EB9FE00E9443E193
:1053E0006CED79E087EB9FE00E94EAE1F8014185EE
:1053F0005285638574852AE030E087EB9FE00E9448
:1054000043E1BBCFDC011196EC911197EF70E150B5
:10541000EB3008F03EC0F0E08827EE5EF54D8F4F90
:105420000D945632282A282A492A1D2A1D2A422A42
:10543000332A332A332A1D2A1D2A14962D913D9191
:105440004D915C911797A4E6B0E00F942032089537
:1054500014966C9184E6689FB0011124072E000C0D
:10546000880B990B089520E030E048EC52E4149644
:105470006D917D918D919C9117970F94FB300F94B6
:105480006733089514966D917D918D919C91179736
:10549000089560E070E0CB010895FC01A7812A2FF8
:1054A0002E7FC9F081818F7081508330A0F4A69542
:1054B000A150BB0B2BE531E00F946D3224E630E0B8
:1054C00040E050E00F940132DA01C90187569F4F46
:1054D000AF4FBF4F08958FEF9FEF08952F923F92E8
:1054E0004F925F926F927F928F929F92AF92BF92F4
:1054F000CF92DF92EF92FF920F93CF93DF9300D082
:105500001F92CDB7DEB77C017A8369835C834B83BE
:10551000DB011C92FC016081662309F44BC030FF63
:1055200049C0F9E06F9FB001112463597E4ECD014F
:105530000F94FC2AD70111968C918F7041F04B810A
:105540005C8162EA77E089819A810F94D336E981A0
:10555000FA8101900020E9F7319729813A81E21B15
:10556000F30B19012E0E3F1E4B815C814E1B5F0B0E
:10557000415051095C834B83D7011196EC911197EF
:10558000EF7009F4F5C0E150EC3008F0F1C0F0E044
:105590008827E253F54D8F4F0D945632DD2A802B2C
:1055A000ED2B4C2C672C2B2BFD2BFD2BFD2B192BC6
:1055B000012B832C29803A80DFCFF7018481282FAB
:1055C00030E050E040E0002359F030E0A4E6B0E0E5
:1055D0000F9433322FEF30E040E050E00F9401326F
:1055E0005F934F933F932F938EEC95E09F938F9310
:1055F000FC81FF932B812F933F922F920F940B37B7
:10560000B2C017968C9117978F9316968C91169718
:105610008F9315968C9115978F9314968C918F93E9
:1056200081ED95E09F938F93BC81BF93EB81EF93C6
:10563000E3CF17968C9117978F9316968C911697A8
:105640008F9315968C9115978F9314968C918F93B9
:1056500085ED95E0E7CF1496CD90DD90ED90FC9030
:105660001797F7FE34C084E6882E912CA12CB12C1C
:10567000C701B601A50194010F9401329B01AC0151
:1056800088279927DC01821B930BA40BB50BBF93D2
:10569000AF939F938F9366277727CB016C197D0972
:1056A0008E099F09A50194010F9401325F934F93D6
:1056B0003F932F9389ED95E09F938F933C813F9388
:1056C0004B814F933F922F920F940B374CC0C701E1
:1056D000B60124E630E040E050E00F9401329F93A1
:1056E0008F937F936F935F934F933F932F938AEDA5
:1056F00095E09F938F939C819F93AB81AF93E2CF73
:10570000C7010E944D2ABC01D7011696CC9016976E
:105710001796DC901797D0FADD24D0F814969C9158
:1057200014971596FC90EB80BC80292F30E050E058
:1057300040E077FD35C0011135C07F936F931F9214
:105740001F921F929F931F92FF92DF92CF9283EE40
:1057500095E09F938F93FC81FF932B812F933F9232
:105760002F920F940B370FB6F894DEBF0FBECDBF4C
:1057700089819A810F900F900F900F90DF91CF91B8
:105780000F91FF90EF90DF90CF90BF90AF909F90E0
:105790008F907F906F905F904F903F902F900895E3
:1057A000002361F0292F30E0A4E6B0E00F943332FB
:1057B0002FEF30E040E050E00F9401325F934F93C1
:1057C0003F932F931F92FF92DF92CF9286EE95E048
:1057D0009F938F93BF92EF9275CF15968C911597EB
:1057E0001F928F9316969C91169717968C918170A5
:1057F0008F939F9389EE95E015CF14968D909D9091
:10580000AD90BC90179720E030E0A901C501B4012C
:105810000F9495302401350187FF04C077FA709406
:1058200077F87094C301B2010F9467336B01072EB0
:10583000000C880B990B0F949C309B01AC01C301A9
:10584000B2010F94883220E030E04AE754E40F942C
:10585000FB300F94F2330F946733062F772E20E03E
:1058600030E0A901C501B4010F94953087FF07C04E
:105870007F920F93DF92CF928FEE95E0D3CE7F92FF
:105880000F93DF92CF9280EF95E09F938F933C81AF
:105890003F934B814F93B0CE14968C9114971F92E7
:1058A0008F9315968C9115971F928F9316968C91C6
:1058B0001F928F9386EE95E09F938F93BC81BF9349
:1058C000EB81EF933F922F920F940B374CCF1796AB
:1058D0008C9117971F928F9314968C9114971F9207
:1058E0008F9315968C9115971F928F9316968C9186
:1058F0001F928F9383EE95E09F938F93BC81BF930C
:10590000EB81EF93DFCE14966D917C914B815C819E
:10591000C1010F94F1362CCFEF92FF920F93CF93EA
:10592000DF93CDB7DEB7A0970FB6F894DEBF0FBEFA
:10593000CDBF7C0100E020E033E040E250E0BE015A
:105940006F5F7F4F0E946E2ABE016F5F7F4F87EBB4
:105950009FE00E94D4E165E572E187EB9FE00E9441
:10596000EAE1F70161816F704AE050E087EB9FE068
:105970000E94A1E06EE472E187EB9FE00E94EAE101
:105980004AE050E0F701628187EB9FE00E94A1E0CE
:1059900087EB9FE00E947EE0A0960FB6F894DEBFF2
:1059A0000FBECDBFDF91CF910F91FF90EF90089583
:1059B000CF93DF93EC016115710539F48F8181700C
:1059C0008F8381E0DF91CF9108958981982F9F7017
:1059D00029F180E09430B0F79B01770F440B550B11
:1059E0002959310941095109A4E6B0E00F94203248
:1059F0002BE531E040E050E00F94013237FF02C068
:105A000030E020E02536310514F024E630E02F5F49
:105A1000220F8F818170282B2F83D3CF807F8260CC
:105A20008983DACFFC019181892F8F7021F0823038
:105A300029F080E00895907F926091839B0177FF29
:105A400002C030E020E02E3681E0380714F02DE669
:105A500031E02683878130FB80F9878381E00895D8
:105A6000EF92FF920F931F93CF93DF93FC01892B4B
:105A700069F19081992351F19D3291F180ED890F67
:105A80008A3070F1C8E0D0E0953211F1CEEFDFEF4F
:105A90009B37F1F0C7E1D0E09332D1F08F0186E778
:105AA000E82E81E1F82EC1E0D0E0C7010F94D52A9D
:105AB000AC01B701C8010F94EE2A892B49F0219659
:105AC00089E0E80EF11CC931D10579F7CFEFDFEF9E
:105AD000CE01DF91CF911F910F91FF90EF9008952C
:105AE000D0E0C0E0F5CFEF92FF920F931F93CF93DA
:105AF000DF93EC01892B51F188858F70843009F593
:105B0000E984FA84C7010E94302D8C011816190609
:105B1000ECF4C7010E9481E6C801012E000CAA0B1B
:105B2000BB0B89879A87AB87BC878885807F82601B
:105B30008887C801DF91CF911F910F91FF90EF905F
:105B40000895823019F409851A85F3CF10E000E03A
:105B5000F0CF2F923F924F925F926F927F928F92EF
:105B60009F92AF92BF92CF92DF92EF92FF920F93EC
:105B70001F93CF93DF93CDB7DEB7A0970FB6F894FE
:105B8000DEBF0FBECDBF6115710549F528E0FC01F0
:105B9000DE01119601900D922A95E1F729813A8153
:105BA0004B815C816D817E818F819885A0960FB637
:105BB000F894DEBF0FBECDBFDF91CF911F910F9143
:105BC000FF90EF90DF90CF90BF90AF909F908F901D
:105BD0007F906F905F904F903F902F9008956B0152
:105BE0008C016FEB77E0C6010E94ADFFFC01892BB1
:105BF00009F40EC180858F70843009F452C085305D
:105C000009F006C1E680F780E114F10409F400C14F
:105C1000F70180858F70823011F4E280F380E11407
:105C2000F10409F4F5C0F70180858F70853011F01B
:105C3000F701F3CFC7010F94F0008230C9F760E09D
:105C4000C7010F945F005C010E94732D61E0C701E2
:105C50000F945F004C01FC0180858F70823041F70A
:105C6000C8010E940B29F401418452846384748426
:105C70006415750586059705D9F6A114B10409F4D4
:105C8000C7C019821A821B821C821D821E821F823B
:105C900018868A81807F8A83F5016185CE0101960D
:105CA0004EC064EC77E0818592850F94C336892BD2
:105CB00009F0AEC0C8010E940B296115710581056C
:105CC000910509F48BC0660F771F881F991F2FEF6E
:105CD00030E040E050E00F94013257FD15C0233012
:105CE0003105410551050CF05FC0DA01C90101968B
:105CF000A11DB11D82309105A105B105D9F1039710
:105D0000A105B10509F450C019821A821B821C82B8
:105D10001D821E821F8218868A81807F8A8367E0A7
:105D2000CE0101960E94B72129873A874B875C876D
:105D30006D877E878F87988B62E1CE0109960E94DE
:105D4000D921298B3A8B4B8B5C8B6D8B7E8B8F8B08
:105D5000988F49895A896B897C898D899E89AF89F9
:105D6000B88D49835A836B837C838D839E83AF83F5
:105D7000B88714CF19821A821B821C821D821E8250
:105D80001F8218868A81807F8A8367E0CE01019610
:105D90000E94B72129873A874B875C876D877E876A
:105DA0008F87988B61E1C9CF19821A821B821C826E
:105DB0001D821E821F8218868A81807F8A8367E007
:105DC000CE0101960E94B72129873A874B875C87CD
:105DD0006D877E878F87988B60E1AFCF19821A829B
:105DE0001B821C821D821E821F8218868A81807FF0
:105DF0008A8367E0CE0101960E94B72129873A87FE
:105E00004B875C876D877E878F87988B62E095CF05
:105E100068EF75E0C6010E94ADFF7C01009709F4B0
:105E2000D1C0FC0180858F70853009F0BAC0C701F0
:105E30000F94F000843009F0C5C060E0C7010F94F2
:105E40005F005C0161E0C7010F945F006C0162E0DC
:105E5000C7010F945F00FC0121853285438554857D
:105E6000298F3A8F4B8F5C8F63E0C7010F945F00DF
:105E70007C01C8010E940B29298D3A8D4B8D5C8DC8
:105E800062177307840795079CF419821A821B8294
:105E90001C821D821E821F8218868A81807F8A83CF
:105EA00040E050E0BA01CE0101960E94FC2649CFA5
:105EB000F5010184F285E02DFE8FED8FF60121843E
:105EC0003284F7010184F285E02DF8A3EF8F198267
:105ED0001A821B821C821D821E821F8218868A8162
:105EE000807F8A836101032C000CEE08FF082D8D52
:105EF0003E8D4901330FAA08BB08498D5A8D2A01EE
:105F0000550F66087708C8010E940B299B01AC0158
:105F10002419350946095709C701B60168197909D5
:105F20008A099B090F94CF31EF8DF8A19F01FF0FD4
:105F3000440B550B24193509460957090F940132B2
:105F4000820E931EA41EB51EC1012D8D3E8D821B97
:105F5000930B6F8D78A1498D5A8D641B750B0F942F
:105F6000423277FF02C06F5F7F4F75956795CB0117
:105F7000770FAA0BBB0B880E991EAA1EBB1EB7FC7F
:105F80000BC0A601B701C814D904EA04FB040CF441
:105F90008ACFA401B50187CF40E050E060E070E017
:105FA00082CF81110FC019821A821B821C828A81C2
:105FB000807F8A8349815A816B817C8180E090E077
:105FC000DC01CFCEF80140815181628173818481EF
:105FD0009581A681B781C5CE4F925F926F927F92D5
:105FE0008F929F92AF92BF92CF92DF92EF92FF92E9
:105FF0000F931F93CF93DF93CDB7DEB760970FB6A4
:10600000F894DEBF0FBECDBF6115710539F528E0EC
:10601000FC01DE01119601900D922A95E1F729818C
:106020003A814B815C816D817E818F8198856096FC
:106030000FB6F894DEBF0FBECDBFDF91CF911F9199
:106040000F91FF90EF90DF90CF90BF90AF909F9017
:106050008F907F906F905F904F9008956B018C01AF
:106060006FEB77E0C6010E94ADFF5C01F801F080A4
:10607000FF2009F456C0009709F453C0FC01808545
:106080008F70843009F4C7C0853009F04AC0809110
:106090003102893020F480913002893050F06CEF69
:1060A00075E087EB9FE00E94D4E187EB9FE00E94C0
:1060B0007EE0F501E680F780E114F10491F1F7014B
:1060C00080858F705701823061F0B12CA12CE114D2
:1060D000F10409F41DC1F70180858F70853021F02E
:1060E000F701E280F380F3CFC7010F94F000823014
:1060F000B9F760E0C7010F945F000E94732D4C0157
:1061000061E0C7010F945F00F80120812815190490
:1061100039F7FC0120852F70223011F7009709F024
:1061200001C168EF75E0C6010E94ADFF7C01F80176
:1061300081818F7009F407C1E114F10409F47DC075
:10614000F70180858F70853009F001C1C7010F9478
:10615000F000843009F0FBC0C8010E940B294B01FC
:106160005C0160E0C7010F945F00FC0181859285AE
:10617000A385B48519821A821B821C821D821E820D
:106180001F82188688169906AA06BB060CF499C0C9
:106190008A81807F8A8363E0C7010F945F005C017E
:1061A00062E0C7010F945F00FC0141845284638464
:1061B000748461E0C7010F945F004C0160E0C70187
:1061C0000F945F00FC01C184D284E384F484C8018D
:1061D0000E940B29F50121853285438554852419B8
:1061E0003509460957096C197D098E099F090F94D5
:1061F000CF31F40121853285438554852C193D0921
:106200004E095F090F940132BA01A901440D551DD1
:10621000661D771D31C064EC77E0818592850F940F
:10622000C336892B09F07DCFF0E1FF1609F460C079
:10623000FF1568F082E0F816E1F1F8014081518124
:106240006281738184819581A681B78129C0E1E152
:10625000FE16F1F1F2E1FF12F0CF19821A821B82D1
:106260001C821D821E821F8218868A81807F8A83FB
:1062700044E150E060E070E0CE0101960E94FC260F
:1062800029873A874B875C876D877E878F87988BB6
:1062900049855A856B857C858D859E85AF85B889B6
:1062A00049835A836B837C838D839E83AF83B887B6
:1062B000B6CE19821A821B821C821D821E821F8208
:1062C00018868A81807F8A8340E050E0BA01D4CF6B
:1062D00019821A821B821C821D821E821F821886CE
:1062E0008A81807F8A8340E850E060E070E0C4CF1C
:1062F00019821A821B821C821D821E821F821886AE
:106300008A81807F8A834FEF50E060E070E0B4CFF5
:10631000A114B10409F405CFF50180858F7009F44B
:1063200000CFC50119821A821B821C821D821E8227
:106330001F8218862A81207F2A83FC01418552858D
:106340006385748599CFE114F10409F476CFF701E0
:1063500080858F7009F071CF19821A821B821C828E
:106360008A81807F8A8349815A816B817C8180E028
:1063700090E0DC0195CF0F931F93CF93DF93EC0157
:10638000088119816FE270E0C8010F94003700970F
:1063900049F0FC011192CF01DF91CF911F910F9134
:1063A0000C94FB1EC8010E94FB1E009711F019827D
:1063B0001882DF91CF911F910F910895DC01129601
:1063C000ED91FC91309729F090859F7081E0953098
:1063D00009F080E00895EF92FF920F931F93CF93FF
:1063E000DF93EC017B0188859985892BA9F48A814B
:1063F0009B810F94F000082F10E00530110564F424
:106400000F94A30599878887BC018A819B810F948B
:10641000B0050F5F1F4FF1CFE885F9853097D9F0B0
:106420008085982F9F70A9F4807F82608087E8859F
:10643000F9851186128613861486E885F985F78218
:10644000E682C701DF91CF911F910F91FF90EF90EE
:106450000895923061F3F12CE12CF3CFCF92DF92CB
:10646000EF92FF920F931F93CF93DF93EC016A019A
:106470007B0188859985892BA9F48A819B810F945A
:10648000F000082F10E00530110564F40F94A30507
:1064900099878887BC018A819B810F94B0050F5F23
:1064A0001F4FF1CFE885F985309781F08085982FCF
:1064B0009F7051F4807F82608087E885F985C1866E
:1064C000D286E386F48602C09230B9F3DF91CF9191
:1064D0001F910F91FF90EF90DF90CF900895FC01F6
:1064E00080859185009799F0FC0120852F702230DE
:1064F00029F461857285838594850895253039F462
:1065000060E00F945F00009711F0FC01F2CF60E0B3
:1065100070E0CB0108950F931F93CF93DF93FC019D
:10652000C481D5812097C9F18B0188858F70853012
:1065300021F5CE010F94F0008017110671F16CF176
:10654000602FCE010F945F00FC01892B31F1808513
:106550008F70823039F461857285838594850F94BC
:106560009C3006C08330C9F461857285838594852B
:10657000DF91CF911F910F910895672B71F48230B5
:1065800029F469857A858B859C85E9CF833029F448
:1065900069857A858B859C85EBCF60E070E0CB01C7
:1065A000E7CF0F931F93CF93DF93FC01C481D58175
:1065B0002097F9F088858F70823049F4672BC9F4F1
:1065C00089859A85DF91CF911F910F91089585302C
:1065D00081F48B01CE010F94F0008017110649F071
:1065E00044F0602FCE010F945F00FC0181859285FD
:1065F000E9CF90E080E0E6CF0F931F93CF93DF9336
:10660000EC018B017B836A8383E892E09983888322
:1066100070E060E0C8010E94D13297FD0CC09D83FC
:106620008C83C8010E94C01C9F838E83DF91CF9111
:106630001F910F910895919581959109F0CF8F92B7
:106640009F92AF92BF92DF92EF92FF920F931F93B0
:10665000CF93DF93EC018A819B810F94F000082F88
:1066600010E00430110554F40F94A305BC018A8195
:106670009B810F94B0050F5F1F4FF3CFEA81FB8121
:10668000068117810115110529F0F8018281938196
:106690009D838C83EC81FD81309721F082819381F1
:1066A0009F838E83EE81FF81309721F082819381D9
:1066B000998788870115110549F0F80180858F7049
:1066C000843009F438C028F4823079F0DD24DA947B
:1066D0000DC0853009F42CC08630C1F76AE076E041
:1066E000C8010E94ADFF8C01E5CFD184DA86F4E1C8
:1066F000FD1508F459C0ED2DF0E08827ED57FC4C4E
:106700008F4F0D945632E033E033E033C333D4334C
:10671000D433D433D433D433D433FF33EE3330349F
:1067200053344034D4335E34E033AD34D433C934DD
:1067300006811781BFCFA184B284A114B10409F4EA
:10674000C5CFF5018081882309F4C0CF87E0882E6A
:1067500080E1982EF12CE12CDE2CC4010F94D52A77
:10676000AC01B401C5010F94EE2A892B09F41FC1B5
:10677000FFEFEF1AFF0A89E0880E911CE7E1EE16A1
:10678000F10451F7A3CF8AE090E00F9489278C01A0
:10679000BE010E94FC328BE693E0F8019183808376
:1067A000118610861C870B87DF91CF911F910F9167
:1067B000FF90EF90DF90BF90AF909F908F900895E3
:1067C00088E090E00F9489278C01BE010E94FC3282
:1067D00087E493E0F80191838083E4CF8DE090E03B
:1067E0000F9489278C01BE010E94FC3283E293E062
:1067F000F80191838083C8010E94E4ABD3CF89E084
:1068000090E00F9489278C01FC01D383C28381E03F
:1068100093E091838083CE010E94F418F801958360
:1068200084838FEB9CE090878783CE010E94C01CFD
:10683000892B09F4B7CF70E060E0CE010E94D1321D
:10684000F8018683882331F0833009F0ABCF82E2F0
:106850009CE002C08AE19FE0F80190878783A2CF85
:106860008EE090E00F9489278C01FC01D383C283D2
:1068700085EF93E091838083C8010E9418AC92CF8A
:1068800086E090E00F9489278C01FC01D383C283BA
:106890008FED92E091838083CE010E94F418F8017D
:1068A000958384837FCF86E090E00F9489278C01C5
:1068B000FC01D383C2838DEB92E0ECCF8BE090E0C0
:1068C0000F9489278C01FC01D383C28383ED93E06D
:1068D00091838083168270E060E0CE010E94D13205
:1068E00097FD28C0F80195838483F8018481958100
:1068F000009719F0863491052CF080E290E0F801C1
:106900009583848361E070E0CE010E948B3220E0A9
:1069100030E04AE754E40F94FB300F946E33611576
:1069200071058105910579F0F8016783708781878A
:10693000928738CF919581959109F8019583848349
:1069400081E08683D2CF88E893E1A0E0B0E0F8014F
:1069500087839087A187B28725CF86E090E00F9448
:106960008927FC01D383C28381EB93E091838083E9
:1069700015821482AC81BD81109741F018968C91DC
:1069800018978F70863011F4B583A483FC87EB874A
:106990000BCF84E090E00F948927FC01D383C2835E
:1069A0002FE833E0318320839C878B87FDCEC501A0
:1069B0000E9481E68E2D90E0B0E0A0E0F801818792
:1069C0009287A387B4878085807F826080878ECE00
:1069D000CF92DF92EF92FF926A017B0163E0FC01AC
:1069E000828193810F945F00FC01892BA9F080853F
:1069F0008D7091F4C094D094E094F094CC24CA9417
:106A000081859285A385B4858C219D21AE21BF21EE
:106A100081879287A387B487FF90EF90DF90CF9014
:106A20000895CF92DF92EF92FF926A017B0163E0BB
:106A3000FC01828193810F945F00FC01892BA9F0F6
:106A40009085892F8D7089F4907F92609087CC24F7
:106A5000FF2441855285638574854C295D296E2903
:106A60007F294187528763877487FF90EF90DF907B
:106A7000CF900895CF92DF92EF92FF926A017B014F
:106A800063E0FC01828193810F945F00009791F095
:106A9000FC0120852F70223069F461857285838521
:106AA00094856C217D218E219F21FF90EF90DF90B6
:106AB000CF90089560E070E0CB01F7CFAF92BF9226
:106AC000CF92DF92EF92FF920F931F93CF93DF93BA
:106AD000CDB7DEB7CD56D1090FB6F894DEBF0FBEE5
:106AE000CDBF5C01A7960FAFA797A8961FAFA89739
:106AF000A9962FAFA997AA963FAFAA97AB964FAF8B
:106B0000AB97AC965FAFAC97AD966FAFAD97AE96C7
:106B10007FAFAE9723961FAE1EAE2397FE01ED5BAF
:106B2000FF4F82E1DF011D928A95E9F7729611927B
:106B3000119287E0DF011D928A95E9F76FE076E018
:106B400087EB9FE00E94D4E1B60187EB9FE00E94B3
:106B5000D4E1CE018A599F4F0E948C2CF0FE2CC0AC
:106B6000A796EFADA797E83108F050C1F0E088276D
:106B7000E354FA4C8F4F0D9456320C37D53503370A
:106B8000063706370337D535063706370637063753
:106B9000063706370637D535D53506370637063773
:106BA000D535D535D53506370C376BEB7EE0CE01C4
:106BB0008B5A9F4F0F94CE2A0E94CBFF882309F453
:106BC00007C18091A60A811103C1C114D10409F043
:106BD0005EC030E020E043E050E060E4CE0101968A
:106BE0000E947DA8D5011296ED91FC916081718182
:106BF0004FE350E0CE0101960F94D336F1FE0FC162
:106C0000A7968FADA797823009F409C1853009F4A2
:106C100006C1A8968FADA8978F709FE0980F9F70C0
:106C2000923018F0883009F0FAC001E020E032E03C
:106C300044E150E0BE016F5B7F4FCE018A599F4F08
:106C40000E946E2ABE016F5B7F4FCE0101960F94AA
:106C5000C71362E97EE087EB9FE00E94EAE1BE0194
:106C60006F5F7F4F87EB9FE00E94D4E16FE87EE08B
:106C700087EB9FE00E94EAE1BE016F5B7F4F87EBED
:106C80009FE00E94D4E187EB9FE00E947EE0A896FF
:106C90008FADA8978F70870100271072882311F09D
:106CA000F1FC04C00115110509F4F5C030E020E045
:106CB00043E050E060E4CE0101960E947DA8D5013A
:106CC0001296ED91FC91608171814FE350E0CE010D
:106CD00001960F94D336C114D10469F064EC76E0C8
:106CE000CE0101960F94AD364FE350E0B601CE01D0
:106CF00001960F94D33664EC76E0CE0101960F94A2
:106D0000AD364FE350E064E57EE00115110511F466
:106D10006AE47EE0CE0101960F94DE2AA8968FAD3C
:106D2000A8978F708450823008F09FC067E1CE0131
:106D30008A599F4F0E94D9216F962FAF6F97A096C7
:106D40003FAFA097A1964FAFA197A2965FAFA29732
:106D5000A3966FAFA397A4967FAFA497A5968FAF86
:106D6000A597A6969FAFA69700E020E033E044E108
:106D700050E0BE016F5B7F4FCE018A599F4F0E944A
:106D80006E2A6AE37EE087EB9FE00E94EAE1BE01A3
:106D90006F5F7F4F87EB9FE00E94D4E167E37EE067
:106DA00087EB9FE00E94EAE1BE016F5B7F4F87EBBC
:106DB0009FE00E94D4E187EB9FE00E947EE00E946A
:106DC000CBFF882329F08091A60A882309F455C0B7
:106DD000A701FF0C660B770BC5010E94113590E0EF
:106DE00080E0C359DF4F0FB6F894DEBF0FBECDBFB2
:106DF000DF91CF911F910F91FF90EF90DF90CF9097
:106E0000BF90AF90089564EC7EE0D1CE68E97EE05B
:106E100087EB9FE00E94EAE1E894F0F8CDCEF0FE27
:106E200036CF66968FAD6697882309F430CFBE01C2
:106E30006B5A7F4FCE0101960F94C71369E87EE02D
:106E400087EB9FE00E94EAE1BE016F5F7F4F87EB17
:106E50009FE00E94D4E166E87EE087EB9FE00E941D
:106E6000EAE1BE016B5A7F4F0ACF20E032E0012BEE
:106E700011F020E033E000E07ACFBE016F5B7F4F7E
:106E8000CE0101960F94C71340E052E060E070E03D
:106E9000C5010E94E834F0FE91C0A796EFADA79718
:106EA000E150E53118F5F0E08827E65AF84C8F4FAD
:106EB0000D945632673876377637763776376738B7
:106EC00076377637763776377637763776376C3863
:106ED00064387637763776376F375E3861386DE5E8
:106EE0007FE0CE018B5A9F4F0F94CE2A30E020E0F6
:106EF00043E050E060E4CE0101960E947DA8D501F8
:106F00001296ED91FC91608171814FE350E0CE01CA
:106F100001960F94D336C114D10469F064EC76E085
:106F2000CE0101960F94AD364FE350E0B601CE018D
:106F300001960F94D33664EC76E0CE0101960F945F
:106F4000AD364FE350E065E47EE0CE0101960F944C
:106F5000DE2A61E37EE087EB9FE00E94EAE1BE016A
:106F60006F5F7F4F87EB9FE00E94D4E16EE27EE08F
:106F700087EB9FE00E94EAE1BE016B5A7F4F87EBEF
:106F80009FE00E94D4E187EB9FE00E947EE00E9498
:106F9000CBFF882309F41CCF8091A60A811118CF5A
:106FA000BE016B5A7F4FCE0101960F94C71340E08C
:106FB00051E060E070E0C5010E94E834F2FE7BC061
:106FC00040E050E061E070E0C5010E943A35672B77
:106FD000682B692B09F483C065E17FE0CE018B5AF1
:106FE0009F4F0F94CE2A30E020E043E050E060E471
:106FF000CE0101960E947DA8D5011296ED91FC91DB
:10700000608171814FE350E0CE0101960F94D33639
:10701000C114D10469F064EC76E0CE0101960F94BE
:10702000AD364FE350E0B601CE0101960F94D33652
:1070300064EC76E0CE0101960F94AD364FE350E05C
:107040006DE67EE0CE0101960F94DE2A68E27EE0D6
:1070500087EB9FE00E94EAE1BE016F5F7F4F87EB05
:107060009FE00E94D4E165E27EE087EB9FE00E9412
:10707000EAE1BE016B5A7F4F87EB9FE00E94D4E1AB
:1070800087EB9FE00E947EE00E94CBFF882309F4FB
:107090009FCE8091A60A81119BCEBE016B5A7F4F75
:1070A000CE0101960F94C71340E054E060E070E019
:1070B000C5010E94E83481E090E093CE66E67FE06F
:1070C00010CF6FE67FE00DCF69E37FE00ACFF501D7
:1070D0008285853009F00ACF60E37FE002CF40E08F
:1070E00050E062E070E0C5010E943A35672B682BE2
:1070F000692B19F067E27FE071CF6CE07FE06ECF23
:10710000AF92BF92CF92EF920F931F93CF93DF93E3
:10711000CDB7DEB7C856D1090FB6F894DEBF0FBEA3
:10712000CDBF5C01A2960FAFA297A3961FAFA39706
:10713000A4962FAFA497A5963FAFA597A6964FAF5D
:10714000A697A7965FAFA797A8966FAFA897A9969F
:107150007FAFA9979E2D28E0FE01EF59FF4FDE017A
:10716000A75ABF4F01900D922A95E1F7A296EFAD75
:10717000A297E150ED3008F0F2C0EC2CF0E0882747
:10718000EB53F74C8F4F0D9456323C394539A339A8
:10719000AD399939D2383339AF39AF394E396039D1
:1071A00086397339992331F0C5010E94ED1C00978F
:1071B00009F449C067E0CE01875A9F4F0E94D92148
:1071C00068EC79E087EB9FE00E94EAE14AE050E05A
:1071D0006A966FAD6A9787EB9FE00E94A1E06DEB26
:1071E00079E087EB9FE00E94EAE1CE01875A9F4F4A
:1071F0000E940B29AB01BC012AE030E087EB9FE045
:107200000E9443E187EB9FE00E947EE06A960FAD0B
:107210006A976B961FAD6B976C962FAD6C976D96BA
:107220003FAD6D976E964FAD6E976F965FAD6F9752
:10723000A0966FADA097A1967FADA197C5010E94C2
:107240004F2981E090E0C859DF4F0FB6F894DEBFB8
:107250000FBECDBFDF91CF911F910F91EF90CF90D7
:10726000BF90AF900895911105C0C5010E94ED1C1B
:10727000009749F366E09FCF992329F0C5010E944A
:10728000ED1C009701F362E096CF911105C0C50196
:107290000E94ED1C0097B9F261E08DCF40E050E014
:1072A00061E070E0C5010E943A35672B682B692BBD
:1072B00029F4C5010E94ED1C009729F26BE07BCFF9
:1072C00040E050E061E070E0C5010E943A35672B74
:1072D000682B692B31F0C5010E94ED1C009709F461
:1072E000B2CF6AE068CF40E050E062E070E0C501F4
:1072F0000E943A35672B682B692B31F0C5010E943B
:10730000ED1C009709F49FCF6CE055CF40E050E0B2
:1073100062E070E0C5010E943A35672B682B692B4B
:1073200031F4C5010E94ED1C009709F48CCF6DE08B
:1073300042CF911106C0C5010E94ED1C009709F4CF
:1073400082CF63E038CF992331F0C5010E94ED1C54
:10735000009709F478CF65E02ECF64E02CCF90E061
:1073600080E071CFCF93C62F63E0FC0182819381CF
:107370000F945F00FC01892B91F09085892F8D700F
:1073800071F4907F9260908781859285A385B48502
:107390008827BB278C2B81879287A387B487CF91BF
:1073A0000895CF92DF92FF920F931F93CF93DF93B5
:1073B000F12C6115710509F492C06A01EB018C0191
:1073C000CB010E94DE31F82E882309F488C0D2FE5A
:1073D0000AC0D8018C918B3009F44DC008F03EC032
:1073E0008A3009F44DC0D0FE09C0F801608186EFF3
:1073F000860F843018F0CE010E94B239D1FE6FC0E2
:10740000D80114964D915D916D917C9117971196CD
:107410008C918F70873038F0893008F440C08A50E2
:10742000823008F465C0CE010E940419EE81FF810C
:10743000309709F454C080858F709EEF980F92307A
:1074400010F081114CC0D80111968C91982F929513
:10745000907F80858F70892B808741C08C30B9F0F8
:1074600040E050E062E070E08D3009F0BCCFCE012A
:107470000E941135B8CF40E050E061E070E0F7CFF6
:1074800040E050E061E070E0CE010E94E83440E06E
:1074900050E062E070E0CE010E94E834A4CFEE81BB
:1074A000FF813097E1F080858F709EEF980F9230CA
:1074B00010F0811114C04187528763877487EE8171
:1074C000FF818085807F83608087EE81FF8180855A
:1074D000982F907F8F708067903609F4BDCF8F2DE5
:1074E000DF91CF911F910F91FF90DF90CF90089582
:1074F000CE010E940419F3CF63E0FC0182819381E5
:107500000F945F00009719F0FC01818508958FEFBB
:107510000895AF92BF92CF92DF92EF92FF920F93B6
:107520001F93CF93DF9300D000D01F921F92CDB74F
:10753000DEB76115710509F45FC05A016B017C016A
:10754000CB010E94DE31082F882369F1D6011696FF
:107550008D919C91009709F443C0FC011085212F67
:107560002F703EEF320F323010F021112EC01295E5
:107570001F70B0FE59C0C6010E947C3AF70180839B
:10758000112381F18181807F182B1183D6011696FA
:10759000ED91FC9181859285A385B485F701848363
:1075A0009583A683B783802F28960FB6F894DEBF05
:1075B0000FBECDBFDF91CF911F910F91FF90EF9044
:1075C000DF90CF90BF90AF900895253049F460E0F0
:1075D0000F945F00009721F0DC0118961C91C7CF33
:1075E00010E0C7CFD6011696ED91FC9180858F7083
:1075F000823021F0833051F000E0D5CF41855285B3
:1076000063857485C7010E942527CDCF41855285AA
:1076100063857485F7018181807F876081834483DE
:10762000558366837783BFCF1123E1F2F701AACF99
:10763000AF92BF92CF92DF92EF92FF920F931F9380
:10764000CF93DF9300D000D01F921F92CDB7DEB74B
:107650005C017B0160FF03C0E894E0F8F4F8F4FCFF
:107660000DC00E94FEA9663971058105910530F0B3
:107670008091AB0A9091AC0A059719F5A7014427B0
:107680005770052E000C660B770BC5010E94113553
:1076900064E17EE087EB9FE00E94EAE18FEF9FEFDD
:1076A00028960FB6F894DEBF0FBECDBFDF91CF9105
:1076B0001F910F91FF90EF90DF90CF90BF90AF9010
:1076C000089519821A821B821C821D821E821F82CB
:1076D00018868A81807F8A8340E053E0B501CE011D
:1076E00001960E94893A40E057E060E070E0C501F1
:1076F0000E943A35E62AF72AD12CC12C09811A8139
:107700002B813C814D815E816F817885C5010E940E
:107710005E35C6CFCF93DF93EC0140E053E060E0ED
:1077200070E00E943A35611571058105910599F067
:107730002091AB0A3091AC0A2630310561F4CE01BC
:107740000E94183B40E053E060E070E0CE01DF9122
:10775000CF910C94E834DF91CF9108958F929F924E
:10776000AF92CF92EF92FF920F931F93CF93DF933D
:1077700000D000D01F921F92CDB7DEB74C01098315
:107780001A832B833C834D835E836F8378876AE003
:1077900079E087EB9FE00E94EAE1CE0101960E942A
:1077A0008C2C898181112FC00B81013089F140F12E
:1077B000023019F010E00530F1F5D401ED91FC91A3
:1077C000068CF78DE02D09811A812B813C814D813A
:1077D0005E816F817885C401199581E090E02896DB
:1077E0000FB6F894DEBF0FBECDBFDF91CF911F91D2
:1077F0000F91FF90EF90CF90AF909F908F90089552
:10780000CC24C394DACF813071F1823009F451C0B5
:107810006DEF78E087EB9FE00E94EAE14AE050E0FC
:10782000698187EB9FE00E94A1E087EB9FE00E94C7
:107830007EE001E010E06DEE78E087EB9FE00E94D3
:10784000EAE14AE050E0B80187EB9FE00E948BE15B
:1078500087EB9FE00E947EE0CE0101960E948C2C77
:1078600090E080E0BCCFCE0101960F946E0044976B
:10787000B8F46EE170E0CE0101960E947228F40126
:107880006281738140E052E0CE0101960E94D139BD
:1078900060E072E1D40112968D919C910E94183B98
:1078A000D401ED91FC91068CF78DE02DCC24C3948E
:1078B0008ACF1D821E821F821886D401ED91FC9111
:1078C000068CF78DE02DCC24C39402E01A812B8125
:1078D0003C8140E07DCF8F929F92AF92BF92CF923A
:1078E000DF92EF92FF920F931F93CF93DF93CDB769
:1078F000DEB760970FB6F894DEBF0FBECDBF8C0128
:107900007B0140E058E060E070E00E943A35672B70
:10791000682B692B09F0A9C062E070E0C8010E94E1
:10792000D1326C0119861A861B861C861D861E861E
:107930001F86188A8A85807F8A87D7FC96C040E098
:1079400052E0B801CE0109960E94893A63E070E0E6
:10795000C8010E94D132AC011816190614F04FE389
:1079600050E081E0C816D10429F4EF2CFF0CFF0889
:10797000FF2404C082E0C816D104D4F32FEF30E016
:10798000D7010F946D329A01550F440B550B0F948C
:10799000013249016901C8010E947C3AE82EF12CAC
:1079A00060E0CE0109960E94A62788169906F9F490
:1079B000CD2841F082E0E816F10419F185E0E816DF
:1079C000F104F9F081E090E060960FB6F894DEBF24
:1079D0000FBECDBFDF91CF911F910F91FF90EF9020
:1079E000DF90CF90BF90AF909F908F900895CD285B
:1079F00059F186E0E816F10441F081E0E816F1045F
:107A000021F061E0C8010E94B239B401CE010996AB
:107A10000E944E2740E052E0B801CE0109960E9434
:107A2000D13982E0E816F10421F085E0E816F1048E
:107A300029F460E071E0C8010E94183B60E072E048
:107A4000C8010E94183BBECF85E0E816F10409F496
:107A5000B9CF82E0E816F10409F4B4CF62E0C801BE
:107A60000E94B23960E071E0EBCF90E080E0ACCFF3
:107A700081E090E008950F931F93CF93DF9300D0A0
:107A800000D01F921F92CDB7DEB719821A821B82D7
:107A90001C821D821E821F8218862A81207F2A83D3
:107AA000FC0102811381C8010E947C3A813041F0BF
:107AB00020F0823011F0853081F490E080E002C047
:107AC00081E090E028960FB6F894DEBF0FBECDBFE0
:107AD000DF91CF911F910F91089540E052E0B801DE
:107AE000CE0101960E94893A60E0CE0101960E9483
:107AF000A627E8CF8F929F92AF92BF92CF92DF924C
:107B0000EF92FF920F931F93CF93DF93CDB7DEB722
:107B100067970FB6F894DEBF0FBECDBF8C017B0117
:107B20006A014C018DE0880E911C9F8A8E8AF801B3
:107B300051834083148613861586168E158E672B07
:107B400009F45EC0452B09F45BC06FE270E0C70129
:107B50000F94B8365C01892B09F44AC0F701DE01A5
:107B6000119690E080E0BD012191222341F02F3257
:107B700031F08431910519F02D930196F5CF860FE0
:107B8000971FFC011082C6010E94ADFFF80193838C
:107B90008283B5016F5F7F4F4FE050E0C4010F94C7
:107BA000F136CE0146960E94BB31F801968F858F43
:107BB0008E899F89892B09F41586C8010E94DE31C0
:107BC000882319F0C8010E941F3367960FB6F894F6
:107BD000DEBF0FBECDBFDF91CF911F910F91FF9000
:107BE000EF90DF90CF90BF90AF909F908F900895CF
:107BF000B701C6010E94ADFFF80193838283DDCFF8
:107C0000F80113821282D9CFDC011B968D919C91D1
:107C1000009739F0DC01ED91FC910280F381E02DB9
:107C2000199408958F929F92AF92BF92CF92DF9254
:107C3000EF92FF920F931F93CF93DF93CDB7DEB7F1
:107C4000CF55D1090FB6F894DEBF0FBECDBF8C0162
:107C50006B016115710519F04115510579F569E25E
:107C600073E187EB9FE00E94EAE160E273E187EB5A
:107C70009FE00E94EAE1B80187EB9FE00E94D4E117
:107C80006EE173E187EB9FE00E94EAE187EB9FE002
:107C90000E947EE0C15ADF4F0FB6F894DEBF0FBEE0
:107CA000CDBFDF91CF911F910F91FF90EF90DF90AB
:107CB000CF90BF90AF909F908F900895460F571F21
:107CC000DA011C920E94FEA94B0168E173E187EB87
:107CD0009FE00E94EAE14AE050E0B40187EB9FE0B8
:107CE0000E948BE165E173E187EB9FE00E94EAE18E
:107CF000B80187EB9FE00E94D4E162E173E187EB7A
:107D00009FE00E94EAE1BAE38B16B1E09B064CF4D7
:107D100065E073E182E19FE00E94EAE182E19FE099
:107D2000B7CF63E073E187EB9FE00E94EAE1B60121
:107D300087EB9FE00E94D4E161E073E187EB9FE075
:107D40000E94EAE187EB9FE00E947EE01A8219829E
:107D5000FE0133968EE3DF011D928A95E9F780914B
:107D6000AB0A9091AC0A059791F563E070E0C80109
:107D70000E94251F7C01892BD1F5E091940DF09193
:107D8000950D808180FF86CF61E070E0C8010E9480
:107D9000251F892B09F47ECF64E270E0C8010F949F
:107DA0000037892B09F076CF63EE72E187EB9FE015
:107DB0000E94EAE1B80187EB9FE00E94D4E187EBE3
:107DC0009FE00E947EE0C8010F94070E63CF61E040
:107DD00070E0C8010E94251F7C01892B09F46DC049
:107DE0004FE350E0B801CE0101960F94F136A12C7B
:107DF000BB24B394E00EF11E6AED72E1C7010F944B
:107E0000C52A892B49F4F60101900020E9F7319742
:107E1000EC19FD093297B8F664E270E0C8010F94DE
:107E20000037892B09F036CFB11003C0AA2009F41E
:107E300031CF4091AD0A5091AE0AB701CE018F5BB0
:107E40009F4F0E947A3DCE018F5B9F4F0E94DE3193
:107E5000182F882359F0B601CE018F5B9F4F0F94E6
:107E6000610611E0181619060CF010E0CE018F5BC8
:107E70009F4F0E94043E112309F40CCF898188236F
:107E800009F408CF8091AB0A9091AC0A059709F4E8
:107E900001CF6CEB72E187EB9FE00E94EAE1BE014B
:107EA0006F5F7F4F87EB9FE00E94D4E187EB9FE0FD
:107EB0000E947EE0CE01019687CF62E070E0C801AB
:107EC0000E94251F7C01892B09F4E4CEAA24A394E7
:107ED000B12C90CF0F931F93CF93DF93CDB7DEB725
:107EE0006F970FB6F894DEBF0FBECDBF20916E0A1C
:107EF00030916F0A232B09F4E4C02091A70A022EC7
:107F0000000C330B82179307B4F465EA72E182E147
:107F10009FE00E94EAE182E19FE00E947EE080E033
:107F20006F960FB6F894DEBF0FBECDBFDF91CF9135
:107F30001F910F9108956FE872E187EB9FE00E9417
:107F4000EAE187EB9FE00E947EE08091F2098F5F7B
:107F50008093F209E091AD0AF091AE0A3097A1F159
:107F60000681178101151105C9F1D80118968C9168
:107F70008F70853029F5C8010F94F000882301F136
:107F80004091AD0A5091AE0AF80160817181CE0135
:107F900001960E947A3DCE0101960E94DE3188232F
:107FA00059F08C859D85009739F0DC01ED91FC91AD
:107FB0000084F185E02D1995CE0101960E94043EC2
:107FC000F80102811381CECF6FE772E187EB9FE06A
:107FD0000E94EAE187EB9FE00E947EE01092A50AF2
:107FE0001092A40A67E772E187EB9FE00E94EAE142
:107FF00087EB9FE00E947EE064E670E080E090E026
:108000000F942A1110926D0A6FE572E187EB9FE0E1
:108010000E94EAE10E94FEA9AB01BC012AE030E027
:1080200087EB9FE00E9499E080916E0A90916F0A21
:10803000009711F00F940A0B10926F0A10926E0ABB
:108040001092AA0A1092A90A1092AE0A1092AD0AD2
:108050001092780A1092770A10926C0A10926B0AAA
:108060001092690A1092680A1092760A1092750AA4
:1080700010926A0A1092670A1092660A1092B00A69
:108080001092AF0A1092720A1092710A6AE572E1B8
:1080900087EB9FE00E94EAE10E94FEA9AB01BC01D0
:1080A0002AE030E087EB9FE00E9499E087EB9FE0B9
:1080B0000E947EE010925F0A8091F20981508093C5
:1080C000F20981E02DCFCF93DF93EC0159834883F0
:1080D0007B836A831C861B861D861E8E1D8E0E94D6
:1080E000DE31882329F0CE01DF91CF910C941F332C
:1080F000DF91CF910895CF93DF93EC01FB012481B1
:10810000358140815181628173810E9443E1CE01BA
:10811000DF91CF910895CF92DF92EF92FF921F935C
:10812000CF93DF9300D000D0CDB7DEB76DE273E11F
:108130008AE09FE00E94EAE18EEEE82E8EE0F82EC3
:1081400010E090E1C92ED12CF70181917F0180319F
:1081500030F46CE176E08AE09FE00E94D4E11530D3
:1081600041F1F7013197808190E0B0E0A0E0898390
:108170009A83AB83BC83DE82CD82BE016F5F7F4F6B
:108180008AE09FE00E947B406BE273E10E94EAE19B
:108190001F5F1630C9F626960FB6F894DEBF0FBEE5
:1081A000CDBFDF91CF911F91FF90EF90DF90CF90E7
:1081B00008958091F30E90E0B0E0A0E089839A8367
:1081C000AB83BC83DE82CD82BE016F5F7F4F8AE0CE
:1081D0009FE00E947B400E947EE0DACFEF92FF9208
:1081E0000F931F93CF93DF9300D000D01F92CDB792
:1081F000DEB77B01CE0107969F938F9301979F93E4
:108200008F9301979F938F9301979F938F930197DC
:108210009F938F9301979F938F938E010F5F1F4FB3
:108220001F930F938EE196E09F938F93DB0113963C
:108230008C9113978F9312968C918F930F9478371C
:108240000FB6F894DEBF0FBECDBF0697ECF460EE1C
:108250007DE182E19FE00E94EAE1D70112966D91F3
:108260007C9182E19FE00E94D4E180E991E0279631
:108270000FB6F894DEBF0FBECDBFDF91CF911F9137
:108280000F91FF90EF9008958091E60E9091E70E88
:10829000892B09F449C00F940001882309F444C0D4
:1082A000A091E60EB091E70E52961C921E92519745
:1082B00054961C921E92539784E890E01D969C93CE
:1082C0008E931C971E961C921E9782E755968C9350
:1082D0005597ED91FC9111970088F189E02D64E0AC
:1082E00070E0CD0119958091E60E9091E70EDC01CA
:1082F000ED91FC910280F381E02D46E050E0B80161
:10830000199586E0F801AEEEBEE001900D928A95D7
:10831000E1F78091E60E9091E70EDC01ED91FC9182
:108320000488F589E02D19950E948B4062EF7DE16C
:108330008AE09FE00E94EAE188EC90E098CFEF921B
:10834000FF920F931F93CF93DF9300D000D0CDB750
:10835000DEB77C018B016CE97FE087EB9FE00E9438
:10836000EAE1D7011296ED91FC916081718187EB72
:108370009FE00E94D4E163E97FE087EB9FE00E94E9
:10838000EAE1012E000C220B330B09831A832B83A5
:108390003C8380E190E09E838D83BE016F5F7F4FC1
:1083A00087EB9FE00E947B400E947EE040E058E027
:1083B00060E070E0C7010E94113526960FB6F89470
:1083C000DEBF0FBECDBFDF91CF911F910F91FF9008
:1083D000EF9008953F924F925F926F927F928F92AB
:1083E0009F92AF92BF92CF92DF92EF92FF920F9344
:1083F0001F93CF93DF93CDB7DEB72C970FB6F894CA
:10840000DEBF0FBECDBF5C01362E972E3A0169014B
:108410006DEF7FE087EB9FE00E94EAE14AE050E0E9
:10842000632D792D87EB9FE00E948BE165EF7FE064
:1084300087EB9FE00E94EAE1C301B0E0A0E08F83F8
:108440009887A987BA8730E1432E512C5C864B86EA
:10845000BE01695F7F4F87EB9FE00E947B404C012C
:1084600061EF7FE00E94EAE14AE050E0B601C4011A
:108470000E948BE169EE7FE0C4010E94EAE1C7013E
:10848000B0E0A0E089839A83AB83BC835E824D8297
:10849000BE016F5F7F4FC4010E947B400E947EE05F
:1084A0008091730A9091740A70E060E0892B09F062
:1084B00047C081E090E09093740A8093730A26E0AD
:1084C00040E855E260E070E082E29CE00E9437E321
:1084D0003092B90D82E29CE09093B80D8093B70D75
:1084E0001092C70E1092C90E1092C80E01301105DD
:1084F00009F44EC00CF041C0012B09F44EC0C11468
:10850000D10409F457C082E0C816D10409F062C052
:108510007092420E6092410E1092440E1092430EE1
:10852000F092460EE092450E86E00F9450141092A1
:10853000740A1092730A882309F456C0682F70E0F9
:10854000C5010E949F4190E080E02C960FB6F89400
:10855000DEBF0FBECDBFDF91CF911F910F91FF9076
:10856000EF90DF90CF90BF90AF909F908F907F90D3
:108570006F905F904F903F9008950330110581F008
:108580000430110509F0BBCFFE24EF24FE24B7CF41
:10859000FE2CEE24EE24EA94B2CFFF24FA94AFCF5F
:1085A000EF2821F492E0E92EF12CEECFEE24E394B3
:1085B000F12CEACF7092420E6092410E90E080E082
:1085C000EE2011F080E09FEF9093440E8093430ED5
:1085D00085E0ABCF6DEC7FE087EB9FE00E94EAE1A6
:1085E0001092740A1092730A81E090E0AECF2F923D
:1085F0003F924F925F926F927F928F929F92AF9233
:10860000BF92CF92DF92EF92FF920F931F93CF937F
:10861000DF93CDB7DEB72C970FB6F894DEBF0FBE51
:10862000CDBF5C0109831A832B833C834D835E831A
:108630006F837887CE0101960F946E001C01023083
:1086400011F0053011F4312C212CF5010481158134
:10865000F80180858F70853009F07FC0C8010F94C4
:10866000F000E82EF12CF2E0EF16F1040CF475C0E6
:1086700060E0C8010F945F00FC01818592859C87B2
:108680008B8761E0C8010F945F00FC014184528434
:108690006384748488248A94982CF2E0EF16F104A1
:1086A00059F062E0C8010F945F00FC01818492845C
:1086B000F3E0EF16F104A1F48FE390E09A87898745
:1086C00092E0C92ED12C29853A85D1010F946532CB
:1086D00024E630E040E050E00F94013279011CC004
:1086E00063E0C8010F945F00FC01818592859A8741
:1086F000898782E0C82ED12CF4E0EF16F10439F01E
:1087000064E0C8010F945F00FC01C184D2848985B4
:108710009A857101892BB9F684019601A2016B85B6
:108720007C85C5010E94EA412C960FB6F894DEBF05
:108730000FBECDBFDF91CF911F910F91FF90EF90B2
:10874000DF90CF90BF90AF909F908F907F906F9071
:108750005F904F903F902F90089590E080E0E4CF9D
:108760008F929F92AF92BF92DF92EF92FF920F9300
:108770001F93CF93DF93CDB7DEB7A7970FB6F894CB
:10878000DEBF0FBECDBF7C0108A319A32AA33BA364
:108790004CA35DA36EA37FA3CE0180960E94C52843
:1087A0004B015C01D7011496ED91FC9180858F708F
:1087B000843009F0EDC0102F4091AD0A5091AE0AFF
:1087C00061857285CE0101960E947A3DCE010196A7
:1087D0000E94DE31882309F44AC08B85893009F074
:1087E00046C070E060E0CE0101960E94D132082FB1
:1087F000D92E60EC7FE087EB9FE00E94EAE14AE03F
:1088000050E0602F7D2D87EB9FE00E948BE16EEBA7
:108810007FE087EB9FE00E94EAE1B501A40187EBCE
:108820009FE00F94D60468EB7FE087EB9FE00E9407
:10883000EAE1612F70E04AE050E087EB9FE00E94A0
:108840008BE187EB9FE00E947EE08091730A90911C
:10885000740A892B29F140E053E0B701CE018096DC
:108860000E94D13970E060E0C7010E949F4110E092
:1088700000E0CE0101960E94043EC801A7960FB603
:10888000F894DEBF0FBECDBFDF91CF911F910F9146
:10889000FF90EF90DF90BF90AF909F908F900895E2
:1088A00081E090E09093740A8093730A26E040E898
:1088B00055E260E070E082E29CE00E9437E30093C2
:1088C000B90D82E29CE09093B80D8093B70D1092A1
:1088D000C70E1092C90E1092C80EEB81FC811530A4
:1088E00021F01F3011F0123011F580858F708087D4
:1088F00070E060E083ED97E09093420E8093410E2C
:108900001092440E1092430E7093460E6093450EE3
:1089100086E00F9450141092740A1092730A01E0CA
:1089200010E0882309F4A5CF682F70E09DCF8085E3
:108930008F708061808722E538EB42E152E4C50107
:10894000B4010F94893220E030E040E251E40F940A
:10895000FB302DEE3EE94CE35EE30F94F5324B0124
:108960005C0120E030E0A9010F949D3320E030E06D
:1089700040E05FE387FD07C0C501B4010F94893271
:108980000F946733B7CFC501B4010F948832F8CF85
:1089900010E000E072CFCF92DF92EF92FF920F9340
:1089A0001F93CF93DF9300D000D01F921F92CDB7BB
:1089B000DEB77C0109831A832B833C834D835E835E
:1089C0006F837887CE0101960F946E008C018981A8
:1089D000882351F09B81923008F0BAC0823011F0A8
:1089E000853011F410E000E070E060E0C7010E9403
:1089F000D132D82EC92E60EB7FE087EB9FE00E943A
:108A0000EAE14AE050E06D2D7C2D87EB9FE00E946B
:108A10008BE16EEA7FE087EB9FE00E94EAE14AE0AB
:108A200050E0B80187EB9FE00E948BE187EB9FE06D
:108A30000E947EE08091730A9091740A892BE9F07C
:108A400040E053E0B701CE0101960E94D13970E0B9
:108A500060E0C7010E949F4190E080E028960FB639
:108A6000F894DEBF0FBECDBFDF91CF911F910F9164
:108A7000FF90EF90DF90CF90089581E090E0909389
:108A8000740A8093730A26E040E855E260E070E0E3
:108A900082E29CE00E9437E3D092B90D82E29CE032
:108AA0009093B80D8093B70D1092C70E1092C90E17
:108AB0001092C80E80ED97E09093420E8093410E85
:108AC0001092440E1092430E01151105E1F185E05C
:108AD00090E09093460E8093450E86E00F945014DC
:108AE000D82E64E670E080E090E00F942A11D11057
:108AF0000AC067EA7FE087EB9FE00E94EAE187EB2C
:108B00009FE00E947EE082ED97E09093420E80937A
:108B1000410E1092440E1092430E24E6209FC00195
:108B2000219F900D11249093460E8093450E86E070
:108B30000F9450141092740A1092730A882359F0FB
:108B4000682F70E086CF1092460E1092450EC5CF6A
:108B50008FEF9FEF83CF81E090E080CFEF92FF9285
:108B60000F931F93CF93DF93EC018B011E821D8225
:108B70001A821B821C82E880F980E114F10409F456
:108B800063C080916E0A90916F0A892B09F45CC0D2
:108B9000672B09F48701F80180858F708630D9F43E
:108BA00061E179E0C8010E94ADFF009719F0FC0176
:108BB00081858A836EEB76E0C8010E94ADFFFC01DF
:108BC000892B09F463C080858F70823009F45BC003
:108BD000853009F440C062E376E0C7010E94ADFF32
:108BE000009779F569E179E087EB9FE00E94EAE17F
:108BF0004AE050E06B8187EB9FE00E94A1E067E1D3
:108C000079E087EB9FE00E94EAE14AE050E06A8168
:108C100087EB9FE00E94A1E087EB9FE00E947EE04F
:108C200020E030E0A90162E376E0888199810F9429
:108C30004B0962E376E0888199810E94ADFF00973D
:108C400019F009969E838D83DF91CF911F910F912B
:108C5000FF90EF9008950680F781E02D309709F49A
:108C6000BACF80858F70823009F0B5CF81858B8334
:108C70000680F781E02D309709F4ADCF80858F70A5
:108C8000823009F0A8CF81858B83A5CFF801808140
:108C900091810F94592AF8CF6F927F928F929F9271
:108CA000AF92BF92CF92DF92EF92FF920F931F93FA
:108CB000CF93DF93CDB7DEB7AE970FB6F894DEBF94
:108CC0000FBECDBF80916E0A90916F0A892B09F477
:108CD00054C68091A70A811150C68091A70A8F5F60
:108CE0008093A70A6EEE7BE18AE09FE00E94EAE1B2
:108CF0008AE09FE00E947EE000916E0A10916F0A68
:108D000065E376E0C8010E94ADFF9093AE0A8093C0
:108D1000AD0A6BE376E0C8010E94ADFF9093780A3C
:108D20008093770A65E776E0C8010E94ADFF9093D3
:108D3000AA0A8093A90A62E476E0C8010E94ADFF06
:108D400090936C0A80936B0A009749F1DC011696A8
:108D5000ED91FC91309719F120852F702530F9F4B1
:108D60006AED7BE18AE09FE00E94EAE180916B0A74
:108D700090916C0A0F94F00080936A0A4AE050E0E8
:108D8000682F8AE09FE00E94A1E08AE09FE00E94B5
:108D90007EE0E0916B0AF0916C0A86819781909356
:108DA000690A8093680A67E476E080916E0A909180
:108DB0006F0A0E94ADFF9093670A8093660A00973E
:108DC00009F4B2C00F94F000082F10E0011511054E
:108DD00009F4AAC0000F111F000F111F8091640A2F
:108DE0009091650A892B09F08EC078010138110530
:108DF0001CF040E8E42EF12CC7010F9489279093D2
:108E0000650A8093640AE092630A10929B0A1092AA
:108E10009A0A1092620A1092610A1092990A1092AC
:108E20009D0A10929C0AC70101960F94892790937E
:108E30009F0A80939E0A9093980A8093970A8E0DBA
:108E40009F1D9093920A8093910A0F942A13609326
:108E5000930A7093940A8093950A9093960A90E0EF
:108E600080E0E0919E0AF0919F0AE80FF91F1082BE
:108E70000196E816F906ACF782E090E090939B0A21
:108E800080939A0A8091610A9091620A009741F05A
:108E900061E00F94E50E60E08091610A0F94B70ED7
:108EA00080E98093C9001092C8001092CD0083E041
:108EB0008093CC008EE08093CA00F0922F02E09263
:108EC0002E0220919E0A30919F0A80912E0290914D
:108ED0002F02820F931F9093920A8093910A232B63
:108EE00009F45FC06AE67BE187EB9FE00E94EAE15C
:108EF000B70187EB9FE00F94C2048AE89DE190934D
:108F0000900A80938F0A60EC7BE18AE09FE00E94E8
:108F1000EAE14AE050E0B8018AE09FE00E948BE17C
:108F20008AE09FE00E947EE06DE476E080916E0A28
:108F300090916F0A0E94ADFF8C01009709F471C0F7
:108F40000F94F000882309F46CC06FEF680FC8011C
:108F50000F945F00FC01E184F28490918D0A9923C3
:108F600059F0809170008E7F8093700010928D0A6E
:108F700010922A021092290282E180932802911114
:108F80000E9440F7C7010E9468F701E010E0E01678
:108F9000F10674F060E0C8010E949CF70F5F1F4F5C
:108FA000F6CF63E57BE187EB9FE00E940EE2A5CF61
:108FB00065E47BE187EB9FE00E94EAE10E94FEA965
:108FC000AB01BC012AE030E087EB9FE00E9499E012
:108FD00087EB9FE00E947EE064EA7BE18AE09FE00D
:108FE0000E94EAE14AE050E0B7018AE09FE00E9477
:108FF0008BE18AE09FE00E947EE06EE97BE187EBF7
:109000009FE00E94EAE10E94FEA9AB01BC012AE0B8
:1090100030E087EB9FE00E9499E087EB9FE00E94A1
:109020007EE000916E0A10916F0A61E576E0C8015A
:109030000E94ADFF9093720A8093710A68E576E012
:10904000C8010E94ADFF9093B00A8093AF0A892BAC
:1090500009F448C08091B10A811144C08091A20AEC
:109060009091A30A892B09F0DFC16FE17BE187EBC7
:109070009FE00E94EAE187EB9FE00E947EE08FE0A4
:1090800090E00F9489278C0188E1D80111968C9388
:10909000119712961C9212971C921E961C921E9269
:1090A0001D970F94450A1093A30A0093A20A012B5F
:1090B00009F08CC060E17BE182E19FE00E94EAE17F
:1090C00082E19FE00E947EE080E081708093B10A9F
:1090D0008091B10A882331F06EE87BE18AE09FE05D
:1090E0000E94EAE11092A50A1092A40AE091AD0A4A
:1090F000F091AE0A309709F4CCC2C680D7800091B7
:10910000AD0A1091AE0A0115110509F4BBC2C114D4
:10911000D10409F4B7C2F60180858F70853099F7C4
:10912000C6010F94F000823070F3A801B601CE01A1
:1091300001960E946340CE0101960E94DE31882391
:10914000E1F18C859D85009709F40DC2DC01ED915C
:10915000FC910284F385E02D1995892B49F08C85CB
:109160009D85DC01ED91FC910084F185E02D199540
:109170008C859D85DC01ED91FC910680F781E02DC9
:109180001995892BD1F0CE0101960E947C3A882353
:1091900041F040E051E060E070E0CE0101960E94B5
:1091A00011358F819885892B41F040E052E060E0D5
:1091B00070E0CE0101960E941135D6011296CD9035
:1091C000DC90CE0101960E94043E99CF0F94450A8F
:1091D0008091A20A9091A30A0E94CAF78AE69DE0B4
:1091E0000E947CF9811189C061EF7AE18AE09FE0F9
:1091F0000E940EE28091A20A9091A30A0E941BFB9A
:10920000E091A20AF091A30A81E080838091A20AF2
:109210009091A30A0E9429FB6DED7AE1811102C0B1
:1092200068EC7AE187EB9FE00E940EE28091AF0A42
:109230009091B00A892B09F447CF8091A00A9091B0
:10924000A10A892B09F0E2C083E190E00F948927FD
:109250008C018091A20A9091A30A2AE738EDF801C7
:10926000328B218B968385831482108289E08183DF
:1092700081E0828383831093A10A0093A00A0F9454
:109280002A136B017C01F0E1CF0EF7E2DF1EE11C37
:10929000F11CD8011596ED91FC9116978FEF8387FD
:1092A0001486138214821582168217821086118604
:1092B000128614961C92BB24B394BE01605E7F4F4D
:1092C000F801858196810E9403FC18160CF099C064
:1092D0000F942A136C157D058E059F0508F091C02B
:1092E000DE01909698E080E0915039F1ED91E82709
:1092F000F0E0E85FF24D8491F7CF0E94139B8091DC
:10930000A20A9091A30A0E94CAF78AE69DE00E94F1
:109310007CF981110BC06BEA7AE18AE09FE00E9440
:10932000EAE18AE09FE00E947EE080CF6FE87AE188
:1093300082E19FE00E940EE2C7CE9FA19813BDCFAD
:10934000D8018C91811138C015968D919C910E9405
:1093500029FBBE01605E7F4FF801858196810E94E6
:10936000FCFA40E064EBD80115968D919C910E9427
:10937000D6FAF80185809680C4010E945AFAC40189
:109380000E94CAF767E88AE69DE00E94E2DB60E897
:109390008AE69DE00E94E2DB0F94B10AC4010E94BC
:1093A0005AFAA82ED80115968D919C910E9429FBFE
:1093B000A5FC02C0F801B082AE014F5F5F4FBE0155
:1093C000605E7F4FC8010E946AFBD8011196AC9085
:1093D00088A1803109F4D3C2BE01605E7F4FC8010D
:1093E0000E94D9FB8A1510F5F8018181D8011196E8
:1093F0008C93119714968C9114978F5F14968C937D
:109400005CCFE091A00AF091A10A1282E091AF0A2C
:10941000F091B00AE680F7803FE7D32E8091AF0A43
:109420009091B00A892B71F481E04FCE88A18031F0
:1094300011F48CE0DBCFBE01605E7F4FC8010E945B
:10944000D9FBD4CFE114F10479F3BE01605E7F4F04
:10945000F701808191810E948AAB882329F368E714
:109460007AE187EB9FE00E94EAE1D7016D917C9160
:1094700087EB9FE00E94D4E187EB9FE00E947EE0B3
:109480000091A00A1091A10AAE014F5F5F4FBE018B
:10949000605E7F4FC8010E94BFFB882309F45EC055
:1094A00088A1803109F45AC0DD82F8018581968156
:1094B0000E9429FBBE01605E7F4FD80115968D91F9
:1094C0009C910E94FCFA40E06EE4F801858196814F
:1094D0000E94D6FA40E06B81D80115968D919C913F
:1094E0000E94D6FA40E06C81F801858196810E9445
:1094F000D6FA88A1803141F040E06D81D8011596FF
:109500008D919C910E94D6FAF801858196810E94E6
:1095100029FBBE01605E7F4FD80115968D919C910D
:109520000E94FCFAF801408168E4858196810E94DE
:10953000D6FA64E170E080E090E00F942A11D8013F
:109540008C91882331F06AE070E080E090E00F9425
:109550002A11F801858196810E9429FBD701129674
:10956000ED90FC905BCF70E060E0CE0101960E9430
:10957000D1328C01912C812C97FF06C01195019559
:10958000110988248394912CCE0101960E947C3A83
:10959000E82EF12C8B85853091F0863009F00DCEC8
:1095A000B02E61E0802F0F94E50E61E0892809F468
:1095B00043C0EA94EF2809F043C060E041C0EF28BF
:1095C00029F462E0CE0101960E94B23940E051E0F8
:1095D00060E070E0CE0101960E9411358F81988580
:1095E000892B41F040E052E060E070E0CE0101964E
:1095F0000E94113561E0802F0F94E50E60E0802F0E
:109600000F94B70E66E87BE187EB9FE00E94EAE1EA
:109610004AE050E0B80187EB9FE00E948BE161E8EF
:109620007BE187EB9FE00E94EAE16FE77BE187EB5C
:109630009FE00E94EAE1C1CDEA94EF2809F0BDCF96
:10964000E62EF12C8B2D0F94B70E6AE77BE187EBAA
:109650009FE00E94EAE14AE050E0B80187EB9FE01A
:109660000E948BE168E77BE187EB9FE00E94EAE1E3
:109670004AE050E0B70187EB9FE00E948BE166E78C
:109680007BE1D5CFF801868197819093A50A8093DD
:10969000A40A87EB9FE00E947EE064E67AE18AE01C
:1096A0009FE00E94EAE18AE09FE00E947EE0E09174
:1096B000A90AF091AA0A309709F4B0C08091A70ACC
:1096C0008F5F8093A70A068117815E01F8E2AF0ED3
:1096D000B11C81E3682E84E0782E99E4892E94E011
:1096E000992E0115110509F494C0D80118968C9192
:1096F0008F70863009F06BC019A708A770E060E092
:10970000C5010E94AE458DA59EA5892B09F45FC0B9
:1097100080916E0A90916F0A892B09F458C0E8A4D1
:10972000F9A4E114F104C1F1F70180858F7086304E
:1097300099F5F9A2E8A270E060E0CE0180960E945F
:10974000AE45EDA1FEA110821182128213826BE55B
:1097500076E0C7010E94ADFF0097F1F0DC0118969A
:109760002C9118972F702530B9F41696CD90DC9077
:10977000C114D10489F0DA82C982B701CE01019601
:109780000E94AE45EE81FF81108211821282138207
:10979000F601C280D380ECCFEDA5FEA51082118228
:1097A000128213828AA5843068F462E0823008F065
:1097B00060E08BA50F94E50EEDA5FEA58181807F6D
:1097C000818305C08630E1F038F4853081F0D8011E
:1097D00012960D911C9185CF803439F060E082346F
:1097E000B1F78BA50F94E50EF2CF62E0FACFBC8201
:1097F000AB829A828982CE0101960E942D99E7CF91
:10980000BC82AB827A826982CE0101960E94029A62
:10981000DECF8091A70A81508093A70A67E57AE19D
:109820008AE09FE00E94EAE16FE47AE18AE09FE04B
:109830000E94EAE181E02091AD0A3091AE0A232B2B
:1098400009F480E00E94521A66E47AE18AE09FE01F
:109850000E94EAE181E02091A90A3091AA0A232B13
:1098600009F480E00E94521A67E37AE18AE09FE0FF
:109870000E94EAE16CE27AE18AE09FE00E94EAE17C
:1098800081E02091710A3091720A232B09F480E063
:109890000E94521A65E27AE18AE09FE00E94EAE1C2
:1098A00081E02091680A3091690A232B09F480E055
:1098B0000E94521A6CE17AE18AE09FE00E94EAE19C
:1098C00081E02091AF0A3091B00A232B09F480E0A7
:1098D0000E94521A8AE09FE00E947EE067E17AE1EE
:1098E0008AE09FE00E94EAE10E94FEA9AB01BC0170
:1098F0002AE030E08AE09FE00E9499E08AE09FE061
:109900000E947EE081E080936D0A89ED9EE00E94D6
:1099100099EE882351F089ED9EE00E9451F584E094
:1099200090E09093AC0A8093AB0A8091AB0A90913F
:10993000AC0A079731F484E090E09093AC0A8093EE
:10994000AB0A8091A70A81508093A70A80916D0A83
:10995000AE960FB6F894DEBF0FBECDBFDF91CF91AC
:109960001F910F91FF90EF90DF90CF90BF90AF903D
:109970009F908F907F906F90089580E0E9CFBCE03A
:10998000BA1508F431CD55CDFC016115710519F4F6
:1099900084819581089586819781681779072CF0D5
:1099A00084819581860F971F0895828193810C94FD
:1099B000D132EF92FF920F931F93CF93DF93DC018D
:1099C0001296ED91FC91309709F17A018B01EC012F
:1099D00061EC75E0808191810E94ADFF0097B1F04C
:1099E000FC0120852F70243089F461857285E8811F
:1099F000F9810288F389E02D9701A801CE01DF915A
:109A0000CF911F910F91FF90EF90199490E080E01B
:109A1000DF91CF911F910F91FF90EF900895EF92FA
:109A2000FF920F931F93CF93DF93CDB7DEB760976D
:109A30000FB6F894DEBF0FBECDBF8C017901CE0109
:109A400001960E94A5A9A701BE016F5F7F4FC801C3
:109A50000E94D94C60960FB6F894DEBF0FBECDBF02
:109A6000DF91CF911F910F91FF90EF900895FF929A
:109A70000F931F93CF93DF9300D000D0CDB7DEB705
:109A80008C01BC01CE0101960E940BDEBE016F5F0E
:109A90007F4F87EB9FE00E94DCE187EB9FE00E9415
:109AA0007EE0CE0101960E9403DE1A8219821C829A
:109AB0001B821E821D8266E27EE1CE0101960E941B
:109AC000A6DDF801248135818D819E81F12C281736
:109AD000390738F0BE016F5F7F4FC8010F94F20D58
:109AE000F82ECE0101960E9403DEFF2069F0B80136
:109AF000CE0101960E940BDECE0101960F94B11BA0
:109B0000CE0101960E9403DE26960FB6F894DEBFC2
:109B10000FBECDBFDF91CF911F910F91FF900895A0
:109B2000AF92BF92DF92EF92FF920F931F93CF936A
:109B3000DF9300D000D0CDB7DEB78C017B01D42EEF
:109B4000FB0184819581892BF9F0A080B1806FE3BE
:109B500070E0C5010F94B8360097B1F09C012A1946
:109B60003B0937FD11C050E040E0B701CE0101963E
:109B70000E9425DEBE016F5F7F4FC7010E945BDD43
:109B8000CE0101960E9403DEF70184819581892B25
:109B9000D9F1E080F1806FE576E0C7010F94C3361C
:109BA000892B01F5F801128A118A80E090E19587EE
:109BB000848784E890E0948B838B81E08687D58AC4
:109BC00081E090E026960FB6F894DEBF0FBECDBFC1
:109BD000DF91CF911F910F91FF90EF90DF90BF9099
:109BE000AF9008956CE676E0C7010F94C336892BD9
:109BF00059F4F801128A118A148A138A84E890E0D1
:109C0000958784871686DBCF90E080E0DBCF0F93CB
:109C10001F93CF93DF9300D000D0CDB7DEB7A091D4
:109C2000E60EB091E70E109709F478C052961C9298
:109C30001E92519754961C921E92539784E890E07E
:109C40001D969C938E931C971E961C921E9787E7D9
:109C500055968C935597ED91FC9111970088F18959
:109C6000E02D70E060E0CD01199510E000E08091FA
:109C7000E60E9091E70EDC01ED91FC9111971C9698
:109C80002D913C910217130740F40190F081E02DD3
:109C900060E019950F5F1F4FEACF0088F189E02D32
:109CA00070E060E0199508EE14E08091E60E909166
:109CB000E70EF80161918F01DC01ED91FC910190BB
:109CC000F081E02D1995B4E00C3E1B0771F78091EF
:109CD000E60E9091E70EDC01ED91FC910488F58988
:109CE000E02D199565E279E0CE0101960E9414DE1F
:109CF000CE0101960F94B11BCE0101960E9403DEA6
:109D000087E090E00F94AC0487E090E00F94B604F5
:109D10006BEF7DE18AE09FE00E94EAE11092060F7E
:109D20001092050F80E090E19093010F8093000F57
:109D300084E890E09093080F8093070F81E0809370
:109D4000020F82E78093090F84EF9EE00E94F119D1
:109D500084EF9EE00E948D1A88EC90E026960FB664
:109D6000F894DEBF0FBECDBFDF91CF911F910F9151
:109D70000895EF92FF920F931F93CF93DF93CDB788
:109D8000DEB760970FB6F894DEBF0FBECDBF8091EF
:109D9000A70A81113DC18091A70A8F5F8093A70A0E
:109DA00069E47CE18AE09FE00E94EAE18AE09FE0CA
:109DB0000E947EE01092060F1092050F80E090E165
:109DC0009093010F8093000F84E8E82EF12CF0921D
:109DD000080FE092070F81E08093020F12E71093C3
:109DE000090F84EF9EE00E9453208B37910509F004
:109DF000E6C06BE37CE187EB9FE00E94EAE187EB42
:109E00009FE00E947EE081E090E00E946A3F1C8219
:109E10001B828BE794E09A83898384EF9EE09E8384
:109E20008D838FEF9FEF98878F83CE0101960F94DC
:109E3000E00C90936F0A80936E0A84EF9EE00E947C
:109E40008D1A80916E0A90916F0A892B01F56FE24D
:109E50007CE182E19FE00E94EAE182E19FE00E94D2
:109E60007EE065E279E0CE0109960E9414DECE0123
:109E700009960F94B11BCE0109960E9403DE8091D2
:109E8000A70A81508093A70A90E080E019C06CE196
:109E90007CE18AE09FE00E94EAE18AE09FE00E9484
:109EA0007EE08091A70A81508093A70A0E944C46C9
:109EB0008091E60E9091E70E892B79F481E090E095
:109EC00060960FB6F894DEBF0FBECDBFDF91CF9185
:109ED0001F910F91FF90EF9008950F940001882338
:109EE00069F3A091E60EB091E70E52961C921E9275
:109EF000519754961C921E9253971D96FC92EE9287
:109F00001C971E961C921E9755961C935597ED9183
:109F1000FC9111970088F189E02D60E670E0CD0199
:109F200019950091E60E1091E70E65E279E0CE01F9
:109F300009960E9414DEC8010E94D2DF1816190685
:109F400064F48F87188A41E050E0BE01615F7F4F63
:109F5000CE0109960E942FDDEECFBE01675F7F4FD5
:109F600088EE9EE00E945BDDCE0109960E9403DE32
:109F70008091E60E9091E70EDC01ED91FC91048852
:109F8000F589E02D19956EEF7BE187EB9FE00E944C
:109F9000EAE168EE7EE0CE0109960E940BDEBE018A
:109FA000675F7F4F87EB9FE00E94DCE187EB9FE0DC
:109FB0000E947EE0CE0109960E9403DE7FCF84EFEF
:109FC0009EE00E94C719892BA1F084EF9EE00E94B9
:109FD000F11965E279E0CE0101960E9414DECE010E
:109FE00001960F94B11BCE0101960E9403DE0F94DF
:109FF000321C84EF9EE00E948D1A6BE07CE18AE0C7
:10A000009FE00E94EAE18AE09FE00E947EE037CF75
:10A010008FEF9FEF55CF4F925F926F927F928F920B
:10A020009F92AF92BF92CF92DF92EF92FF920F93E7
:10A030001F93CF93DF93CDB7DEB7C659D1090FB6C3
:10A04000F894DEBF0FBECDBF8E010F5B1F4FD8014E
:10A050001D921C92FE01ED5BFF4F8EE1DF011D9210
:10A060008A95E9F78091E60E9091E70E892B09F425
:10A07000FEC10F940001882309F4F9C1A091E60EF6
:10A08000B091E70E52961C921E92519754961C92D4
:10A090001E92539784E890E01D969C938E931C9794
:10A0A0001E961C921E9782E755968C935597ED91BC
:10A0B000FC9111970088F189E02D60E270E0CD01FC
:10A0C00019954FE150E0B8018091E60E9091E70EAE
:10A0D0000F9455017C018091E60E9091E70EDC0112
:10A0E000ED91FC910488F589E02D1995E114F104B6
:10A0F00009F4BDC1F801EE0DFF1D10828091F30E31
:10A100001F928F938091F20E1F928F938091F10E88
:10A110001F928F938091F00E1F928F938091EF0E7C
:10A120001F928F938091EE0E1F928F9388E796E097
:10A130009F938F931F9280E48F93FE0131966F015E
:10A14000FF93EF930F940B3765E17FE18AE09FE087
:10A150000E94EAE1B8018AE09FE00E94D4E1B601E2
:10A160008AE09FE00E94D4E18AE09FE00E947EE0C6
:10A170007E01F1E6EF0EF11CD70113961C921E92A0
:10A18000129788EE93E0A0E0B0E0F7018483958316
:10A19000A683B78384E0848781E295E091838083FE
:10A1A00016861586108B0787128A118A80E590E043
:10A1B000948B838B178A6DE27EE187EB9FE00E9490
:10A1C000EAE168EE7EE0CE0187589F4F0E940BDEE9
:10A1D000BE0167587F4F87EB9FE00E94DCE187EB71
:10A1E0009FE00E947EE0CE0187589F4F0E9403DED1
:10A1F00067EA76E0CE0185579F4F0E9414DE67EA3A
:10A2000076E0CE0187589F4F0E9414DEBE0167584A
:10A210007F4FCE018D579F4F0E940BDE4091EC0E79
:10A220005091ED0E6091E80E7091E90ECE018D57C0
:10A230009F4F0E942FDD0FB6F894DEBF0FBECDBF3B
:10A24000811105C0CE018D579F4F0E9494DDC157EB
:10A25000DF4F48815981CF58D040C557DF4F6881C3
:10A260007981CB58D040CE018D579F4F0E942FDD72
:10A27000811105C0CE018D579F4F0E9494DDBE0114
:10A280006D577F4FCE018F569F4F0E940BDECE0140
:10A290008D579F4F0E9403DECE0187589F4F0E942B
:10A2A00003DECE0185579F4F0E9403DE89EA96E0C8
:10A2B000CD57DF4F99838883C358D040C957DF4FAC
:10A2C00019821882C758D040C757DF4F19821882A9
:10A2D000C958D040CF56DF4F88819981C159D040AD
:10A2E000CB57DF4F99838883C558D0406FE07FE11B
:10A2F00087EB9FE00E94EAE10E94FEA9AB01BC014E
:10A300002AE030E087EB9FE00E9499E087EB9FE036
:10A310000E947EE064E670E080E090E00F942A11F5
:10A3200087E39DE4D7011E969C938E931D9768EA60
:10A3300070EE84E698EE0F94AA2B8C01892B09F419
:10A34000EEC083E090E00F948927F8019587848719
:10A35000DC011196FC92EE9212961C92C7010E94AB
:10A3600099EE882319F0C7010E9451F5F701618920
:10A370007289A388B4886115710509F48FC0CE0174
:10A3800087589F4F0E942FE2A501BE0167587F4F5B
:10A39000C7010E9401F6181619060CF0BDC0D701BE
:10A3A0001F96BC901F975096AC90DF92CF9288E892
:10A3B0009EE19F938F931F930F930F94312CDF9205
:10A3C000CF9283E89EE19F938F931F930F930F94F7
:10A3D000312CD8011C96ED91FC9181E08283DF92B3
:10A3E000CF9280E89EE19F938F931F930F930F94DA
:10A3F000312CD8011C96ED91FC911282AF92BF9244
:10A400008AE49EE19F938F931F930F930F94312CB7
:10A410000FB6F894DEBF0FBECDBFB12C81E4C82EBD
:10A420008EE1D82EBB2D24E0B202F001112483E886
:10A4300090E08C0F9D1FE80FF91F8081918100979C
:10A44000A1F12281338121153105C9F33F932F9367
:10A450009F938F93DF92CF921F930F930F94312C82
:10A46000B3940FB6F894DEBF0FBECDBFDBCF40E292
:10A4700050E067E47FE1C8010F94FC2A69E27FE1C4
:10A480008AE09FE00E94EAE1B8018AE09FE00E9432
:10A49000D4E18AE09FE00E947EE030CE678570893B
:10A4A000A501C7010E944CF276CF85E89EE19F93FB
:10A4B0008F931F930F930F94312CF701168A158AEF
:10A4C000D8011C96ED91FC91C080D1800F900F9027
:10A4D0000F900F9043E3A42EB12CD601ED91FC9187
:10A4E0000084F185E02DC601199541975CF4B1E037
:10A4F000AB1AB10839F064E170E080E090E00F94AD
:10A500002A11EBCFD601ED91FC910084F185E02D6D
:10A51000C6011995419734F4C8010E943DE810E046
:10A5200000E065C065E279E0CE0185579F4F0E944B
:10A5300014DE912CA12CD601ED91FC910688F789AF
:10A54000E02DC6011995882309F446C0BDE0AB1281
:10A5500001C0A92CD601ED91FC910688F789E02D68
:10A56000C60119958111C5C0D601ED91FC910084F9
:10A57000F185E02DC6011995892B09F4CCC0D601CF
:10A58000ED91FC910284F385E02DC6011995B82E5A
:10A59000BAE08B1709F4C1C0EDE08E1709F4BDC015
:10A5A000FFEF8F1709F4B7C0EA968FAFEA97EB96E3
:10A5B0001FAEEB9741E050E0BE0167587F4FCE01E0
:10A5C00085579F4F0E942FDD9A2CAB2CB4CFBAE059
:10A5D000BB12FACFAB12F8CFCC24C394D12CCE014E
:10A5E00085579F4F0E9403DECD2809F498CFD701ED
:10A5F0005596ED90FC9061E07FE187EB9FE00E9433
:10A60000EAE14AE050E0B70187EB9FE00E948BE16E
:10A6100087EB9FE00E947EE064E670E080E090E0DF
:10A620000F942A110115110509F47DC1B8ECEB1640
:10A63000F10409F054C165EF7EE18AE09FE00E94D9
:10A64000EAE164EF71E080E090E00F942A11ED966A
:10A650001FAE1EAEED97EF961FAE1EAEEF978FEFBB
:10A660009FEFC158DF4F99838883CF57D04081E651
:10A6700094E0EB969FAF8EAFEB97CF57DF4F1983E8
:10A680000883C158D040F89490E080E00E946A3F6F
:10A690008111E6C069EE7EE182E19FE00E94EAE17D
:10A6A00082E19FE00E947EE0C8010E943DE824EF25
:10A6B000E22EFF24F394CE018F569F4F0E9403DEBB
:10A6C000C701CA56DF4F0FB6F894DEBF0FBECDBF2D
:10A6D000DF91CF911F910F91FF90EF90DF90CF907E
:10A6E000BF90AF909F908F907F906F905F904F90B2
:10A6F0000895D601ED91FC910084F185E02DC6010D
:10A700001995892B09F030CF64E670E080E090E085
:10A710000F942A111FCFBB24BA9467EB76E08AE12D
:10A720009FE00E94D4E1BE0165577F4F8AE19FE020
:10A730000E94DCE18AE19FE00E947EE0EB961FAE82
:10A740001EAEEB97ED961FAE1EAEED97EF961FAEC9
:10A750001EAEEF9768E37EE1CE0187589F4F0E94BF
:10A76000A6DDC157DF4F28813981CF58D040EF9601
:10A770008EAD9FADEF97912C2817390748F0BE0199
:10A7800067587F4FCE0185579F4F0F94F20D982E3B
:10A79000CE0187589F4F0E9403DE992079F1C1575F
:10A7A000DF4F28813981CF58D04049E050E0BE01C9
:10A7B00065577F4FCE0187589F4F0E9425DEEB964D
:10A7C0008EAD9FADEB97412C512C3201009719F0C3
:10A7D0000F94772A2B014201CE0187589F4F0E9488
:10A7E00003DE4114510429F0D70156965C924E9233
:10A7F0005597B4018AE19FE00F94C204F701858464
:10A80000968481149104D1F0C157DF4F88819981DA
:10A81000CF58D040892B91F0BE0165577F4FCE01B4
:10A8200087589F4F0E940BDECE0187589F4FF4013F
:10A830001995CE0187589F4F0E9403DE50E040E0FB
:10A8400065E279E0CE0185579F4F0E94CBDDFFEF97
:10A85000BF12BDCEC8010E943DE8D12CC12CBFCE95
:10A86000CE0187589F4F0F94E00C90936F0A80930E
:10A870006E0A7894C8010E943DE880916E0A90911A
:10A880006F0A892BD1F465E279E0CE0185579F4F9D
:10A890000E9414DECE0185579F4F0F94B11BCE014D
:10A8A00085579F4F0E9403DE62ED7EE182E19FE0CB
:10A8B0000E94EAE1F12CE12CFECE0E944C468091F0
:10A8C0006D0A882329F00F94E50370FF0E94C9AC3C
:10A8D0006BEC7EE18AE09FE00E94EAE1ECCEE0E3EF
:10A8E000EE16E1E0FE0651F467EB7EE18AE09FE0C0
:10A8F0000E94EAE1C8010E943DE8DDCE6FE97EE1F9
:10A9000082E19FE00E94EAE1C8010E943DE84AE03E
:10A9100050E0B70182E19FE00E948BE182E19FE07D
:10A920000E947EE0C8CE6CE87EE187EB9FE00E944B
:10A93000EAE1EE24EA94FE2CBECE4F925F926F9233
:10A940007F928F929F92AF92BF92CF92DF92EF92BF
:10A95000FF920F931F93CF93DF93CDB7DEB7C3570B
:10A96000D1400FB6F894DEBF0FBECDBF2091AB0A29
:10A970003091AC0AF9017196E532F10508F095C500
:10A980008827EA53FB4A8F4F0D9456323563206374
:10A99000555A555A555A555A61624D62555A555A2B
:10A9A000555A555A555A555A555A555A555AEB549F
:10A9B000D058F559095A8A5B345F4462555A555A42
:10A9C000555A555A555A82629562DB62B162555AA0
:10A9D000555A555ABF6280916D0A81E795E0C25978
:10A9E000DE4F99838883CE56D140C059DE4F1882FE
:10A9F00019821A821B82C057D140C859DE4F9983F1
:10AA00008883C856D140C659DE4F188219821A82EF
:10AA10001B82CA56D140CE59DE4F99838883C256D5
:10AA2000D140CC59DE4F188219821A821B82C4563B
:10AA3000D140CE5BDE4F99838883C254D140CC5B3A
:10AA4000DE4F188219821A821B82C454D14067EEED
:10AA500073E18AE09FE00E94EAE18AE09FE00E94C1
:10AA60007EE08091E60E9091E70E892B09F471C08B
:10AA70000F940001882309F46CC0A091E60EB091F8
:10AA8000E70E52961C921E92519754961C921E925B
:10AA9000539784E890E01D969C938E931C971E9686
:10AAA0001C921E9782E755968C935597ED91FC91D9
:10AAB00011970088F189E02D60E170E0CD011995D2
:10AAC00044E050E0BE016F5F7F4F8091E60E9091B1
:10AAD000E70E0E9400E089819A81AB81BC81C05958
:10AAE000DE4F88839983AA83BB83C057D14080916E
:10AAF000E60E9091E70EDC01ED91FC910488F5895A
:10AB0000E02D1995C059DE4F8881C057D140882368
:10AB100001F18F3FA9F4CF58DE4F8881C157D14052
:10AB20008F3F71F4CE58DE4F8881C257D1408F3F9E
:10AB300039F4CD58DE4F8881C357D1408F3F49F05B
:10AB40000F94E50371FF0FC180915A0A833008F01A
:10AB50000AC16BED73E18AE09FE00E94EAE10FB663
:10AB6000F894A895809160008861809360001092AD
:10AB700060000FBE8091510A81112AC01092390ADB
:10AB80001092380A88EE93E0A0E0B0E080933A0A91
:10AB900090933B0AA0933C0AB0933D0A8BEA94E061
:10ABA0009093370A8093360A81E795E09093450A9F
:10ABB0008093440A1092460A1092470A1092480A5B
:10ABC0001092490A84E080934E0A81E08093510AF2
:10ABD00083EF99E09093690D8093680D0F9489112C
:10ABE00080E590E00F94CD0C46E050E06EEE7EE004
:10ABF00089E090E00E944AE981E795E09A838983A1
:10AC00001B821C821D821E82CE0103960E94FCE9DB
:10AC10000E9411EA8091680D9091690DFC0112A2C9
:10AC200013A214A215A2DC0116A217A210A611A647
:10AC300012A613A614A615A640EE5EE260E070E030
:10AC400046AB57AB60AF71AF40EA5FE060E070E0E9
:10AC500042AF53AF64AF75AF189626E0FD01322FB7
:10AC600011923A95E9F7AC01425F5F4F34E1FA0186
:10AC700011923A95E9F7EEEEFEE001900D922A95D9
:10AC8000E1F7FC01EE5BFF4F10820E94CDF38C01D7
:10AC9000019709F046C080E590E00F94CD0C6091DB
:10ACA000680D7091690D625F7F4FCE0101960E9421
:10ACB0002FE2CE0103960E94FCE96091680D70912D
:10ACC000690D6A5E7F4FCE0101960E942FE2CE0190
:10ACD00003960E940AEA6091680D7091690D6E5E9C
:10ACE0007F4FCE0101960E942FE2CE0103960E9473
:10ACF00003EA0E9411EA6091680D7091690D625E2D
:10AD00007F4FCE0101960E942FE28B819C81AD8105
:10AD1000BE818093640D9093650DA093660DB093F2
:10AD2000670D88E199E20FB6F894A89580936000CA
:10AD30000FBE90936000A895012B09F0C4C261E793
:10AD400073E182E19FE00E94EAE162E473E182E163
:10AD50009FE00E94EAE180915A0A8F5F80935A0A2D
:10AD600086EF9FEF1FC265EC73E18AE09FE00E94CF
:10AD7000EAE181E795E09A838983C059DE4F8881B3
:10AD80009981AA81BB81C057D1408B839C83AD83BD
:10AD9000BE83CE0101960E9411A98091E60E90918A
:10ADA000E70E892B09F47AC20F940001882309F475
:10ADB00075C2A091E60EB091E70E52961C921E92BB
:10ADC000519754961C921E92539784E890E01D96DA
:10ADD0009C938E931C971E961C921E9782E7559605
:10ADE0008C935597ED91FC9111970088F189E02D96
:10ADF00064E170E0CD01199544E050E0BE016F5F61
:10AE00007F4F8091E60E9091E70E0E9400E08981CD
:10AE10009A81AB81BC81C659DE4F88839983AA830E
:10AE2000BB83CA56D1408091E60E9091E70EDC01BB
:10AE3000ED91FC910488F589E02D1995C659DE4FF6
:10AE40008881CA56D140882309F428C28F3FB1F4C3
:10AE5000C559DE4F8881CB56D1408F3F79F4C45914
:10AE6000DE4F8881CC56D1408F3F41F4C359DE4F2D
:10AE70008881CD56D1408F3F09F410C26FEB73E14A
:10AE80008AE09FE00E94EAE181E795E09A83898366
:10AE9000C659DE4F88819981AA81BB81CA56D140AB
:10AEA0008B839C83AD83BE83CE0101960E9411A942
:10AEB0008091E60E9091E70E892B09F4C0C10F94A2
:10AEC0000001882309F4BBC1A091E60EB091E70E02
:10AED00052961C921E92519754961C921E92539712
:10AEE00084E890E01D969C938E931C971E961C926E
:10AEF0001E9782E755968C935597ED91FC9111978B
:10AF00000088F189E02D68E170E0CD01199544E0F9
:10AF100050E0BE016F5F7F4F8091E60E9091E70E8B
:10AF20000E9400E089819A81AB81BC81CC59DE4FBF
:10AF300088839983AA83BB83C456D1408091E60E4F
:10AF40009091E70EDC01ED91FC910488F589E02DEC
:10AF50001995CC59DE4F8881C456D140882309F415
:10AF60006EC18F3FB1F4CB59DE4F8881C556D140B9
:10AF70008F3F79F4CA59DE4F8881C656D1408F3F42
:10AF800041F4C959DE4F8881C756D1408F3F09F43B
:10AF900056C16AEB73E18AE09FE00E94EAE181E733
:10AFA00095E09A838983CC59DE4F88819981AA8163
:10AFB000BB81C456D1408B839C83AD83BE83CE01BD
:10AFC00001960E9411A98091E60E9091E70E892BBF
:10AFD00009F4EDC00F940001882309F4E8C0A091A2
:10AFE000E60EB091E70E52961C921E92519754961F
:10AFF0001C921E92539784E890E01D969C938E932A
:10B000001C971E961C921E9782E755968C93559717
:10B01000ED91FC9111970088F189E02D6CE170E0D1
:10B02000CD01199544E050E0BE016F5F7F4F8091E4
:10B03000E60E9091E70E0E9400E089819A81AB8133
:10B04000BC81CC5BDE4F88839983AA83BB83C454C5
:10B05000D1408091E60E9091E70EDC01ED91FC91DC
:10B060000488F589E02D1995CC5BDE4F8881C454A6
:10B07000D140882309F49BC08F3FB1F4CB5BDE4FF6
:10B080008881C554D1408F3F79F4CA5BDE4F8881F7
:10B09000C654D1408F3F41F4C95BDE4F8881C7540D
:10B0A000D1408F3F09F483C063EB73E18AE09FE0F6
:10B0B0000E94EAE101E715E01A830983CC5BDE4FC9
:10B0C00088819981AA81BB81C454D1408B839C83A0
:10B0D000AD83BE83CE0101960E9411A91A83098314
:10B0E000CC5BDE4F88819981AA81BB81C454D14059
:10B0F0008B839C83AD83BE83CF57DF4F1983088337
:10B10000C158D040CC59DE4F88819981AA81BB813A
:10B11000C456D140CD57DF4F88839983AA83BB8320
:10B12000C358D040CE53DF4F19830883C25CD04050
:10B13000C659DE4F88819981AA81BB81CA56D14008
:10B14000CC53DF4F88839983AA83BB83C45CD040F0
:10B15000CE5FDE4F19830883C250D140C059DE4F05
:10B1600088819981AA81BB81C057D140CC5FDE4FD5
:10B1700088839983AA83BB83C450D1409E012F5FEB
:10B180003F4FAE014F575F4FBE016E537F4FCE0111
:10B190008E5F9E4F0F9419128AE09FE00E947EE01E
:10B1A00082E090E09093AC0A8093AB0A7EC181E785
:10B1B00095E09A838983CC59DE4F488159816A8111
:10B1C0007B81C456D1404B835C836D837E83CF5794
:10B1D000DF4F99838883C158D040C659DE4F4881DC
:10B1E00059816A817B81CA56D140CD57DF4F488350
:10B1F00059836A837B83C358D040CE53DF4F9983F2
:10B200008883C25CD040C059DE4F88819981AA8171
:10B21000BB81C057D140CC53DF4F88839983AA8329
:10B22000BB83C45CD040AE014F5F5F4FBE016F5720
:10B230007F4FCE018E539F4F0F945612ADCF81E7B3
:10B2400095E09A838983C659DE4F488159816A8186
:10B250007B81CA56D1404B835C836D837E83CF57FD
:10B26000DF4F99838883C158D040C059DE4F888111
:10B270009981AA81BB81C057D140CD57DF4F8883C8
:10B280009983AA83BB83C358D040BE016F5F7F4FB1
:10B29000CE018F579F4F0F94A8127ECF81E795E084
:10B2A0009A838983C059DE4F88819981AA81BB81A5
:10B2B000C057D1408B839C83AD83BE83CE01019662
:10B2C0000F94F31269CF62E373E18AE09FE00E947A
:10B2D000EAE1CE0101960F94FE0C8B819C81AD8139
:10B2E000BE81C059DE4F88839983AA83BB83C05730
:10B2F000D14001E715E01A830983CE0101960E942F
:10B3000011A98AE09FE00E947EE0CE0182599E4F03
:10B310000F9441028091640D9091650DA091660D8E
:10B32000B091670D8B839C83AD83BE83C659DE4F7E
:10B3300088839983AA83BB83CA56D140CE0188599A
:10B340009E4F0F9413031A8309831B821C821D8254
:10B350001E8280E590E00F94CD0C44E050E0BE01E9
:10B360006D5F7F4F81E090E00E941AE90E9411EA30
:10B370008B819C81AD81BE81CC59DE4F88839983BE
:10B38000AA83BB83C456D140CE018E599E4F0F94E1
:10B390007C031A8309831B821C821D821E8280E526
:10B3A00090E00F94CD0C44E050E0BE016D5F7F4F04
:10B3B00085E090E00E941AE90E9411EA8B819C814D
:10B3C000AD81BE81CC5BDE4F88839983AA83BB832A
:10B3D000C454D140CE018E5B9E4F0F94AA0281E0EF
:10B3E0000F94A30410925A0ADBCE8091600A811157
:10B3F0000DC06EE277E187EB9FE00E94EAE187EB08
:10B400009FE00E947EE081E08093600A83E090E00C
:10B41000C9CE80916D0A8091A70A81115FC10F94F6
:10B42000E50364FD2DC080915F0A81111EC00E945A
:10B430000B50883C910519F484E090E0B3CE8091E4
:10B440006D0A67E077E1811112C0CE0101960F9479
:10B45000FE0C8B819C81AD81BE81892B8A2B8B2B2D
:10B4600009F47ECC8FE090E09DCE67EF76E18AE034
:10B470009FE00E94EAE18AE09FE00E947EE0DCCF4C
:10B4800080916D0A882309F442C184E090E0909392
:10B49000AC0A8093AB0A6DEB76E18AE09FE00E94F4
:10B4A000EAE18AE09FE00E947EE00FB6F894A8955A
:10B4B00080916000886180936000109260000FBEF0
:10B4C0008091AB0A9091AC0A02970CF4F9C080917C
:10B4D0005A0A8111F5C00091680D1091690D01158E
:10B4E000110509F4EDC00F942A134B015C0178019A
:10B4F000FEE3EF0EF11CF70180819181A281B381FF
:10B50000A5019401281B390B4A0B5B0BCA01B90139
:10B51000683E33E0730781059105B0F128EE33E012
:10B5200040E050E00F94DF31861A970AA80AB90A62
:10B53000D7018D929D92AD92BC921397F80186A58A
:10B5400097A5A0A9B1A969017A01CC0CDD1CEE1C5C
:10B55000FF1C8C159D05AE05BF0510F00C945263C1
:10B5600016A617A610AA11AAF80182A993A9A4A940
:10B57000B5A98C159D05AE05BF0510F00C945C6354
:10B5800012AA13AA14AA15AAF80186A597A5A0A91C
:10B59000B1A9892B8A2B8B2B11F00C946663EE5B7F
:10B5A000FF4F8081833011F00C94666384E08083C8
:10B5B000C8010E94CDF301967C01F80182A993A9EC
:10B5C000A4A9B5A9892B8A2B8B2BA1F4EE5BFF4F85
:10B5D0008081833011F081110DC01082F8013E96F8
:10B5E00084E1DF011D928A95E9F7C8010E94CDF33D
:10B5F00003967C01B2E0EB16F10429F0E4E0EE16CC
:10B60000F10409F046C080E590E00F94CD0C609104
:10B61000680D7091690D625F7F4FCE0101960E94A7
:10B620002FE2CE0103960E94FCE96091680D7091B3
:10B63000690D6A5E7F4FCE0101960E942FE2CE0116
:10B6400003960E940AEA6091680D7091690D6E5E22
:10B650007F4FCE0101960E942FE2CE0103960E94F9
:10B6600003EA0E9411EA6091680D7091690D625EB3
:10B670007F4FCE0101960E942FE28B819C81AD818C
:10B68000BE818093640D9093650DA093660DB09379
:10B69000670DF3E0EF16F10411F40C94896314F0D4
:10B6A0000C946A6331E0E316F10411F40C948663A0
:10B6B00069E076E142E0E416F10411F40C948E6343
:10B6C00088E199E20FB6F894A895809360000FBEC8
:10B6D000909360002091AB0A3091AC0AC901CD581B
:10B6E000DE4F0FB6F894DEBF0FBECDBFDF91CF9116
:10B6F0001F910F91FF90EF90DF90CF90BF90AF9090
:10B700009F908F907F906F905F904F9008958FE003
:10B7100090E0BDCEA89580916D0A8091680A9091C5
:10B72000690A009721F00F94F000823068F46AEA09
:10B7300076E18AE09FE00E94EAE18AE09FE00E94D1
:10B740007EE087E090E02ECDCE59DE4F1882C256C3
:10B75000D140FE01EE5FFE4F119211928EE0DF01AB
:10B760001D928A95E9F70E94CBFF882319F085E0A6
:10B7700090E018CDE090680AF090690AE114F104B5
:10B7800041F0C7010F94F000082F10E002301105BE
:10B790005CF461E075E182E19FE00E94EAE182E110
:10B7A0009FE00E947EE05ECE70E060E0C7010E94F4
:10B7B000D71C009709F489C09093760A8093750A84
:10B7C00064EF74E18AE09FE00E94EAE16091750A0B
:10B7D0007091760A8AE09FE00E94D4E18AE09FE0BF
:10B7E0000E947EE0E090680AF090690A61E070E0F3
:10B7F000C7010E94D71C5C010230110509F468C022
:10B8000062E0C7010F945F00FC01C184D284033061
:10B81000110509F466C063E070E0C7010E94D71CFF
:10B820007C018091E60E9091E70E892B09F45EC0B1
:10B830000F940001882309F459C0A091E60EB0913D
:10B84000E70E52961C921E92519754961C921E928D
:10B85000539784E890E01D969C938E931C971E96B8
:10B860001C921E9782E755968C935597ED91FC910B
:10B8700011970088F189E02D60E470E0CD01199501
:10B880004FE050E0BE016E5F7E4F8091E60E9091DA
:10B89000E70E0F9455014C018091E60E9091E70E52
:10B8A000DC01ED91FC910488F589E02D1995811456
:10B8B0009104E1F0E2E0F1E0EC0FFD1FE80DF91D6D
:10B8C00010828E010E5F1E4F27C083E194E074CF7B
:10B8D000FBE5CF2EF7E0DF2E9E012E593E4F79017A
:10B8E000A0CFAE014E595E4F7A019BCF05301105B6
:10B8F00044F364E070E08091680A9091690A0E94C4
:10B90000D71C8C0164ED74E18AE09FE00E94EAE1BB
:10B910008AE09FE00E947EE0B092B00DA092AF0D51
:10B92000D092B20DC092B10D82E19EE39093A80D2A
:10B930008093A70D40E150E067EC74E1CE018E5397
:10B940009F4F0F94FC2A30E020E041E050E060E29D
:10B95000CE018F579F4F0E947DA840E250E062E1E8
:10B960007FE2CE018F579F4F0F94DE2A66EA74E183
:10B970008AE09FE00E94EAE1B5018AE09FE00E9430
:10B98000D4E164EA74E18AE09FE00E94EAE14AE0DF
:10B9900050E0B6018AE09FE00E948BE16DE974E11E
:10B9A0008AE09FE00E94EAE1B7018AE09FE00E94FE
:10B9B000D4E168E974E18AE09FE00E94EAE1F701DE
:10B9C0008081811104C010E000E0F12CE12CA090F6
:10B9D000750AB090760A0E94CBFF8111C6C1809192
:10B9E000920D9091930DDC01ED91FC910688F78901
:10B9F000E02D1995882309F498C081E090E0909398
:10BA00009D0D80939C0D87E0ECE4F2E0DE01119641
:10BA100001900D928A95E1F7FE01319685E090E064
:10BA20002191A091940DB091950DA80FB91F2C9361
:10BA300001968C309105A1F786E3E114F10429F019
:10BA400086EB0115110509F086EFC090940DD0909A
:10BA5000950DF60184878091990D85878091980DC9
:10BA600086878090960D9090970DB401C5010F9434
:10BA70000F2B41968816990608F08EC08091920D82
:10BA80009091930DDC01ED91FC910488F589E02DF6
:10BA9000199565E574E182E19FE00E94EAE1609119
:10BAA000B50D7091B60D4AE050E082E19FE00E9432
:10BAB0008BE16DE374E182E19FE00E94EAE182E1C3
:10BAC0009FE00E947EE080916A0A882379F0E091ED
:10BAD000680AF091690A828193819093690A809340
:10BAE000680A892B09F0B2C10E94681A0F942A13C0
:10BAF00060935B0A70935C0A80935D0A90935E0A80
:10BB00008091590A8F5F8093590A83330CF4A9C13D
:10BB10006FE074E182E19FE00E94EAE182E19FE050
:10BB20000E947EE01092590A1BC96091AF0D70917E
:10BB3000B00D8091920D9091930DDC01ED91FC91EF
:10BB40004091B10D5091B20D6115710571F00088F1
:10BB5000F189E02D1995019709F44FCF8EEF9FEFF2
:10BB60009093B60D8093B50D94CF0684F785E02DA4
:10BB700021E735E03A8329834090AB0D5090AC0D1E
:10BB80006090AD0D7090AE0D4B825C826D827E82B6
:10BB9000BE016F5F7F4FDECF4FE050E0B601C501C1
:10BBA0000F9403006C01A090960DB090970DB50115
:10BBB000CE018F579F4F0F940F2B8C0D9D1D02961A
:10BBC000A816B90608F45ACF6091940D7091950D9E
:10BBD000A601CE018F579F4F0F9403006C01A090D8
:10BBE000960DB090970DB501CE018E539F4F0F94D7
:10BBF0000F2B8C0D9D1D0296A816B90608F43ECF9A
:10BC00006091940D7091950DA601CE018E539F4FBA
:10BC10000F9403006C01E114F104B9F1A090960DAA
:10BC2000B090970DB501C7010F940F2B96012E5FB1
:10BC30003F4F820F931FA816B90608F41FCF6091DB
:10BC4000940D7091950DA601C7010F9403006C012E
:10BC500001151105D1F0E090960DF090970DB70108
:10BC6000C8010F940F2B96012E5F3F4F820F931F39
:10BC7000E816F90608F402CF6091940D7091950DC5
:10BC8000A601C8010F9403006C01A601455051099B
:10BC90006091940D7091950D80E10F9436130F947F
:10BCA0002A1360939E0D70939F0D8093A00D909327
:10BCB000A10D6093A20D7093A30D8093A40D90939A
:10BCC000A50D8091920D9091930DDC01ED91FC9169
:10BCD0000084F185E02D1995892B21F50F942A1305
:10BCE0000091A20D1091A30D2091A40D3091A50DEE
:10BCF0006B017C01C01AD10AE20AF30A20919A0D65
:10BD000030919B0DA8EEB3E00F943332C616D706E0
:10BD1000E806F906B0F28CEF9FEF9093B60D809392
:10BD2000B50DACCECE018E5B9E4F0F94A91764303B
:10BD300071058105910509F0A1CEE091940DF09176
:10BD4000950D838190E08111E8CF0F942A136093C1
:10BD5000A20D7093A30D8093A40D9093A50D109246
:10BD6000A60D1092B60D1092B50D1092590A6AE800
:10BD700074E18AE09FE00E94EAE16091750A7091A7
:10BD8000760A8AE09FE00E94D4E18AE09FE00E9468
:10BD90007EE081E080935F0A30E020E043E050E005
:10BDA00061E4CE0101960E947DA86AEB76E0CE01A7
:10BDB00001960F94AD36CE0101960F94FD1330E03D
:10BDC00020E042E050E061E4CE0101960E947DA8AF
:10BDD0006EEB76E0CE0101960F94AD36BE016F5F3B
:10BDE0007F4F87EB9FE00E9482E0CE0101960F9487
:10BDF000FD1330E020E041E050E061E4CE01019627
:10BE00000E947DA86EEB76E0CE0101960F94AD36D0
:10BE1000BE016F5F7F4F87EB9FE00E9482E0CE0103
:10BE200001960F94FD1385E090E09093AC0A809307
:10BE3000AB0A0F942A1360935B0A70935C0A809399
:10BE40005D0A90935E0A67E674E127CB64EF73E1C5
:10BE50008AE09FE00E94EAE18AE09FE00E947EE0A3
:10BE600045CE8CE090E09EC90F942A139B01AC0153
:10BE700060915B0A70915C0A80915D0A90915E0A04
:10BE8000A12CB12C650110E4E12E1FE1F12E00E0A0
:10BE900010E00E94B19A882309F407CB30E020E03B
:10BEA00043E050E061E4CE018F579F4F0E947DA890
:10BEB0006AEB76E0CE018F579F4F0F94AD3600911D
:10BEC000960D1091970DB801CE018F579F4F0F948B
:10BED0000F2B09960817190790F10E94CBFF8823B2
:10BEE00071F180919C0D90919D0D019609F441C1D5
:10BEF00090939D0D80939C0DE091940DF091950D84
:10BF000080919D0D8583E091940DF091950D809128
:10BF10009C0D86836091940D7091950D47E050E0E3
:10BF2000CE018F579F4F0F940300AC01455051092C
:10BF30006091940D7091950D82EA0F943613FE0175
:10BF4000EE5FFE4F119211921EE3DF01212F1D9231
:10BF50002A95E9F71A821982FE0133968EE7DF01EE
:10BF60001D928A95E9F730E020E041E050E060E47E
:10BF7000CE018E5F9E4F0E947DA84FE350E062E1AC
:10BF80007FE2CE018E5F9E4F0F94DE2A4FE750E096
:10BF90006CE07FE2CE0101960F94FC2ABE016F5F38
:10BFA0007F4FCE018E5F9E4F0F94C71330E020E08D
:10BFB00041E050E060E4CE018E5F9E4F0E947DA87C
:10BFC0004FE350E064ED75E1CE018E5F9E4F0F941C
:10BFD000DE2A4FE750E06AEC75E1CE0101960F943E
:10BFE000FC2A4FE750E067EB75E1CE0101960F9414
:10BFF000DE2ABE016F5F7F4FCE018E5F9E4F0F9492
:10C00000C71330E020E041E050E060E4CE018E5FF5
:10C010009E4F0E947DA84FE350E069E27FE2CE018F
:10C020008E5F9E4F0F94DE2A4FE750E067EA75E17E
:10C03000CE0101960F94FC2ABE016F5F7F4FCE01A7
:10C040008E5F9E4F0F94C71330E020E041E050E038
:10C0500060E4CE018E5F9E4F0E947DA84FE350E0CA
:10C0600060EA75E1CE018E5F9E4F0F94DE2A4FE7A6
:10C0700050E06AE975E1CE0101960F94FC2ABE01F9
:10C080006F5F7F4FCE018E5F9E4F0F94C7138091DD
:10C09000A70A8F5F8093A70AA091AD0AB091AE0A5C
:10C0A000109709F4DEC18091530290915402AE01C1
:10C0B0004E5B5E4FFA01819391932EE111922A9586
:10C0C000E9F79E012E533F4FF9018193919311920D
:10C0D0001A95E9F716960D911C91F12CE12C80919F
:10C0E000AD0A9091AE0A892B09F42FC101151105F3
:10C0F00009F42BC1D80118968C918F70853009F006
:10C10000FEC0C8010F94F000882309F4F8C0D801DC
:10C11000ED91FC91DF010D900020E9F7EE1AFF0A86
:10C12000EA0EFB1E60E0C8010F945F00FC018185F0
:10C130009285A385B48582319105A105B10550F59D
:10C14000FC018827E955FF498F4F0D9456328461D1
:10C150009761976184618461BC608461846184615A
:10C160008461CA60CA60CA60CA60CA60CA60CA60C4
:10C17000976181E090E0BCCE4FE150E064E975E169
:10C18000CE018E5B9E4F0F94FC2ACE53DF4F188258
:10C19000C25CD04030E020E041E050E060E4CE01FD
:10C1A0008E5F9E4F0E947DA8D8016D917C914FE3D8
:10C1B00050E0CE018E5F9E4F0F94D33660EC76E058
:10C1C000CE018E5F9E4F0F94AD3640E450E062E7A3
:10C1D00075E1CE018E5F9E4F0F94DE2A6DE675E10C
:10C1E000CE018E5F9E4F0F94CE1A30E020E041E0EA
:10C1F00050E060E4CE018E5F9E4F0E947DA8F80162
:10C20000608171814FE350E0CE018E5F9E4F0F94AD
:10C21000D33660EC76E0CE018E5F9E4F0F94AD3644
:10C2200040E450E065E675E1CE018E5F9E4F0F94CD
:10C23000DE2A64E475E1CE018E5F9E4F0F94CE1A24
:10C2400030E020E041E050E060E4CE018E5F9E4FA0
:10C250000E947DA8D8016D917C914FE350E0CE0102
:10C260008E5F9E4F0F94D33666EC76E0CE018E5FE4
:10C270009E4F0F94AD364FE350E062E775E1CE017B
:10C280008E5F9E4F0F94DE2ABE016E5B7E4FCE0105
:10C290008E5F9E4F0F94C713CE53DF4F8881C25CD1
:10C2A000D040882361F130E020E041E050E060E4DC
:10C2B000CE018E5F9E4F0E947DA8F8016081718142
:10C2C0004FE350E0CE018E5F9E4F0F94D33666EC65
:10C2D00076E0CE018E5F9E4F0F94AD364FE350E077
:10C2E00065E675E1CE018E5F9E4F0F94DE2ABE019A
:10C2F0006E537F4FCE018E5F9E4F0F94C713D801B0
:10C3000012960D911C91EBCE4FE150E06CE875E177
:10C31000CE018E5B9E4F0F94FC2A4FE350E066E8FF
:10C3200075E1CE018E539F4F0F94FC2A33CF4FE11E
:10C3300050E060E875E1CE018E5B9E4F0F94FC2AC1
:10C340004FE350E06CE775E1ECCF30E020E041E0F6
:10C3500050E060E4CE018E5F9E4F0E947DA84FE3C7
:10C3600050E06DE375E1CE018E5F9E4F0F94DE2AA3
:10C370000E94CBFF8823F1F16091940D7091950D8F
:10C3800045E050E0CE018E5F9E4F0F9403008C017C
:10C39000B6E0EB1AF108A701480F591F6091940D00
:10C3A0007091950D81E30F942500A091920DB091AD
:10C3B000930DA801480F591F4550510925E030E061
:10C3C000281B390B6091940D7091950D620F731FAE
:10C3D000ED91FC9111970280F381E02DCD0119952B
:10C3E0000F942A1360939E0D70939F0D8093A00D60
:10C3F0009093A10DE091AD0AF091AE0A06811781EC
:10C400008091AD0A9091AE0A892B59F10115110561
:10C4100041F1F80180858F708530F1F4C8010F94E7
:10C42000F0008823C9F0D8016D917C91FB01019047
:10C430000020E9F73197AF01461B570B8EE89DE0CE
:10C440000E9411DCF80182819381892B29F06CE232
:10C450008EE89DE00E9431DCD80112960D911C916E
:10C46000CFCF8091A70A81508093A70A86E090E001
:10C470009093AC0A8093AB0A6DE876E18AE09FE086
:10C480000E94EAE10C94555A80916D0A0E94CBFFFC
:10C4900081110C94555A0C941C5A0F942A136093D2
:10C4A0005B0A70935C0A80935D0A90935E0A85EF45
:10C4B0009FEF9093AC0A8093AB0A80916D0A0C9425
:10C4C000555A0F942A139B01AC0160915B0A70913D
:10C4D0005C0A80915D0A90915E0AA12CB12C6501E5
:10C4E00018E8E12E13E1F12E00E010E00E94B19A6D
:10C4F000882311F40C94555A1092AC0A1092AB0A8E
:10C500000C94555A0E94CBFF81110F94931A0F94EB
:10C510002A1360935B0A70935C0A80935D0A909380
:10C520005E0A8DE090E00C94D2580F942A139B0180
:10C53000AC0160915B0A70915C0A80915D0A9091F8
:10C540005E0AA12CB12C650110E1E12E17E2F12E5B
:10C5500000E010E00E94B19A81110C941C5A0C94D6
:10C56000555A0F942A1360935B0A70935C0A809368
:10C570005D0A90935E0A8EE090E00C94D2580F947E
:10C580002A139B01AC0160915B0A70915C0A809157
:10C590005D0A90915E0AA12CB12C650110ECE12E90
:10C5A00014EDF12E01E010E00E94B19A81110C947B
:10C5B000B0560C94555A0E94B94E009779F18130CB
:10C5C000910511F40C941C5A019611F00C94555AD3
:10C5D0000F942A139B01AC0160915B0A70915C0A75
:10C5E00080915D0A90915E0AA12CB12C650110E347
:10C5F000E12E15E7F12E00E010E00E94B19A8823A9
:10C6000011F40C94555A6AE676E182E19FE00E94AB
:10C61000EAE1F0E0E0E019950C94555A83E190E0EE
:10C620009093AC0A8093AB0A0F942A1360935B0A31
:10C6300070935C0A80935D0A90935E0A0C94555A3D
:10C640000E94CBFF81110F94931A0E94681A0F94D5
:10C650002A1360935B0A70935C0A80935D0A90933F
:10C660005E0A8FEE9FEF0C94D25880916D0A8091F4
:10C67000A70A811133C882E190E09093AC0A8093BD
:10C68000AB0A0E940B50883C910511F40C941C5A83
:10C6900080916D0A882311F40C94255A63E476E1A5
:10C6A0000C94375A821B930BA40BB50B86A797A744
:10C6B000A0ABB1AB0C94B45A821B930BA40BB50B7B
:10C6C00082AB93ABA4ABB5AB0C94C45AF12CE12C68
:10C6D0000C94DD5A54E0E516F104F1F06AE376E1DA
:10C6E00085E0E816F10411F00C94605B82E19FE0B4
:10C6F0000E94EAE182E19FE00E947EE086EF9FEFE8
:10C700009093AC0A8093AB0A0C94605B66E276E18E
:10C71000EDCF66EF75E1EACF6AED75E18AE09FE063
:10C720000E94EAE1CE0101960F94FE0CCE01019623
:10C730000E9411A98AE09FE00E947EE00C94605B59
:10C740002F923F924F925F926F927F928F929F9221
:10C75000AF92BF92CF92DF92EF92FF920F931F930F
:10C76000CF93DF93CDB7DEB7A6970FB6F894DEBFB1
:10C770000FBECDBF6C010F8B188F298F3A8F4B8F57
:10C780005C8F6D8F7E8F22E1E216F10480F5F70158
:10C79000EA52FB4F30813F8FCE0147960E944D2ACF
:10C7A00097FD04C0BC01C6010E94D82C898DD6011A
:10C7B00012968C9312978F898C931196EC91119706
:10C7C000EF70EC3008F06CC0F0E08827E551FC49D0
:10C7D0008F4F0D9456324E65146414649565F96359
:10C7E000136661659F659F659F65616561651F8EC5
:10C7F000D3CF10E0988D9F709D3008F0C2C4E92F10
:10C80000F0E08827E95FFB498F4F0D945632506462
:10C810004A666A664A66156615664A664A66C16869
:10C82000C1684A664A661C65988D9F709D3008F005
:10C8300013C1E92FF0E08827EF5DFB498F4F0D947E
:10C8400056325064FA64ED64466431642E64D164F7
:10C85000FC642C652C65BB64BB641C658E8DF60185
:10C8600087838D8DD60116968C9316978C8D159691
:10C870008C9315978B8D14968C93149711968C919D
:10C880001197807F892B11968C930AC08D8D9E8D78
:10C89000F6018683878190FB80F987838C8D858361
:10C8A000BF8DBB2309F464C0F60181818F702B2FEB
:10C8B00030E08217130609F45BC06BED70E187EB83
:10C8C0009FE00E94EAE1D60111966C916F704AE0F8
:10C8D00050E087EB9FE00E94A1E068ED70E187EBFC
:10C8E0009FE00E94EAE14AE050E06F8D87EB9FE015
:10C8F0000E94A1E066ED70E187EB9FE00E94EAE113
:10C90000F601008119821A821B821C821D821E82FE
:10C910001F8218868F8D8F709A81907F892B8A83D2
:10C920000983EE24EA94FE2C118122813381448113
:10C93000558166817781CE0101960E94A063D60160
:10C940002C9311963C93119712964C931297139631
:10C950005C93139714966C93149715967C93159784
:10C9600016968C93169717969C93C6010E948C2C52
:10C9700088E0F60168C18B8D9C8DAD8DBE8DB7FDB5
:10C980000EC08F3F9105A105B10529F024F08FEF6E
:10C9900090E0A0E0B0E0D60114968C9381CF80E0C7
:10C9A000FACF6B8D7C8D8D8D9E8D20E06D39BFEF24
:10C9B0007B078B079B076CF02FEF6115E4E67E0782
:10C9C0008105910534F424E630E040E050E00F9416
:10C9D0000132D60114962C9363CF8D8D9E8DF60176
:10C9E0008683878190FB80F987838C8D85838B8DEF
:10C9F000848356CF8B8DCFCF8B8C9C8CAD8CBE8C93
:10CA000020E030E0A901C501B4010F94953060E049
:10CA100087FD0FC020E030E04FE753E4C501B401CB
:10CA20000F949D336FEF181624F0C501B4010F94D5
:10CA30006E33F601648334CFD60111968C91119731
:10CA4000807F8C6011968C9311978B8D9C8D1596A1
:10CA50009C938E93149724CF6BE571E187EB9FE055
:10CA60000E94EAE1688D6F704AE050E087EB9FE03A
:10CA70000E94A1E068E571E187EB9FE00E94EAE196
:10CA8000F60161816F704AE050E087EB9FE00E9401
:10CA9000A1E087EB9FE00E947EE002CF988D9F701F
:10CAA00011968C911197807F892B11968C938B8D89
:10CAB0009C8DAD8DBE8DF60184839583A683B7834F
:10CAC000EFCE988D9F70933089F09C3009F4B4CFED
:10CAD0004B8D5C8D6D8D7E8DF60144835583668311
:10CAE00077838181807F892B8183DACE60E0C601E4
:10CAF0000E94A627D60114968C9314978D8D9E8D37
:10CB000016968C93169717968C91179790FB80F931
:10CB100017968C9317978C8D15968C931597119665
:10CB20008C911197807F8260AECE60E0CE014796F7
:10CB30000E94A627D60114968C931497F0CF988D57
:10CB40009F709D3008F057C0E92FF0E08827E4552A
:10CB5000FA498F4F0D9456325064C665F365766579
:10CB6000F365F365B965E565E565E565D465E0659B
:10CB70001C658B8D9C8DAD8DBE8DF6018483958358
:10CB8000A683B7838181807F8660AECF6B8D70E096
:10CB900090E080E00F949A30D60114966D937D93C7
:10CBA0008D939C9317977CCE6B8D7C8D8D8D9E8DF8
:10CBB0000F949C30F601648375838683978370CECF
:10CBC0006B8D7C8D8D8D9E8DE5CFF6018181807F73
:10CBD000982B91838B8D9C8DAD8DBE8D8483958399
:10CBE000A683B7835DCE11968C911197807F982B89
:10CBF00011969C935CCF66E471E187EB9FE00E9405
:10CC0000EAE1688D6F704AE050E087EB9FE00E9498
:10CC1000A1E063E471E187EB9FE00E94EAE1D601C5
:10CC200011966C912FCF11E0E5CD4B8D5C8D6D8D04
:10CC30007E8DF60144835583668377838181807F6F
:10CC4000982B918388E0DE01119601900D928A95D0
:10CC5000E1F729813A814B815C816D817E818F81F1
:10CC60009885A6960FB6F894DEBF0FBECDBFDF91B4
:10CC7000CF911F910F91FF90EF90DF90CF90BF90D9
:10CC8000AF909F908F907F906F905F904F903F906C
:10CC90002F900895963009F442C148F46B8D91307D
:10CCA00071F06FEF70E0933051F060E008C09730A2
:10CCB00009F441C19A506B8D7C8D9230B0F784E6B7
:10CCC0008D8F8E8D8E7F8E8F1C8E888D807F826063
:10CCD000888F6B8F2C8D30E0AFEFB0E00F94333244
:10CCE000812C912C54018A946115F4E67F0781050B
:10CCF000910544F424E630E040E050E00F94013226
:10CD000049015A0114012B8D28A3E22EF12C112385
:10CD100009F474C08E8D8695A82FA150BB0B8D0190
:10CD20000F3F100709F027C1E0E88E1691040CF0C0
:10CD300009C18FE790E0881999098E9DD0018F9DD8
:10CD4000B00D9E9DB00D11242FEF30E00F946D3289
:10CD500021E83EE740E050E00F940132D6011796FB
:10CD60002C93ABE9B0E0A50194010F9420322FE79A
:10CD7000422E512C612C712CA30192010F9401328F
:10CD80002C593F4F4F4F5F4F1901AEEFB1E0A50156
:10CD900094010F942032A30192010F940132D70124
:10CDA0000F9420322FEF30E040E050E00F9401323A
:10CDB00079012F3F310521F01CF0EE24EA94F12C8B
:10CDC00066E371E187EB9FE00E94EAE14AE050E010
:10CDD000B10187EB9FE00E948BE168E271E187EB94
:10CDE0009FE00E94EAE14AE050E0B70187EB9FE054
:10CDF0000E948BE187EB9FE00E947EE030E020E024
:10CE000050E040E070E060E0CE0101960E94F5E362
:10CE1000122D2D8D3E8D3170AFEFBFEF0F94333259
:10CE20002DE631E040E050E00F94013244275527D1
:10CE3000AAEFB5E00F942032DC01CB019058AF4F40
:10CE4000BF4FCD01BB2797FDB095AB2F8E3FE1E0E3
:10CE50009E0708F06FC1382F8F3F910508F48CC1F1
:10CE60004EEF481B50E03FEFF701319633242FEF90
:10CE7000221A320A1095012F10E0329DC001339D15
:10CE8000900D1124292F3327200F311FDF010F941C
:10CE90006D324B015C018824AA24BB24529D900171
:10CEA000539D300D1124232F3327200F311F0F9452
:10CEB0006D32BB27A92F982F872F882A992AAA2A53
:10CEC000429D9001439D300D1124232F3327200FC5
:10CED000311FDF010F946D32B82FA72F962F8827AF
:10CEE00088279927BB2788299929AA29F601A6838B
:10CEF000958384836CEF70E187EB9FE00E94EAE109
:10CF0000C6010E948C2C8A859B850F9425288F81D1
:10CF1000988597FDC5CC60E00F94E50EC1CC6B8D74
:10CF20007C8D8D8D9E8D24E630E040E050E00F94A6
:10CF30000132B901C4CE6B8D7C8D8D8D9E8D0F9489
:10CF40006733BDCEA501940120583109410951092B
:10CF5000ABE9B0E00F9420322FE730E040E050E042
:10CF60000F9401322C593F4F4F4F5F4F1901D6019B
:10CF700017961C9225CF9801AAEBBFEF0F9465324C
:10CF800024E630E040E050E00F94013229013A01FC
:10CF9000B4E64B0E511C611C711C26E430E0D80134
:10CFA0000F946D3224E630E040E050E00F940132FF
:10CFB000DA01C9014E96A11DB11D8BA39CA3ADA39F
:10CFC000BEA390E8891691040CF099C08FE790E019
:10CFD000881999098E9DD0018F9DB00D9E9DB00D31
:10CFE00011242BA13CA14DA15EA10F942B329B01DA
:10CFF000AC01AFEFB0E00F94203224E63AE640E017
:10D0000050E00F940132D60117962C93A50194019C
:10D01000240D351D461D571DAEEFB1E00F94203293
:10D0200023EE30E040E050E00F94013279018A01B4
:10D030003AA329A3AFEFB0E0A50194010F942032E9
:10D040002FE730E040E050E00F9401321901E8A1F1
:10D05000AE2FB0E0A80197010F9420322FEF30E0FF
:10D0600040E050E00F94013279012F3F310521F06B
:10D070001CF0EE24EA94F12C62E271E187EB9FE070
:10D080000E94EAE12AE030E0B301A20187EB9FE0D1
:10D090000E9443E16CE171E187EB9FE00E94EAE1CD
:10D0A0002AE030E04BA15CA16DA17EA187EB9FE05F
:10D0B0000E9443E164E171E187EB9FE00E94EAE1B5
:10D0C0004AE050E0B10187EB9FE00E948BE16CE009
:10D0D00071E187EB9FE00E94EAE14AE050E0B7018E
:10D0E00087EB9FE00E948BE163E071E187EB9FE0BB
:10D0F0000E94EAE14AE050E069A17AA177CEA50159
:10D1000094012058310941095109ABE9B0E00F946D
:10D1100020322FE730E040E050E00F9401322C59EC
:10D120003F4F4F4F5F4F1901D60117961C921AA21D
:10D1300019A2A2CF8C3FF3E09F0768F48D3F22E055
:10D14000920728F452E0580F3FEF40E08DCE3CEFBD
:10D15000381B5FEFFACF8A3F35E0930781F08B3FB2
:10D16000E4E09E0728F444E0480F5FEF30E07CCE17
:10D170005AEF581B30E001C050E04FEF75CE50E041
:10D18000F9CF6AEE70E187EB9FE00E94EAE1688DDB
:10D190006F704AE050E087EB9FE00E94A1E067EEED
:10D1A00070E139CD2F923F924F925F926F927F92B2
:10D1B0008F929F92AF92BF92CF92DF92EF92FF92A7
:10D1C0000F931F93CF93DF93CDB7DEB7CC5CD1091C
:10D1D0000FB6F894DEBF0FBECDBF1C01CF54DF4F9A
:10D1E0000883C15BD040CE54DF4F1883C25BD04070
:10D1F000CD54DF4F2883C35BD040CC54DF4F3883FE
:10D20000C45BD040CB54DF4F4883C55BD040CA5489
:10D21000DF4F5883C65BD040C954DF4F6883C75B7C
:10D22000D040C854DF4F7883C85BD040C754DF4F2D
:10D23000F982E882C95BD040CD53DF4FC882C35C1E
:10D24000D040CC53DF4FA882C45CD0400E94FEA9DE
:10D250006B01CB53DF4F79836883C55CD040683C5A
:10D260007105B4F46FE57CE082E19FE00E94EAE1A1
:10D270004AE050E0B60182E19FE00E948BE182E14A
:10D280009FE00E947EE0AA24AA94BA2C0C94EC722F
:10D290000F942A13C753DF4F688379838A839B8354
:10D2A000C95CD040CD54DF4F8881C35BD040282F6C
:10D2B00030E0C154DF4F39832883CF5BD040809169
:10D2C000AB0A9091AC0AC953DF4F99838883C75C3E
:10D2D000D040C754DF4FE881F981C95BD040309717
:10D2E00021F0808181110C945278D1011D968C918E
:10D2F000882341F0C1010D96C754DF4F998388837D
:10D30000C95BD040C154DF4FE881F981CF5BD04089
:10D31000EF2B11F00C94AE78C754DF4FE881F98100
:10D32000C95BD040309711F00C945B78D1015D96C9
:10D330000D90BC91A02DC154DF4FB983A883CF5B62
:10D34000D040AB2B11F40C94AE78CD54DF4F8881D4
:10D35000C35BD04081110C94AE78C154DF4F68811B
:10D36000CF5BD040CE018F549F4F0E94B721C7564C
:10D37000DF4F2883C959D040C656DF4F3883CA597A
:10D38000D040C556DF4F4883CB59D040C456DF4FFD
:10D390005883CC59D040C356DF4F6883CD59D04015
:10D3A000C256DF4F7883CE59D040C156DF4F8883B5
:10D3B000CF59D040C056DF4F9883C05AD0400C940C
:10D3C000AE78D10112962D913C91232B09F45BCFBD
:10D3D000C154DF4FE881F981CF5BD040349799F594
:10D3E000CC53DF4FE880C45CD040CF54DF4F08817E
:10D3F000C15BD040CE54DF4F1881C25BD040CD54CA
:10D40000DF4F2881C35BD040CC54DF4F3881C45BF1
:10D41000D040CB54DF4F4881C55BD040CA54DF4F6A
:10D420005881C65BD040C954DF4F6881C75BD0408C
:10D43000C854DF4F7881C85BD040C1010E944F299A
:10D440005C010C94EC7228E0FE01EF54FF4FDE010A
:10D45000A755BF4F01900D922A95E1F7CF54DF4FAA
:10D460001881C15BD040143009F40BC348F4112378
:10D4700009F469C0912C812CAA24AA94BA2C85C3E2
:10D4800088EF810F8230B0F788E0FE01EF54FF4F44
:10D49000DE01119601900D928A95E1F7CE54DF4F8F
:10D4A0008881C25BD0408F7009F47EC3CE018F5457
:10D4B0009F4F0E94022A4B015C0181149104A10438
:10D4C000B10409F471C3193041F4B094A09490945C
:10D4D0008094811C911CA11CB11CB101CE018F5400
:10D4E0009F4F0F94CE0560E0CE018F549F4F0E9456
:10D4F000D9216A962FAF6A976B963FAF6B976C9660
:10D500004FAF6C976D965FAF6D976E966FAF6E97DE
:10D510006F967FAF6F97A0968FAFA097A1969FAFA2
:10D52000A197C154DF4FA881B981CF5BD040A23011
:10D53000B10509F492C30CF03DC3AB2B09F4CAC387
:10D54000912C812C4EC519821A821B821C821D824D
:10D550001E821F8218862A81207F2A83CE54DF4FA5
:10D560002881C25BD0402F7009F484CFC154DF4FB3
:10D5700008811981CF5BD0400A30110509F439C206
:10D5800054F40115110571F10230110509F4E1C0DF
:10D59000912C812C25C2C154DF4F28813981CF5B6A
:10D5A000D0402B30310509F4CDC12C30310581F745
:10D5B000B101CE0101960F94CE05CE018F549F4F3D
:10D5C0000E944D2ABC01CE0101960E94D82C88E011
:10D5D000FE013196DE01AF54BF4F01900D928A9546
:10D5E000E1F7FBC1892B59F06CE17CE087EB9FE010
:10D5F0000E94EAE187EB9FE00E947EE0C9CFC10173
:10D600000E94F1798C0161E070E01816190614F09F
:10D6100070E060E04AE050E087EB9FE00E948BE121
:10D6200062EA77E087EB9FE00E94D4E1CE018F545D
:10D630009F4F0E940B29AB01BC012AE030E087EB31
:10D640009FE00E9443E187EB9FE00E947EE0CE01D5
:10D650008F549F4F1016110614F00C9440780E94BE
:10D660000B29672B682B692B09F063C162E0CE019F
:10D670008F549F4F0E94D921CF56DF4F2883C15925
:10D68000D040CE56DF4F3883C259D040CD56DF4F01
:10D690004883C359D040CC56DF4F5883C459D0403B
:10D6A000CB56DF4F6883C559D040CA56DF4F7883C9
:10D6B000C659D040C956DF4F8883C759D040C85695
:10D6C000DF4F9883C859D04088248394982C31E048
:10D6D000C554DF4F3883CB5BD0405524539442C0B0
:10D6E00061E0CE018F549F4F0E94D921C757DF4F71
:10D6F0002883C958D040C657DF4F3883CA58D04016
:10D70000C557DF4F4883CB58D040C457DF4F5883AD
:10D71000CC58D040C357DF4F6883CD58D040C25754
:10D72000DF4F7883CE58D040C157DF4F8883CF5822
:10D73000D040C057DF4F9883C059D040882483948D
:10D74000982C81E0C554DF4F8883CB5BD040512CAF
:10D7500009C0912C812CC554DF4F1882CB5BD0407F
:10D7600055245A94B101CE0101960F94CE058A81B9
:10D770009CE0980F9F70923058F4CE54DF4F988100
:10D78000C25BD0409F70923019F4807F82608A83A0
:10D79000D1011A969C91973069F4CE54DF4F88815D
:10D7A000C25BD0408F708250843020F48A81807FA9
:10D7B00082608A83F101A385B485892F90E0109758
:10D7C00041F0ED91FC911197048CF58DE02DCD0188
:10D7D00019957C01CF54DF4F0881C15BD040CE54F6
:10D7E000DF4F1881C25BD040CD54DF4F2881C35B2F
:10D7F000D040CC54DF4F3881C45BD040CB54DF4F96
:10D800004881C55BD040CA54DF4F5881C65BD040C9
:10D81000C954DF4F6881C75BD040C854DF4F78815F
:10D82000C85BD040CE0101960E94A063CF57DF4F66
:10D830002883C158D040CE57DF4F3883C258D040DC
:10D84000CD57DF4F4883C358D040CC57DF4F588364
:10D85000C458D040CB57DF4F6883C558D040CA5713
:10D86000DF4F7883C658D040C957DF4F8883C758E9
:10D87000D040C857DF4F9883C858D040CE0101969A
:10D880000E948C2CC554DF4FF881CB5BD040FF2326
:10D8900041F1CE54DF4F8881C25BD0408F709FE052
:10D8A000980F9F70923020F08A5F8F708230C8F49A
:10D8B0008A818F7081508230A0F42D8130E0AFEFEB
:10D8C000B0E00F9433322FEF611504E67007810545
:10D8D000910534F424E630E040E050E00F9401324A
:10D8E0002D8388E0FE013196DE01AF54BF4F0190D9
:10D8F0000D928A95E1F712E1912AF12CAA24AA94BB
:10D90000BA2CD1011A968C911A97873009F08DC5DF
:10D91000CB53DF4FE881F981C55CD040EE35F14053
:10D920000CF08CC368ED7BE082E19FE00E94EAE1AD
:10D93000A6CC912C812C91E0C554DF4F9883CB5B12
:10D94000D040CBCEB101CE0101960F94CE05CA5482
:10D95000DF4F8881C65BD0409A819F7039F092304A
:10D9600049F0912C812CFF24F3943BC09A81907F45
:10D9700092609A8390E08536910514F084E690E0F9
:10D980008E8388E0FE013196DE01AF54BF4F0190D7
:10D990000D928A95E1F762E0CE018F549F4F0E946D
:10D9A000B721EA962FAFEA97EB963FAFEB97EC964D
:10D9B0004FAFEC97ED965FAFED97EE966FAFEE97AA
:10D9C000EF967FAFEF97C158DF4F8883CF57D04096
:10D9D000C058DF4F9883C058D040812CF2E19F2E71
:10D9E000F12CC554DF4F1882CB5BD04055245A949C
:10D9F00085CFB101CE0101960F94CE05C954DF4FFA
:10DA00006881C75BD040C854DF4F7881C85BD04085
:10DA10007170CE0101960E94122DC554DF4F88838C
:10DA2000CB5BD040912C812CFF24F3948823F1F21E
:10DA300088E0FE013196DE01AF54BF4F01900D9298
:10DA40008A95E1F762E0CE018F549F4F0E94B72183
:10DA5000E2962FAFE297E3963FAFE397E4964FAF9E
:10DA6000E497E5965FAFE597E6966FAFE697E796A2
:10DA70007FAFE797E8968FAFE897E9969FAFE99772
:10DA8000ACCFC154DF4F28813981CF5BD0402930E2
:10DA9000310509F461C0C1010E94F1791816190617
:10DAA00074F562E0CE018F549F4F0E94D921AA964F
:10DAB0002FAFAA97AB963FAFAB97AC964FAFAC9753
:10DAC000AD965FAFAD97AE966FAFAE97AF967FAFA7
:10DAD000AF97E0968FAFE097E1969FAFE1978824EC
:10DAE0008394982CAA24AA94BA2CF12C31E0C55422
:10DAF000DF4F3883CB5BD0405524539402CF61E095
:10DB0000CE018F549F4F0E94D921A2962FAFA2978A
:10DB1000A3963FAFA397A4964FAFA497A5965FAFE8
:10DB2000A597A6966FAFA697A7967FAFA797A8963B
:10DB30008FAFA897A9969FAFA99788248394982C14
:10DB4000AA24AA94BA2CF12C81E0C554DF4F888313
:10DB5000CB5BD040512CD5CE40E050E061E070E08E
:10DB6000C1010E943A35672B682B692BA9F040E070
:10DB700050E061E070E0C1010E94E83488248394A1
:10DB800024E0922EAA24A394B12CF12CC554DF4F8B
:10DB90001882CB5BD040DBC040E050E061E070E039
:10DBA000C1010E941135EACF95E0892E912CA12C5C
:10DBB000B12C89CCC154DF4FE881F981CF5BD040D3
:10DBC000EA30F10509F4B1C13B9709F0B9CCCE5464
:10DBD000DF4F8881C25BD0408F70823009F021C254
:10DBE000C501B40124E630E040E050E00F9401327A
:10DBF000CA54DF4F8881C65BD04090E0280F391FA0
:10DC000037FF02C030E020E02536310514F024E66D
:10DC100030E0CA54DF4F2883C65BD04062E0CE01BB
:10DC20008F549F4F0E94B7212A962FAF2A972B9689
:10DC30003FAF2B972C964FAF2C972D965FAF2D971C
:10DC40002E966FAF2E972F967FAF2F9760968FAF40
:10DC5000609761969FAF6197C1C1C554DF4F18822D
:10DC6000CB5BD040D1011B968D919C911C97009766
:10DC700009F037C01A968C9190E000E5402E512CA7
:10DC8000612C712C8530910549F0412C512C3201C9
:10DC9000449721F0412C512C32014A94CE54DF4F4D
:10DCA000E881C25BD040EF70E150EB3008F02EC14C
:10DCB000F0E08827E15AF1498F4F0D945632796E82
:10DCC000796E866F866F866F536F196F196F196F34
:10DCD000AA6EAA6EF1E0C554DF4FF883CB5BD0404B
:10DCE000C1CFDC01ED91FC91048CF58DE02D1995EF
:10DCF000C4CFCB54DF4F1881C55BD040C501B40100
:10DD000024E630E040E050E00F940132DA01C9012E
:10DD1000810F911DA11DB11DB7FF03C080E090E0F0
:10DD2000DC018F3F9105A105B10529F024F08FEFAB
:10DD300090E0A0E0B0E0CB54DF4F8883C55BD040DB
:10DD4000812C12E1912EF12CAA24AA94BA2C5524EC
:10DD50005A94D7CDCB54DF4FC880D980EA80FB805E
:10DD6000C55BD040B4E68B169104A104B104DCF588
:10DD7000A4E6B0E0A70196010F942032860E971E0C
:10DD8000A81EB91E4114510461047104B9F0A30125
:10DD900092010F942032362F272FB501A40177FF6F
:10DDA00003C040E050E0BA01832E922E5C0148157A
:10DDB00059056A057B0514F44A015B01CB54DF4F1A
:10DDC00088829982AA82BB82C55BD040CE54DF4F45
:10DDD0008881C25BD040807F8660CE54DF4F8883CD
:10DDE000C25BD040ADCFC501B40124E630E040E0D5
:10DDF00050E00F940132C20ED31EE41EF51E4114F2
:10DE000051046104710461F0F7FE03C0C12CD12CF0
:10DE100076014C145D046E047F0414F473016201F6
:10DE2000CB54DF4FC882D982EA82FB82C55BD040E7
:10DE300087CFCB54DF4F688179818A819B81C55B15
:10DE4000D0400F9467336B017C01C501B40124E617
:10DE500030E040E050E00F940132CA01B9016C0D8E
:10DE60007D1D8E1D9F1D411451046104710481F0BC
:10DE70006B017C01F7FE03C0C12CD12C7601C701D8
:10DE8000B601461657066806790614F4C301B201B6
:10DE90000F949C30CB54DF4F688379838A839B83B4
:10DEA000C55BD0404DCFCB54DF4F88819981AA818B
:10DEB000BB81C55BD040880E991EAA1EBB1E4114B3
:10DEC000510461047104C9F0A4E6B0E0A301920119
:10DED0000F942032362F272FB501A40177FF03C0FE
:10DEE00040E050E0BA01832E922E5C01481559059E
:10DEF0006A057B0514F44A015B01CB54DF4F88822D
:10DF00009982AA82BB82C55BD0401ACF88E0FE010D
:10DF10003196DE01AF54BF4F01900D928A95E1F723
:10DF2000912C812CFF24F3940FCFCE54DF4F8881A6
:10DF3000C25BD0408F70823009F055C0C501B4017A
:10DF400024E630E040E050E00F940132C954DF4F46
:10DF50008881C75BD040C854DF4F6881C85BD04020
:10DF6000962F9170280F391F2E36E1E03E072CF4D2
:10DF700037FF05C02DE631E002C030E020E0C95493
:10DF8000DF4F2883C75BD040C854DF4F8881C85B10
:10DF9000D04030FB80F9C854DF4F8883C85BD04045
:10DFA00062E0CE018F549F4F0E94B72162962FAF3F
:10DFB000629763963FAF639764964FAF6497659699
:10DFC0005FAF659766966FAF669767967FAF679707
:10DFD00068968FAF689769969FAF6997812CB2E179
:10DFE0009B2EF12C18C088E0FE013196DE01AF5463
:10DFF000BF4F01900D928A95E1F760E17CE082E1EC
:10E000009FE00E94EAE182E19FE00E947EE0912C85
:10E01000812CFF24F394C554DF4F1882CB5BD04092
:10E0200093CE88E0FE013196DE01AF54BF4F0190E0
:10E030000D928A95E1F764E07CE0E1CFCD53DF4FAC
:10E040001881C35CD040112309F470C01496ED917F
:10E05000FC9180858F70853009F075C0C953DF4F02
:10E06000E881F981C75CD040359709F46CC0C101E3
:10E070000E94F17921E0181619060CF020E0522ECA
:10E08000C754DF4F28813981C95BD040D101149634
:10E090006D917C91CC53DF4F0881C45CD040AE01C0
:10E0A0004F545F4FC1010E940579C154DF4FE88191
:10E0B000F981CF5BD040319709F045C0CE54DF4F96
:10E0C0008881C25BD0408F70F1F1CC53DF4FC880A4
:10E0D000C45CD040E52CC755DF4F0881C95AD040F9
:10E0E000C655DF4F1881CA5AD040C555DF4F288129
:10E0F000CB5AD040C455DF4F3881CC5AD040C3559D
:10E10000DF4F4881CD5AD040C255DF4F5881CE5A9B
:10E11000D040C155DF4F6881CF5AD040C055DF4F46
:10E120007881C05BD040C1010E948038CF54DF4F5E
:10E130008881C15BD040853009F448C150F48330F8
:10E14000B9F1D12CC3C0CD53DF4F1882C35CD0408E
:10E15000EDCF863009F482C0873099F7C1010E9463
:10E160007C3A182F863009F066C06CEA7BE087EBBA
:10E170009FE00E94EAE14AE050E066E070E087EB51
:10E180009FE00E948BE187EB9FE00E947EE062E0CF
:10E19000CE018F549F4F0E94D92129AF3AAF4BAF88
:10E1A0005CAF6DAF7EAF8FAF21969FAF21973FC021
:10E1B000C1010E947C3A853021F093E0A92EB12C58
:10E1C0000BC263EC7BE087EB9FE00E94EAE14AE050
:10E1D00050E065E070E087EB9FE00E948BE187EB09
:10E1E0009FE00E947EE0B101CE018F549F4F0F94BB
:10E1F000CE0561E0CE018F549F4F0E94D921229617
:10E200002FAF229723963FAF239724964FAF2497A3
:10E2100025965FAF259726966FAF269727967FAFF7
:10E22000279728968FAF289729969FAF29976894AC
:10E2300080F890F886CF6EE87BE087EB9FE00E9445
:10E24000EAE1612F70E04AE050E087EB9FE00E9436
:10E250008BE187EB9FE00E947EE0AFCF40E050E093
:10E2600061E070E0C1010E943A35672B682B692B91
:10E2700009F0A9C0FFEF5F120EC0C1010E94F17941
:10E28000512C181619064CF464E77BE087EB9FE0ED
:10E290000E94EAE192CF5110F7CFB101CE018F5425
:10E2A0009F4F0F94CE0561E0CE018F549F4F0E9487
:10E2B000D92129AB3AAB4BAB5CAB6DAB7EAB8FAB33
:10E2C00098AF689480F890F8E6E0DE2E8401016053
:10E2D000CD54DF4F8881C35BD040823050F4CF549F
:10E2E000DF4F8881C15BD040882319F08401016031
:10E2F0001160CE54DF4F8881C25BD0408F7009F42B
:10E3000089C01260CD53DF4F2881C35CD0402111FA
:10E310001D7FA801B101CE018F549F4F0E94D139BA
:10E320004801AA24A394B12CF1106AC7D1011B960D
:10E330008D919C91009709F0A8C340E050E062E005
:10E3400070E0C1010E943A35672B682B692B09F4F4
:10E35000CEC360E37AE082E19FE00E94EAE182E1DD
:10E360009FE00E947EE092FC76C66EEF79E087EB3C
:10E370009FE00E94EAE14AE050E0B50187EB9FE0B0
:10E380000E948BE167EF79E087EB9FE00E94EAE172
:10E390000F942A13AB01BC01C753DF4F08811981C9
:10E3A0002A813B81C95CD040401B510B620B730B2F
:10E3B0002AE030E087EB9FE00E9499E087EB9FE046
:10E3C0000E947EE009C16FE57BE060CF0FEF501245
:10E3D0000BC0C1010E94F1795524539418161906F7
:10E3E0002CF062E47BE052CF5520D9F362E0CE01FD
:10E3F0008F549F4F0E94D92129A73AA74BA75CA70A
:10E400006DA77EA78FA798AB689480F890F875E009
:10E41000D72E5CCF40E052E0B101CE018F549F4F28
:10E420000E94893A81116DCF6DCF3FEF53129DC08D
:10E43000C1010E94F17955245394181619060CF461
:10E4400097C0512C64E37BE087EB9FE00E94EAE1F8
:10E45000052D052C000C110BCB53DF4F19830883BE
:10E46000C55CD0404AE050E0B80187EB9FE00E94D5
:10E470008BE16DE27BE087EB9FE00E94EAE1C5540F
:10E48000DF4F1881CB5BD040612F70E04AE050E055
:10E4900087EB9FE00E948BE187EB9FE00E947EE08C
:10E4A000C754DF4F08811981C95BD04001151105A0
:10E4B00009F4B7C06BEB7EE0C8010F94C52ACC24E9
:10E4C000C394D12C892B09F45DC064EC7EE0C801B3
:10E4D0000F94C52A42E0C42ED12C892B09F452C0D6
:10E4E0006FED7EE0C8010F94C52A35E0C32ED12C14
:10E4F000892B09F447C068EE7EE0C8010F94C52A55
:10E5000026E0C22ED12C892BE9F16DE57FE0C80110
:10E510000F94C52A892B99F166E67FE0C8010F9414
:10E52000C52A892B09F473C060E37FE0C8010F940A
:10E53000C52ABEE0CB2ED12C892B21F169E37FE0E7
:10E54000C8010F94C52AAFE0CA2ED12C892BD1F077
:10E550006FE67FE0C8010F94C52AD12CC12C892B0E
:10E5600089F4F5E1CF2ED12C0DC0552009F46ACFE6
:10E5700081E0C554DF4F8883CB5BD04063CF93E10C
:10E58000C92ED12CC1010E947C3A682E712C6114D5
:10E59000710431F4CB53DF4F68807980C55CD04083
:10E5A000C114D10409F486C06C147D04A1F161E1A9
:10E5B0007BE087EB9FE00E94EAE14AE050E0B30194
:10E5C00087EB9FE00E948BE187EB9FE00E947EE05B
:10E5D000EDEFAE2EBB24BA94C501C453DF4F0FB686
:10E5E000F894DEBF0FBECDBFDF91CF911F910F9189
:10E5F000FF90EF90DF90CF90BF90AF909F908F9063
:10E600007F906F905F904F903F902F90089584E19E
:10E61000C82ED12CB7CFC754DF4F19821882C95BDF
:10E62000D040C154DF4FE881F981CF5BD0403197B2
:10E63000A9F4CD53DF4FF881C35CD040FF2399F09C
:10E64000CE54DF4F8881C25BD0408F7001E0CD5344
:10E65000DF4F0883C35CD040811105C0CD53DF4F2D
:10E660001882C35CD040CF54DF4FD880C15BD0400C
:10E6700015E11D1508F4E8C1ED2DF0E08827EC5BED
:10E68000FC488F4F0D9456329D73D474BB74DC7369
:10E690009D739C74627427749D739D7310751A75B5
:10E6A00038753875ED74ED74247524752475ED7422
:10E6B000ED74ED74D1011B968D919C91009709F436
:10E6C000B0CFDC01ED91FC910488F589E02DCC53AD
:10E6D000DF4FA880C45CD040C554DF4FC880CB5BFF
:10E6E000D0407801CF54DF4F0881C15BD040CE5479
:10E6F000DF4F1881C25BD040CD54DF4F2881C35B10
:10E70000D040CC54DF4F3881C45BD040CB54DF4F76
:10E710004881C55BD040CA54DF4F5881C65BD040AA
:10E72000C954DF4F6881C75BD040C854DF4F788140
:10E73000C85BD04019950C94206AD12CCD53DF4F83
:10E740008881C35CD040882309F4EECDCC53DF4FE1
:10E75000C880C45CD040952D9170E92EC755DF4F1D
:10E760000881C95AD040C655DF4F1881CA5AD040D7
:10E77000C555DF4F2881CB5AD040C455DF4F388173
:10E78000CC5AD040C355DF4F4881CD5AD040C255F6
:10E79000DF4F5881CE5AD040C155DF4F6881CF5AE4
:10E7A000D040C055DF4F7881C05BD040C1010E948E
:10E7B0008038E89491F8B8CDC1010E947C3A853048
:10E7C00009F0FBCC6CEF7AE087EB9FE00E94EAE176
:10E7D0004AE050E065E070E087EB9FE00E948BE14B
:10E7E00087EB9FE00E947EE0B101CE018F549F4FE6
:10E7F0000F94CE05D1011A968C918530C9F46EE044
:10E80000CE018F549F4F0E94D92129A33AA34BA335
:10E810005CA36DA37EA38FA398A7689480F890F85B
:10E82000D12CB1E0C554DF4FB883CB5BD04086CF4D
:10E8300061E0CE018F549F4F0E94D921298F3A8FDA
:10E840004B8F5C8F6D8F7E8F8F8F98A3E6CFC1012A
:10E850000E947C3A182F863091F565EE7AE087EBBE
:10E860009FE00E94EAE14AE050E066E070E087EB5A
:10E870009FE00E948BE187EB9FE00E947EE062E0D8
:10E88000CE018F549F4F0E94D921298B3A8B4B8BFD
:10E890005C8B6D8B7E8B8F8B988F40E050E068E0B7
:10E8A00070E0C1010E94E834689480F890F8D12C9F
:10E8B000E1E0C554DF4FE883CB5BD0403FCF67EC4E
:10E8C0007AE0BBCC40E050E061E070E0C1010E9422
:10E8D0003A35672B682B692B61F5511027C0B101C0
:10E8E000CE018F549F4F0F94CE0561E0CE018F541F
:10E8F0009F4F0E94D92129873A874B875C876D8774
:10E900007E878F87988B40E050E068E070E0C1011F
:10E910000E941135689480F890F876E0D72EF1E0E7
:10E92000C554DF4FF883CB5BD04008CF6DEA7AE067
:10E93000ADCC68E97AE0AACC5520D1F062E0CE01F6
:10E940008F549F4F0E94D92129833A834B835C8344
:10E950006D837E838F839887689480F890F865E054
:10E96000D62E01E0C554DF4F0883CB5BD040E6CE06
:10E970006BE77AE08BCCCD54DF4F8881C35BD0400E
:10E98000D12C823070F7C1010E947C3A689480F8E3
:10E9900090F8853009F411CCD12C11E0C554DF4F2B
:10E9A0001883CB5BD040CACECD54DF4F8881C35B88
:10E9B000D040823088F7552081F062E67AE087EB1C
:10E9C0009FE00E94EAE161E0C1010E94B23960E08B
:10E9D00071E1C1010E94183BF0CBCD54DF4F88811B
:10E9E000C35BD040823008F048C0DD2091F0CE54A7
:10E9F000DF4F8881C25BD0408F7031F4B101CE010E
:10EA00008F549F4F0F94CE05689480F823E0922A8C
:10EA1000D12C31E0C554DF4F3883CB5BD0408ECE54
:10EA2000689492F8D12C81E0C554DF4F8883CB5B8A
:10EA3000D04084CE689492F8D12C91E0C554DF4F39
:10EA40009883CB5BD0407ACECE54DF4F8881C25BB7
:10EA5000D0408F7051F4689490F8D12CA1E0C55447
:10EA6000DF4FA883CB5BD04069CEB3E09B2A1FCF9A
:10EA7000D12C812C54E0952E52CFD12C21E0C554BD
:10EA8000DF4F2883CB5BD04059CEDC01ED91FC9168
:10EA9000008CF18DE02DCF54DF4F0881C15BD04059
:10EAA000CE54DF4F1881C25BD040CD54DF4F288158
:10EAB000C35BD040CC54DF4F3881C45BD040CB54D3
:10EAC000DF4F4881C55BD040CA54DF4F5881C65BD9
:10EAD000D040C954DF4F6881C75BD040C854DF4F76
:10EAE0007881C85BD0401995811127CC32CCF101D7
:10EAF00083859485892B09F473C08114910439F0BE
:10EB0000A401B101CE018F549F4F0E94D139D10190
:10EB10001B968D919C91C754DF4FE880F980C95BAB
:10EB2000D040DC01ED91FC910488F589E02DCC53B7
:10EB3000DF4FA880C45CD040C554DF4FC880CB5B9A
:10EB4000D040CF54DF4F0881C15BD040CE54DF4F5F
:10EB50001881C25BD040CD54DF4F2881C35BD040C9
:10EB6000CC54DF4F3881C45BD040CB54DF4F488159
:10EB7000C55BD040CA54DF4F5881C65BD040C954F2
:10EB8000DF4F6881C75BD040C854DF4F7881C85BD6
:10EB9000D04019955C01F10183859485DC01ED91EC
:10EBA000FC91048CF58DE02D1995059711F468946E
:10EBB00080F892FC95C1DD2021F06D2DC1010E94ED
:10EBC000B239C953DF4F08811981C75CD040B40105
:10EBD0000530110509F4C9CBC1010E94183BC5CB12
:10EBE0008285863009F477C008F5843009F480C145
:10EBF000853009F78114910439F0A401B101CE01E7
:10EC00008F549F4F0E94D139C154DF4F0881198121
:10EC1000CF5BD0400230110509F466C10330110505
:10EC200009F4D2C00130110531F6CAC0883009F4A8
:10EC3000C3C1893009F0BFCF8114910439F0A40118
:10EC4000B101CE018F549F4F0E94D139C554DF4F7F
:10EC5000E881CB5BD040EE2309F4ADCF552079F0AD
:10EC6000CF54DF4F8881C15BD040813041F4CE5416
:10EC7000DF4F8881C25BD0408F7009F49CCFCF54A6
:10EC8000DF4F0881C15BD040CE54DF4F1881C25B9B
:10EC9000D040CD54DF4F2881C35BD040CC54DF4FF0
:10ECA0003881C45BD040CB54DF4F4881C55BD04036
:10ECB000CA54DF4F5881C65BD040C954DF4F6881CA
:10ECC000C75BD040C854DF4F7881C85BD040C101DA
:10ECD0000E94CB445BC1CF54DF4FF880C15BD04072
:10ECE000FF2009F487CF70E060E0C1010E94D132BB
:10ECF0008C018114910439F0A401B101CE018F542B
:10ED00009F4F0E94D1390115110509F454CF712C80
:10ED1000612C17FF06C011950195110966246394B3
:10ED2000712CC80101978634910508F044CFE02E7C
:10ED300061E0802F0F94E50EEFEFEF0DE53110F558
:10ED4000F0E08827E955F9488F4F0D945632BC768C
:10ED5000BE76C276C276BE76BC76BE76C276C27605
:10ED6000C276C276C276C276BC76BC76C276C276EF
:10ED7000C276C276BC76BC76F1E06F26662D8E2D0B
:10ED80000F94B70E6BE27AE087EB9FE00E94EAE116
:10ED90004AE050E0B80187EB9FE00E948BE169E216
:10EDA0007AE087EB9FE00E94EAE14AE050E0B3019D
:10EDB00087EB9FE00E948BE187EB9FE00E947EE063
:10EDC000689480F890F88CC0C1010E946F32892B42
:10EDD000F1F469E17AE08AE09FE00E94EAE1D10182
:10EDE0001296ED91FC91608171818AE09FE00E9412
:10EDF000D4E18AE09FE00E947EE0D1011296ED917D
:10EE0000FC91608171818CEC96E00F94E213CE014D
:10EE10008F549F4F0E94C52820E030E048EC52E418
:10EE20000F94FB300F946733C154DF4F68837983AD
:10EE30008A839B83CF5BD040C154DF4F4880598089
:10EE4000CF5BD04088E00E94789BC554DF4F688339
:10EE500079838A839B83CB5BD040C554DF4F688026
:10EE60007980CB5BD04062E17AE087EB9FE00E9443
:10EE7000EAE1D1011296ED91FC916081718187EBFD
:10EE80009FE00E94D4E16EE07AE087EB9FE00E9471
:10EE9000EAE14AE050E0C154DF4F68817981CF5BFD
:10EEA000D04087EB9FE00E948BE169E07AE087EB3E
:10EEB0009FE00E94EAE14AE050E0C554DF4F6881DC
:10EEC0007981CB5BD04087EB9FE00E949BE087EB92
:10EED0009FE00E947EE0B301A201C1010E942E3298
:10EEE000AA24A394B12C67CE689480F891F8F8CF47
:10EEF0008114910439F0A401B101CE018F549F4FC8
:10EF00000E94D139C554DF4FB881CB5BD040BB23C1
:10EF100009F451CECF54DF4F8881C15BD0405520DA
:10EF2000B9F1813041F4CE54DF4F8881C25BD040CB
:10EF30008F7009F440CECF54DF4F0881C15BD040C1
:10EF4000CE54DF4F1881C25BD040CD54DF4F2881B3
:10EF5000C35BD040CC54DF4F3881C45BD040CB542E
:10EF6000DF4F4881C55BD040CA54DF4F5881C65B34
:10EF7000D040C954DF4F6881C75BD040C854DF4FD1
:10EF80007881C85BD040C1010E94F7425C0113CE7A
:10EF9000813089F6CE018F549F4F0F946E004497B5
:10EFA00050F66EE170E0CE018F549F4F0E947228A0
:10EFB000689480F891F8BFCF8114910439F0A401CE
:10EFC000B101CE018F549F4F0E94D139C554DF4FFC
:10EFD000F881CB5BD040FF2309F4EDCD552079F0CB
:10EFE000CF54DF4F8881C15BD040813041F4CE5493
:10EFF000DF4F8881C25BD0408F7009F4DCCDCF54E5
:10F00000DF4F0881C15BD040CE54DF4F1881C25B17
:10F01000D040CD54DF4F2881C35BD040CC54DF4F6C
:10F020003881C45BD040CB54DF4F4881C55BD040B2
:10F03000CA54DF4F5881C65BD040C954DF4F688146
:10F04000C75BD040C854DF4F7881C85BD040C10156
:10F050000E94B0439BCFC953DF4F28813981C75CE1
:10F06000D0402530310509F480C940E054E0B101B9
:10F07000CE018F549F4F0E94D13960E074E0ACCD37
:10F080000E940B29672B682B692B11F00C94706B75
:10F09000912C812C11E0C554DF4F1883CB5BD040FD
:10F0A0000C94A76BC154DF4F28813981CF5BD040CE
:10F0B000232B09F053C08081882311F40C949669A6
:10F0C000CE0187549F4F0E94BB31C154DF4F9983BB
:10F0D0008883CF5BD040CD54DF4F8881C35BD04065
:10F0E000811132C0C154DF4F6881CF5BD040CE0167
:10F0F0008F549F4F0E94B721CF55DF4F2883C15AAD
:10F10000D040CE55DF4F3883C25AD040CD55DF4F67
:10F110004883C35AD040CC55DF4F5883C45AD0409F
:10F12000CB55DF4F6883C55AD040CA55DF4F78832F
:10F13000C65AD040C955DF4F8883C75AD040C855FA
:10F14000DF4F9883C85AD040C154DF4FE881F9811E
:10F15000CF5BD040EF2B11F40C94966964E57CE012
:10F1600087EB9FE00E94EAE14AE050E0B60187EBBE
:10F170009FE00E948BE16DE47CE087EB9FE00E94C2
:10F18000EAE1D1011296ED91FC916081718187EBEA
:10F190009FE00E94D4E167E47CE087EB9FE00E945F
:10F1A000EAE1C754DF4F68817981C95BD04087EBC2
:10F1B0009FE00E94D4E165E47CE087EB9FE00E9441
:10F1C000EAE1CE018F549F4F0E948C2CC754DF4F31
:10F1D00088819981C95BD040009711F40C94E16952
:10F1E000FC012081243211F00C94E16961E37CE0A0
:10F1F00087EB9FE00E94EAE187EB9FE00E947EE0C0
:10F200008CEFA82EBB24BA94E7C92F923F924F925D
:10F210005F926F927F928F929F92AF92BF92CF92A6
:10F22000DF92EF92FF920F931F93CF93DF93CDB7AF
:10F23000DEB7A2970FB6F894DEBF0FBECDBFFC01BC
:10F240006115710509F4CBC0DB0118969C919F7084
:10F25000953009F0C4C00AA319013A01F9A3E8A343
:10F26000FB01468057808091A70A8F5F8093A70A91
:10F270004114510409F4AEC0D20118968C918F70DC
:10F28000843049F018F0873008F490C0D20112960B
:10F290004D905C90EDCFF20161857285A8A1B9A176
:10F2A0008D919C910E94ADFF4C01009779F3FC0178
:10F2B00080858F70853051F74091AD0A5091AE0A2C
:10F2C000B401CE0101960E9463406114710419F1EA
:10F2D000CE0101960E94DE318823E9F0AAA0C12C5C
:10F2E0007101D3010C9111961C91119712962C91DA
:10F2F000129713963C91139714964C911497159668
:10F300005C91159716966C91169717967C91CE0185
:10F3100001960E94D2688B858730A1F561E0C40117
:10F320000F945F000AA19101A301BC0188A199A1DA
:10F330000E94057961147104A1F5882391F18091EF
:10F34000A70A81508093A70ACE0101960E94043E2D
:10F3500081E0A2960FB6F894DEBF0FBECDBFDF915D
:10F36000CF911F910F91FF90EF90DF90CF90BF90C2
:10F37000AF909F908F907F906F905F904F903F9055
:10F380002F9008956114710461F4CE0101960E94DA
:10F39000DE31882331F0CE0101960E94F179892B6C
:10F3A00071F6CE0101960E94043E70CF912C812C03
:10F3B000B12CA12CD12CC12CF301E080F180028171
:10F3C000138124813581468157816FEFC2010E94EC
:10F3D0005CAE5CCF8091A70A81508093A70A80E041
:10F3E000B8CFDF92EF92FF920F931F93CF93DF93EB
:10F3F00000D000D01F921F92CDB7DEB77C011982DA
:10F400001A821B821C821D821E821F8218868A819C
:10F41000807F8A8362EA7CE087EB9FE00E94EAE1DA
:10F42000D7011296ED91FC916081718187EB9FE08D
:10F430000E94D4E160EA7CE087EB9FE00E94EAE171
:10F44000C7010E94DE3181111BC067E97CE087EBB8
:10F450009FE00E94EAE187EB9FE00E947EE00FEFD1
:10F460001FEFC80128960FB6F894DEBF0FBECDBFC0
:10F47000DF91CF911F910F91FF90EF90DF90089552
:10F48000C7010E947C3AD82EF701838594850097A6
:10F4900091F0DC01ED91FC910688F789E02D19953A
:10F4A0008C0197FD08C081E00115110509F480E089
:10F4B0000E94831AD6CFF7018285873009F42EC0C7
:10F4C000EFEFED0DE43150F5F0E08827E559F54810
:10F4D0008F4F0D9456327F7A887A8E7A8E7A887A18
:10F4E0007F7A8E7A8E7A8E7A8E7A8E7A8E7A8E7AEB
:10F4F0007F7A8E7A8E7A8E7A8E7A7F7A7F7A68E7B2
:10F500007CE087EB9FE00E94EAE101E010E0A9CFF8
:10F5100080E00E94831A10E000E0A3CF40E052E0B8
:10F52000B701CE0101960E94893AD7011A968C91B3
:10F530001A97873089F160F4833009F458C0843019
:10F5400061F068E87CE087EB9FE00E94EAE1E3CFAE
:10F55000883009F44CC08930A1F760E0CE010196F3
:10F560000E94A6278C016DE77CE087EB9FE00E945C
:10F57000EAE14AE050E0B80187EB9FE00E948BE1AE
:10F5800087EB9FE00E947EE091E080E0012B09F490
:10F5900090E0092F182F65CF1496ED91FC9180858E
:10F5A0008F7010E000E08530F1F665E97CE087EBD4
:10F5B0009FE00E94EAE1F7016481758100E030E09C
:10F5C00020E050E040E0C7010E940579F82E082FA6
:10F5D00010E062E97CE087EB9FE00E94EAE18F2D7A
:10F5E0000E94831A87EB9FE00E947EE03ACFCE0113
:10F5F00001960E940B298B01B6CFAF92CF92EF926A
:10F60000FF920F931F93CF93DF9300D000D01F92F0
:10F610001F92CDB7DEB719821A821B821C821D820F
:10F620001E821F8218861A81107FA12CCC24C394BD
:10F63000F12CE12C02E02B813C8140E05E816F8166
:10F6400078850E94D26828960FB6F894DEBF0FBE68
:10F65000CDBFDF91CF911F910F91FF90EF90CF9091
:10F66000AF9008952F923F924F925F926F927F9248
:10F670008F929F92AF92BF92CF92DF92EF92FF92C2
:10F680000F931F93CF93DF93CDB7DEB7CC55D1093E
:10F690000FB6F894DEBF0FBECDBF4C013B0140E07A
:10F6A00058E060E070E00E943A35672B682B692BC8
:10F6B00009F45DC019821A821B821C821D821E827F
:10F6C0001F8218868A81807F8A8340E053E0B401DC
:10F6D000CE0101960E94893AD4011B968D919C918E
:10F6E000892B09F41BC140E058E060E070E0C401E0
:10F6F0000E94E83465EF7CE087EB9FE00E94EAE13E
:10F70000F40183859485DC01ED91FC910488F589F1
:10F71000E02DA12CCC24C394F12CE12C09811A8179
:10F720002B813C814D815E816F8178851995D40153
:10F730001296ED91FC918F3F9807C9F0608171811D
:10F74000892B09F055C187EB9FE00E94D4E168EB5B
:10F750007CE087EB9FE00E94EAE160EB7CE087EBD6
:10F760009FE00E94EAE187EB9FE00E947EE065E077
:10F77000F401828193810F945F005C01009709F48A
:10F780006FC1DC011896BC916B96BFAF6B97B295B9
:10F79000BF706A96BFAF6A97FC01218432844384AC
:10F7A00054840F942A136A96FFAD6A97FF2309F4D5
:10F7B00057C1261A370A480A590A19A21AA21BA2C7
:10F7C0001CA21DA21EA21FA218A68AA1807F8B6068
:10F7D0008AA3F9A3B201A101CE0181960E94252737
:10F7E00061962FAF619762963FAF629763964FAF76
:10F7F000639764965FAF649765966FAF65976696FB
:10F800007FAF669767968FAF679768969FAF689749
:10F8100024E06216710451F5D12CC12CE12C30E2A8
:10F82000F32E09A11AA12BA13CA14DA15EA16FA1AC
:10F8300078A5C4010E945E35C201B10128EE33E013
:10F8400040E050E00F940132BA01A9012AE030E013
:10F8500087EB9FE00E9443E165E07EE087EB9FE05D
:10F860000E94EAE187EB9FE00E947EE057FEF8C02D
:10F8700082E028163104410480E858060CF4F0C0F8
:10F880000E94FEA91B016D967FAF6EAF6D97D12CC4
:10F89000C12CE12C20E2F22E09A11AA12BA13CA13E
:10F8A0004DA15EA16FA178A5C4010E945E356D9641
:10F8B000AEADBFAD6D97A83CB1050CF0A6C06CEE27
:10F8C0007DE082E19FE00E94EAE14AE050E0B10180
:10F8D00082E19FE00E948BE182E19FE00E947EE056
:10F8E00066246A94762CC301C45ADF4F0FB6F8948D
:10F8F000DEBF0FBECDBFDF91CF911F910F91FF9063
:10F90000EF90DF90CF90BF90AF909F908F907F90BF
:10F910006F905F904F903F902F900895F4018285F3
:10F92000883009F445C0893019F1843009F01FCFBF
:10F930008091730A9091740A892B09F018CF40E0E6
:10F9400058E060E070E0C4010E94E83460EE7CE0C2
:10F9500087EB9FE00E94EAE109811A812B813C81BB
:10F960004D815E816F817885C4010E94F742DFCEB0
:10F970008091730A9091740A892B09F0F8CE40E0C7
:10F9800058E060E070E0C4010E94E8346FEC7CE075
:10F9900087EB9FE00E94EAE109811A812B813C817B
:10F9A0004D815E816F817885C4010E94CB44BFCEBA
:10F9B0008091730A9091740A892B09F0D8CE40E0A7
:10F9C00058E060E070E0C4010E94E8346AEB7CE03B
:10F9D00087EB9FE00E94EAE109811A812B813C813B
:10F9E0004D815E816F817885C4010E94B0439FCEB6
:10F9F00087EB9FE00E94D4E16EEA7CE087EB9FE01A
:10FA00000E94EAE16AEA7CE0AACEF50180858F7067
:10FA1000808719821A821B821C821D821E821F828D
:10FA200018868A81807F8A836A96FFAD6A97F983F8
:10FA30006B968FAD6B978F70AA24A394873009F0D3
:10FA4000A12CCC24C394F12CE12C09811A812B81A7
:10FA50003C814D815E816F817885C4010E94D268AE
:10FA600021E06216710459F4D4011A968C91843005
:10FA700079F0893009F476C1C4010E948A3BF4010F
:10FA800083859485009709F0A8C4712C612C2BCF35
:10FA90008091730A9091740A892BB9F4F40144801F
:10FAA0005580D20118968C918F70853041F4C20137
:10FAB0000F94F000082F10E00230110554F464E5B3
:10FAC0007DE087EB9FE00E94EAE1C4010E948A3B4F
:10FAD0000ACF7092740A6092730A70E060E0C40109
:10FAE0000E94D1321C0161E070E0C4010E94D13259
:10FAF0005C01053011050CF441C064E0C2010F94B3
:10FB00005F00FC010185128526E040E855E260E0D7
:10FB100070E082E29CE00E9437E32092B90D82E21D
:10FB20009CE09093B80D8093B70D1092C70E109281
:10FB3000C90E1092C80E60E47DE087EB9FE00E9442
:10FB4000EAE1D4011296ED91FC916081718187EB1D
:10FB50009FE00E94D4E187EB9FE00E947EE00130AD
:10FB6000110509F4C6C06CF4012B09F4B7C064E2B6
:10FB70007DE087EB9FE00E94EAE125C002E010E013
:10FB8000C3CF0230110579F00330110581F7B0922F
:10FB9000BC0DA092BB0D81E090E09093BE0D8093D0
:10FBA000BD0D84E00BC0B092BC0DA092BB0D81E0F6
:10FBB00090E09093BE0D8093BD0D83E00F945014A0
:10FBC00069968FAF69976996BFAD6997B1119BC070
:10FBD00080E00F94B90C8C016FE17DE087EB9FE032
:10FBE0000E94EAE1D4011296ED91FC91608171814D
:10FBF00087EB9FE00E94D4E168E17DE087EB9FE026
:10FC00000E94EAE1C801012E000CAA0BBB0B8983FC
:10FC10009A83AB83BC8380E190E09E838D83BE0199
:10FC20006F5F7F4F87EB9FE00E947B400E947EE0EA
:10FC3000B801C4010E946B3C4091AD0A5091AE0ADC
:10FC4000E091A40AF091A50A62817381CE01019628
:10FC50000E9463408091A40A9091A50A892BA9F182
:10FC6000CE0101960E94DE31882379F18B858430A4
:10FC700061F570E060E0CE0101960E94D132281655
:10FC8000390619F561E070E0CE0101960E94D1328B
:10FC9000A816B906D1F4B801CE0101960E946B3CBA
:10FCA000E091A40AF091A50A828193819093A50A1C
:10FCB0008093A40A892B49F4D401ED91FC918681AB
:10FCC00097819093A50A8093A40ACE0101960E9481
:10FCD000043E1092740A1092730AF7CEB092BC0DD3
:10FCE000A092BB0D81E090E09093BE0D8093BD0D7E
:10FCF00065CFB092BC0DA092BB0D1093BE0D0093CA
:10FD0000BD0D82E05BCF6BE07DE087EB9FE00E9462
:10FD1000EAE1D4011296ED91FC916081718187EB4B
:10FD20009FE00E94D4E163E07DE087EB9FE00E94CA
:10FD3000EAE16996EFAD69978E2F90E0B0E0A0E020
:10FD400089839A83AB83BC8380E190E09E838D831B
:10FD5000BE016F5F7F4F87EB9FE00E947B400E9458
:10FD60007EE0B7CF8091730A9091740A892B09F0D5
:10FD7000ACCE7092740A6092730A0E9431E82C0132
:10FD8000009741F0DC0118968C911897807F86606F
:10FD900018968C93F20180858F70808730E020E088
:10FDA00043E050E060E2CE0101960E947DA8D401BC
:10FDB0001296ED91FC91608171814FE150E0CE018E
:10FDC00001960F94D3366BED76E0CE0101960F9439
:10FDD000AD3626E040E855E260E070E082E29CE06B
:10FDE0000E9437E370E060E0C4010E94D13280934A
:10FDF000B90D82E29CE09093B80D8093B70D1092FC
:10FE0000C70E1092C90E1092C80E6CED7DE087EB04
:10FE10009FE00E94EAE1D4011296ED91FC9160818D
:10FE2000718187EB9FE00E94D4E187EB9FE00E9405
:10FE30007EE062E370E080E090E00F942A1184E3BA
:10FE400098E09093BC0D8093BB0D8AE090E0909376
:10FE5000BE0D8093BD0D83E00F945014182F8111B7
:10FE600052C26FEC7DE087EB9FE00E94EAE180E107
:10FE7000E82EF12C812F0F94B90C092E000CAA0B3F
:10FE8000BB0B89A39AA3ABA3BCA3FEA2EDA2BE01A8
:10FE90006F5D7F4F87EB9FE00E947B406DEC7DE0C4
:10FEA0000E94EAE11F5F1A3029F787EB9FE00E946A
:10FEB0007EE082E00F94B90CBC0190E080E00F94EA
:10FEC0009C3020E030E048EC52E40F94F5329B0186
:10FED000AC0160E477E0C2010F947C0C84E00F94E5
:10FEE000B90C6C01F12CE12CA7019C0161EE76E0CC
:10FEF000C2010F944B0985E00F94B90CBC0190E04E
:10FF000080E00F949C3020E030E048EC52E40F9405
:10FF1000F5329B01AC0165EE76E0C2010F947C0CDA
:10FF200086E00F94B90CBC0190E080E00F949C3007
:10FF300020E030E040E251E40F94F5329B01AC0147
:10FF400063EE76E0C2010F947C0C80E00F94B90C54
:10FF50009C0150E040E067EE76E0C2010F944B094F
:10FF6000CD28CE28CF2809F486C0D4011496ED916F
:10FF7000FC9190859F70953009F07DC061E0CF01C4
:10FF80000F945F00009709F476C0FC0120852F7064
:10FF9000243009F070C04091AD0A5091AE0A6185DD
:10FFA0007285CE0181960E947A3DCE0181960E9493
:10FFB000DE31882309F45BC024961CAE1DAE1EAE54
:10FFC0001FAE249728961CAE1DAE1EAE1FAE2897FE
:10FFD00022968FAD2297807F816022968FAF2297E5
:10FFE0008FEF25968FAF259726965FAD269727969C
:10FFF0003FAD279728962FAD289721969FAD219743
:020000021000EC
:1000000022967FAD229723966FAD239724964FAD0E
:100010002497092F29969FAF29972A967FAF2A9771
:100020002B966FAF2B972C964FAF2C97482F2D9672
:100030008FAF2D972E965FAF2E972F963FAF2F97AE
:1000400060962FAF6097A12CCC24C394F12CE12CA7
:10005000172F262F2C963FAD2C972F966FAD2F97ED
:1000600060967FAD6097CE0181960E94D268CE01E6
:1000700081960E94043E80E00F94B90C83FF6FC10B
:1000800062EA7DE087EB9FE00E94EAE1D4011296EC
:10009000ED91FC916081718187EB9FE00E94D4E13A
:1000A00087EB9FE00E947EE062E370E080E090E0FA
:1000B0000F942A118EE398E09093BC0D8093BB0DB2
:1000C00081E090E09093BE0D8093BD0D83E00F948E
:1000D000501481110AC00F94B90C9C0150E040E00B
:1000E0006AEE76E0C2010F944B091092740A1092E6
:1000F000730AC4010E94F179181619061CF4C40190
:100100000E94FD7A81E090E09093740A8093730AD4
:1001100062E97DE087EB9FE00E94EAE1D40112965C
:10012000ED91FC916081718187EB9FE00E94D4E1A9
:1001300087EB9FE00E947EE062E370E080E090E069
:100140000F942A1183E190E09093BC0D8093BB0D36
:1001500084E090E09093BE0D8093BD0D83E00F94FA
:100160005014182F81110DC165E87DE087EB9FE0E9
:100170000E94EAE1812F0F94B90C4AE050E0BC01E3
:1001800087EB9FE00E948BE163E87DE087EB9FE0D7
:100190000E94EAE11F5F143069F787EB9FE00E943D
:1001A0007EE080E00F94B90C8C010097C9F0BC018F
:1001B000990F880B990B0F949C302DEE3EE94CE380
:1001C0005EE30F94FB3022E538EB42E152E40F94FA
:1001D00088329B01AC016AEB77E0C2010F947C0C82
:1001E00081E00F94B90CBC01990F880B990B0F9407
:1001F0009C302DEE3EE94CE35EE30F94FB3022E5AC
:1002000038EB42E152E40F9488326B017C01AC017F
:100210009B016FED76E0C2010F947C0C83E00F949C
:10022000B90C181619060CF0A3C0BC01990F880B65
:10023000990B0F949C3020E030E040E251E40F94A1
:10024000F5329B01AC016EEE76E0C2010F947C0C9E
:1002500020E030E040E252E4C701B6010F949D3344
:100260001816BCF4012BA9F00E94CBFF882371F073
:100270008091A60A81110AC0D4011296ED91FC91D9
:100280006081718182EF96E00F94E213C4010E94B5
:10029000FD7A80E091E00F9489278C01892BD9F0B9
:1002A0001CA21BA21EA21DA28FEF9FEF98A78FA3D7
:1002B00087EA92E09AA389A31AA619A61CA70BA7FE
:1002C00080E091E098AB8FA71EA61DA6B201CE01DB
:1002D00081960F94360B0E94CBFF882349F08091C2
:1002E000A60A811105C0B801CE0101960F94E21350
:1002F000C8010F9425284114510409F4EACCC20125
:100300000F940A0BE6CC60EC7DE087EB9FE00E9447
:10031000EAE1D4011296ED91FC916081718187EB45
:100320009FE00E94D4E168EB7DE087EB9FE00E94B4
:10033000EAE1812F90E0B0E0A0E089A39AA3ABA30B
:10034000BCA380E190E09EA38DA3BE016F5D7F4FB3
:1003500087EB9FE00E947B400E947EE08CCE20E0F5
:1003600030E0A9016AEE76E0C2010F944B09D0CECD
:1003700020E030E0A9016EEE76E0C2010F944B0957
:1003800067CF63E77DE087EB9FE00E94EAE1D4015D
:100390001296ED91FC916081718187EB9FE00E9444
:1003A000D4E16BE67DE087EB9FE00E94EAE1812FDC
:1003B00090E0B0E0A0E089A39AA3ABA3BCA380E146
:1003C00090E09EA38DA3BE016F5D7F4F87EB9FE002
:1003D0000E947B400E947EE05CCFDC01ED91FC91AD
:1003E0000284F385E02D1995892B09F44ECBF40195
:1003F00083859485DC01ED91FC910480F581E02DED
:10040000B30119953C016FCA2F923F924F925F92B0
:100410006F927F928F929F92AF92BF92CF92DF9214
:10042000EF92FF920F931F93CF93DF93CDB7DEB779
:10043000CB56D1090FB6F894DEBF0FBECDBF3C013D
:100440006AEC75E0DC018D919C910E94ADFF8C01FE
:10045000F30183819091C50F8913FCC09091C60F61
:10046000903409F0F7C08091C70F9091C80F2C010C
:100470000115110509F415C1D80118962C912F709A
:10048000253009F00EC1C8010F94F000A2968FAF7D
:10049000A297843008F4EAC063E0C8010F945F00BB
:1004A000FC01818592854AE0E42EE89E1001E99ED8
:1004B000300C112462E0C8010F945F00DC01199632
:1004C0008D919C91E89E6001E99ED00C1124AC9620
:1004D000DFAECEAEAC974601DD0CAA08BB0861E0EA
:1004E000C8010F945F007C0160E0C8010F945F00B9
:1004F000DC0119962D913D914D915C911C97A6962A
:100500002CAF3DAF4EAF5FAFA6979201052C000C0C
:10051000440B550BA6968CAD9DADAEADBFADA69769
:10052000281B390B4A0B5B0BB101032C000C880B09
:10053000990B681979098A099B090F94CF31D70162
:1005400019962D913D914D915C911C97A696CCAC3E
:10055000DDACEEACFFACA6972C193D094E095F0946
:10056000A6962CAF3DAF4EAF5FAFA6970F9401326A
:10057000820E931EA41EB51EA2962FADA297253003
:1005800009F486C081E090E0A101032C000C660B09
:10059000770B481559056A057B0534F44A015B0160
:1005A00044244A9423E0522EAC96CEACDFACAC97F8
:1005B000A601DD0C660B770B84169506A606B7061A
:1005C00024F44A015B01512C412CA2962FADA29735
:1005D000223009F079C06201550CEE08FF0860E096
:1005E000C8010F945F00FC0181859285A385B485C5
:1005F000812C912C5401C816D906EA06FB060CF48E
:1006000057C261E0C8010F945F00FC0181859285AB
:10061000A385B4858C159D05AE05BF050CF444C2B9
:10062000C559DF4F0FB6F894DEBF0FBECDBFDF91C7
:10063000CF911F910F91FF90EF90DF90CF90BF90DF
:10064000AF909F908F907F906F905F904F903F9072
:100650002F9008958093C50F90E49093C60F0F9448
:10066000F80F9093C80F8093C70F01CF8AE0849D45
:100670004001859D900C1124092C000CAA08BB0890
:10068000AC961FAE1EAEAC97212C38E2332E7ACF3B
:1006900064E0C8010F945F00DC0119968D919C9174
:1006A00073CF2AE0289F4001299F900C1124092C28
:1006B000000CAA08BB08AC961FAE1EAEAC97212C4E
:1006C00098E2392E81E090E0D3011596ED91FC91EE
:1006D00022813381A201421B530B57FF03C0519566
:1006E00041955109841795070CF4C4C08081982F57
:1006F000929596959770963008F0BFC09F5F92953F
:10070000990F907E8F71892BB7C0F7016185728533
:10071000DB018C91811164C2A114B10409F45BC0A6
:10072000D50118968C9118978F70843009F053C0BA
:100730004091AD0A5091AE0A19966D917C91CE010F
:1007400001960E947A3DCE0101960E94DE318823F7
:10075000F1F18114910409F460C0E114F10431F065
:10076000F70180858F70843009F44CC025961CAE4B
:100770001DAE1EAE1FAE259729961CAE1DAE1EAE39
:100780001FAE299723961FAD2397107F23961FAF87
:10079000239781E022968FAF2297A12CCC24C3947B
:1007A000F12CE12C01E024962FAD249725963FAD46
:1007B000259740E027965FAD279728966FAD28973D
:1007C00029967FAD2997CE0101960E94D268CE016D
:1007D00001960E94043ED3011596ED91FC919382FF
:1007E00082821ECF0115110529F0F80180858F70D6
:1007F000843019F065E278E0F3C161857285FB0110
:10080000808188CF61857285FB0180818823F9F220
:10081000CE0101960F946106DACF0115110531F072
:10082000D80118968C918F708430F1F025961CAE0B
:100830001DAE1EAE1FAE259729961CAE1DAE1EAE78
:100840001FAE299723961FAD2397107F23961FAFC6
:10085000239782E022968FAF2297A12CCC24C394B9
:10086000F12CE12C02E09FCFF80161857285DB015C
:100870008C91CCCF80818F7180838081803AB8F059
:10088000AC96EEADFFADAC976F01FF0FEE08FF0821
:10089000C814D904EA04FB0451F0C101330CAA0BBB
:1008A000BB0B88159905AA05BB0509F0B9CE24151F
:1008B000350509F4B5CE6D961CAE1DAE1EAE1FAE4D
:1008C0006D976B968FAD6B97807F86606B968FAFC1
:1008D0006B976D968CAD9DADAEADBFAD6D976596CA
:1008E0008CAF9DAFAEAFBFAF6597AAE0B0E0A501FA
:1008F00094010F94203269966CAF7DAF8EAF9FAF9D
:1009000069976CEA79E087EB9FE00E94EAE14AE0B0
:1009100050E0D30113966C9187EB9FE00E94A1E019
:100920006AEA79E087EB9FE00E94EAE1CE018F5A04
:100930009F4F0E948C2C6BE576E0F30180819181C2
:100940000E94ADFF912C812CB12CA12CD12CC12C5B
:100950006296EFAC62976396FFAC639764960FADB7
:10096000649765961FAD659766962FAD66976796F7
:100970003FAD679768964FAD689769965FAD699789
:100980006FEF0E945CAED3010D911C916CEB75E092
:10099000C8010E94ADFF7C0161EC75E0C8010E94B6
:1009A000ADFF8C010097E1F1FC0180858F708430F0
:1009B000B9F56185728540E450E0CE0101960F944F
:1009C000F1366FE270E0CE0101960F94B836892BB4
:1009D00059F4D80119962D913C9143E050E060E420
:1009E000CE0101960E947DA800E020E032E040E1C7
:1009F00050E0BE016F5B7F4FCE018F5A9F4F0E9428
:100A00006E2A0E94CBFF882359F08091A60A81119B
:100A100007C0BE016F5B7F4FCE0101960F94C713D5
:100A2000E114F104D1F1F70180858F708430A9F5CC
:100A30004091AD0A5091AE0A61857285CE01019652
:100A40000E947A3DCE0101960E94DE31882309F191
:100A5000A12CCC24C394F12CE12C62960FAD6297AB
:100A600063961FAD639764962FAD649765963FAD0F
:100A7000659766964FAD669767965FAD6797689680
:100A80006FAD689769967FAD6997CE0101960E9418
:100A9000D268CE0101960E94043ED3011596ED91D5
:100AA000FC9153824282BCCD812C912C54018394C1
:100AB000D3011596ED91FC9182819381092E000C52
:100AC000AA0BBB0B88159905AA05BB0509F4A8CD8F
:100AD000D3010D911C916CEB75E0C8010E94ADFF34
:100AE0005C0161EC75E0C8010E94ADFF6C0166EC31
:100AF00075E0C8010E94ADFFA114B10431F4C11426
:100B0000D10419F4892B09F466CE66E875E0C801B2
:100B10000E94ADFF7C0161E875E0C8010E94ADFF55
:100B20008C0162EB79E087EB9FE00E94EAE14AE00A
:100B300050E0F301638187EB9FE00E94A1E060EB4E
:100B400079E087EB9FE00E94EAE14AE050E0B401DF
:100B500087EB9FE00E948BE187EB9FE00E947EE0A5
:100B6000C114D10409F4D8CDD60118968C911897E8
:100B70008F70843009F0D0CD19966D917C9140E44E
:100B800050E0CE0101960F94F1360E94CBFF8823EE
:100B900009F4C2CD8091A60A8111BECD6FE270E04A
:100BA000CE0101960F94B836892B51F4F6012185B8
:100BB000328543E050E060E4CE0101960E947DA8BA
:100BC0008114910409F40ECEE114F10439F0D70137
:100BD00018968C918F70843009F497CD64E178E099
:100BE000CE0101960F94C71397CD2F923F924F924B
:100BF0005F926F927F928F929F92AF92BF92CF92AD
:100C0000DF92EF92FF920F931F93CF93DF93CDB7B5
:100C1000DEB7CD56D1090FB6F894DEBF0FBECDBFFB
:100C2000DC0115962D913C911697232B09F45BC49A
:100C30003C01A2969FAF8EAFA29789E494E0A09664
:100C40009FAF8EAFA097A696BFAFAEAFA69781E33A
:100C500094E0A4969FAF8EAFA497FD01828162308D
:100C6000710534F064307105A4F06430710569F1E8
:100C7000863009F47DC0B8F5843009F481C0853030
:100C8000D1F461E070E0CE01825A9F4F0E94F4D40B
:100C900012C0803499F040F4843068F4873059F001
:100CA000C3010E94262407C0823441F020F090E85E
:100CB000980F943098F390E080E017C4633071058A
:100CC000D1F3C3010E940482F6CF8730A1F7CD0192
:100CD0000E940482D30115968D919C91892B59F322
:100CE00064E070E0DDCF883009F40FC3803119F77C
:100CF0000F942A131B012C01C3010E945519A12C2A
:100D0000B12C650110E3E12E15E7F12E00E010E0B3
:100D1000A20191010E94B19A882369F261EC75E009
:100D2000D3018D919C910E94ADFF8C01009709F435
:100D3000C3C2FC0180858F70843009F0BDC20F945E
:100D40002A132AE0AE014F5F5F4F0F945E2B0E9483
:100D5000CBFF882309F4B0C28091A60A8111ACC2EE
:100D6000BE016F5F7F4FD80119968D919C91A2C2F1
:100D700061E070E0CE018E599F4F0E94A3D69BCFB9
:100D80000F942A131B012C01C3010E945519A12C99
:100D9000B12C650118E9E12E1AE3F12E00E010E014
:100DA000A20191010E94B19A882309F484CFF30132
:100DB000838127968FAF279796E128969FAF289734
:100DC000282F30E0F901E650F04DE4912996EFAF7D
:100DD0002997F901E05CFF4CE4912A96EFAF2A973E
:100DE00040E85EE360E070E062964CAF5DAF6EAFEE
:100DF0007FAF629762E00F94E50E0F942A13605D57
:100E00007740810991092E966CAF7DAF8EAF9FAF71
:100E10002E9787E364968FAF6497CE018F5B9F4FC9
:100E20000F945A16882349F028968FAD28978C3056
:100E300009F473C048F48B3011F1212C312C50ECA3
:100E4000452E5FE7552E47C085518230B0F7249676
:100E50001FAD2497612F70E0762F662766277F7776
:100E600025968FAD2597682B90E080E00F949A30FF
:100E70002DEC3CEC4CEC5DE30F94FB306CC0249605
:100E80006FAD249770E090E080E00F949A306B0192
:100E90007C0125961FAD259717FF0AC0AC019B0169
:100EA00060E070E080E89FEB0F9488326B017C017A
:100EB0001F70612F70E090E080E00F949C302DEC6B
:100EC0003CEC4CEC5DE30F94FB30A70196010F94D2
:100ED00089321B012C01CE018F5B9F4F0F945A1654
:100EE000882309F403C228968FAD28978B3030F001
:100EF0008D30D0F18551823008F4E6C1A7961FAE3F
:100F0000A797A8961FAEA89730ECA9963FAFA997D0
:100F10008FE7AA968FAFAA9751C024961FAD24974A
:100F2000612F70E090E080E00F949A306B017C01BB
:100F300025966FAD25976F7070E090E080E00F947C
:100F40009C302DEC3CEC4CEC5DE30F94FB30A701A6
:100F500096010F9489321B012C0117FFBCCF57FA61
:100F6000509457F85094B7CF23966FAD239770E005
:100F700090E080E00F949C302DEC3CEC4CEC5DE379
:100F80000F94FB306B017C0122966FAD229770E0CD
:100F900090E080E00F949C309B01AC01C701B6014A
:100FA0000F948932A7966FAFA797A8967FAFA8979F
:100FB000A9968FAFA997AA969FAFAA9767E379E002
:100FC00087EB9FE00E94EAE14AE050E0D3011396EC
:100FD0006C9187EB9FE00E94A1E067E279E087EBEC
:100FE0009FE00E94EAE1B201A10187EB9FE00F942C
:100FF000D60460E279E087EB9FE00E94EAE1A796E1
:101000004FADA797A8965FADA897A9966FADA99782
:10101000AA967FADAA9787EB9FE00F94D6046EE166
:1010200079E087EB9FE00E94EAE187EB9FE00E9476
:101030007EE0F3010081118163EE78E0C8010E9437
:10104000ADFFAC969FAF8EAFAC976FEF76E0C80167
:101050000E94ADFFAE969FAF8EAFAE97A2019101F9
:10106000C201B1010F94FD33811121C019821A828E
:101070001B821C828A81807F8760F82E8A83222DC2
:101080002D823E824F825886912C812CB12CA12C2E
:10109000D12CC12CE9800B811C813E814F81588568
:1010A0006FEFAC968EAD9FADAC970E945CAEA796ED
:1010B0002FADA797A8963FADA897A9964FADA99732
:1010C000AA965FADAA97A7966FADA797A8967FAD92
:1010D000A897A9968FADA997AA969FADAA970F94A6
:1010E000FD3381112DC019821A821B821C828A81D4
:1010F000807F8760F82E8A83A7962FADA797822FCF
:10110000A8969FADA897A996AFADA997AA96BFAD8F
:10111000AA978D839E83AF83B887912C812CB12CA5
:10112000A12CD12CC12CE9800B811C813E814F81E7
:1011300058856FEFAE968EAD9FADAE970E945CAEB8
:1011400061EC75E0D3018D919C910E94ADFF7C0113
:10115000009709F4B1C0FC0180858F70843009F0DC
:10116000ABC020E030E0A901C201B1010F9495307D
:10117000882309F4A1C020E030E0A901A7966FAD53
:10118000A797A8967FADA897A9968FADA997AA967D
:101190009FADAA970F949530882309F48DC0A201C2
:1011A0009101C201B1010F949530811185C0A796BC
:1011B0002FADA797A8963FADA897A9964FADA99731
:1011C000AA965FADAA97A7966FADA797A8967FAD91
:1011D000A897A9968FADA997AA969FADAA970F94A5
:1011E0009530811169C01A821982FE0133968EE30F
:1011F000DF011D928A95E9F7F7016185728540E468
:1012000050E08E010F5F1F4FC8010F94F1366FE25F
:1012100070E0C8010F94B836892B51F4D7011996A4
:101220002D913C9143E050E060E4C8010E947DA80C
:1012300061E179E0C8010F94AD36B201A101CE01A0
:101240008C5A9F4F0E94A5A90E94CBFF882351F082
:101250008091A60A811106C0BE016C5A7F4FC80159
:101260000F94E213F80101900020E9F73197E01B99
:10127000F10BEC0FFD1F88E48083A7964FADA79775
:10128000A8965FADA897A9966FADA997AA967FADCE
:10129000AA97CE018C5A9F4F0E94A5A90E94CBFF0E
:1012A000882351F08091A60A811106C0BE016C5AB4
:1012B0007F4FC8010F94E2130F942A13AB01BC01B6
:1012C000C3010E942E19F7CC23966EAD7FAD2397F4
:1012D00076276727762790E080E00F949A302DECF0
:1012E0003CEC4CEC5DE30F94FB305CCEA7961FAE5C
:1012F000A797A8961FAEA897F0ECA996FFAFA9975D
:101300002FE7AA962FAFAA9759CE0F942A131B0145
:101310002C01C3010E945519A12CB12C650118E9BB
:10132000E12E1AE3F12E00E010E0A20191010E94EB
:10133000B19A882309F4BFCCD3011596ED91FC91A5
:101340001697818113961C91811155C01630F0F5C6
:101350008CE0E3E7F2E0DE01119601900D928A95B0
:10136000E1F7E12FF0E0EE0FFF1F21E030E02C0F5E
:101370003D1FE20FF31F60E080810F94E50E65EAE8
:1013800079E183E01330C9F070F46DEA79E181E02E
:10139000113099F069EA79E182E0123071F061EB85
:1013A00079E180E00AC061EA79E184E0143029F053
:1013B0006DE979E185E0153091F70F945C0AD3016E
:1013C0001596ED91FC9181E0818375CC6FE879E011
:1013D00087EB9FE00E94EAE14AE050E0F30163817D
:1013E00087EB9FE00E94A1E062E679E087EB9FE057
:1013F0000E94EAE160CC24E0129FF0011124E55440
:10140000F64FC080D180E280F3806EE579E087EB13
:101410009FE00E94EAE14AE050E0D30113966C910C
:1014200087EB9FE00E94A1E06AE479E087EB9FE010
:101430000E94EAE12AE030E0B701A60187EB9FE0D5
:101440000E9443E161EC75E0F301808191810E948B
:10145000ADFF8C01009709F443C0DC0118968C9114
:1014600018978F708430E1F519966D917C9140E466
:1014700050E0CE0101960F94F1366FE270E0CE019C
:1014800001960F94B836892B51F4F80121853285E5
:1014900043E050E060E4CE0101960E947DA8FF92F7
:1014A000EF92DF92CF9285ED95E09F938F938E011F
:1014B0000F5B1F4F1F930F930F9448370E94CBFF72
:1014C0000FB6F894DEBF0FBECDBF882309F4F4CE6B
:1014D0008091A60A8111F0CEB801CE010196EACE24
:1014E0006BE379E083CF8FEF9FEFC359DF4F0FB6E8
:1014F000F894DEBF0FBECDBFDF91CF911F910F914A
:10150000FF90EF90DF90CF90BF90AF909F908F9023
:101510007F906F905F904F903F902F900895AF9283
:10152000BF92CF92DF92EF92FF920F931F93CF93D0
:10153000DF93CDB7DEB7C754D1090FB6F894DEBF3D
:101540000FBECDBF8091B7099091B809A091B9099C
:10155000B091BA09892B8A2B8B2B09F4D0C00F9438
:101560002A139B01AC016091B7097091B809809171
:10157000B9099091BA09A12CB12C65011CE2E12EA8
:10158000FF24F39400E010E00E94B19A882309F44C
:10159000B6C01092B7091092B8091092B90910920A
:1015A000BA098091630A90E09595879595958795FE
:1015B00010E000E0E1E0F0E08017910709F49FC03F
:1015C0009F01002E02C0220F331F0A94E2F7C09041
:1015D000B309D090B409E090B509F090B609A9011B
:1015E000032E000C660B770B4C215D216E217F21B1
:1015F000452B462B472B09F4E0C04091B30950918D
:10160000B4096091B5097091B60920953095C9016A
:10161000330FAA0BBB0B84239523A623B7238093F8
:10162000B3099093B409A093B509B093B60980911A
:10163000660A9091670A009709F461C0FC01208551
:101640002F70253009F05BC0602F0F945F00FC0104
:1016500090859F70943009F052C061857285611544
:10166000710509F44CC0E091640AF091650A000F1D
:10167000111F000F111FE00FF11F13810281F18074
:10168000E0804091AD0A5091AE0ACE0101960E94D1
:101690007A3DE11046C0F11044C0011142C0111161
:1016A00040C018A619A61AA61BA61CA61DA61EA6F3
:1016B0001FA689A5807F89A762E0CE0188960E9437
:1016C000D92128A339A34AA35BA36CA37DA38EA32E
:1016D0009FA361E0CE0180960E94B721A12CCC246B
:1016E000C394F12CE12C89019A01AB01BC01CE011C
:1016F00001960E94D268CE0101960E94043EC95B09
:10170000DF4F0FB6F894DEBF0FBECDBFDF91CF9194
:101710001F910F91FF90EF90DF90CF90BF90AF900F
:10172000089518A619A61AA61BA689A5807F85600C
:1017300089A7EEA6FDA60CA71FA78CA59DA5AEA503
:10174000BFA548A559A56AA57BA548A359A36AA327
:101750007BA38CA39DA3AEA3BFA362E0CE01809622
:101760000E94B721A12CCC24C394F12CE12C890137
:101770009A01AB01BC01CE0101960E94D26818A665
:1017800019A61AA61BA61CA61DA61EA61FA689A5DD
:10179000807F89A761E0CE0188960E94D92128A385
:1017A00039A34AA35BA36CA37DA38EA39FA361E08F
:1017B000CE0180960E94B72196CF0F5F1F4FFCCEBF
:1017C00090E0FC01E05CFF4CE491F0E0EE0FFF1FC5
:1017D000E058F04DA591B4912C918650904DFC01AC
:1017E0008491822391E009F490E0892F089590E09C
:1017F00080E00895DC01ED91FC910284F385E02DF9
:101800001994DF92EF92FF920F931F93CF93DF9380
:10181000EC010C891D890115110559F01D8A1C8ADE
:10182000C801DF91CF911F910F91FF90EF90DF9052
:101830000895EC85FD858E859F85DF01A80FB91F72
:101840002C91243209F055C011962C912B3709F0B8
:1018500050C00296E80FF91FF12CE12CDF01D19066
:10186000DD2009F446C08DE7D816E9F08FEFE81ABD
:10187000F80AF4CF198A188A2C853D85211531057F
:1018800079F08E859F85280F391FF9012081222349
:1018900021F001969F878E873EC01D861C86C0CF93
:1018A0000FEF1FEFBDCFE114F10419F11C928E85EB
:1018B0009F8502966C857D85680F791FE881F98187
:1018C0000684F785E02DCE011995998B888B1B8AAC
:1018D0001A8AEC85FD858E859F85E80FF91FEE0D30
:1018E000FF1DD2828E859F850396E80EF91EFF8626
:1018F000EE86288939892115310509F4BDCF8A89F9
:101900009B89280F391FF9012081222309F4B2CFC6
:1019100001969B8B8A8B022F220F110B81CFDC014A
:101920001C96ED91FC911D971E968D919C91E80F50
:10193000F91F8081082E000C990B0895FC01A581E8
:10194000B681109769F0948180913102891740F037
:10195000ED91FC9111970190F081E02DCD01199549
:1019600081E090E00895DC0115968D919C9100979F
:1019700039F0DC01ED91FC910680F781E02D19949E
:101980000895FC01838594859C0144E03595279555
:101990004A95E1F756E0959587955A95E1F728170E
:1019A000390719F081E090E0089582E090E0089511
:1019B00083E090E00895DC011296ED91FC9113977D
:1019C0003097B9F016968D919C918430910541F035
:1019D0008530910541F0039749F482E090E0089545
:1019E00081E090E0089581E190E00895828590E0A3
:1019F000089590E080E0089585E090E0089590E0FB
:101A000080E008958EE090E00895DC011296ED915B
:101A1000FC9113973097B9F016968D919C91843074
:101A2000910541F08530910541F0039749F482E03A
:101A300090E0089581E090E0089581E190E00895BC
:101A4000828590E0089590E080E0089584E190E040
:101A50000895DC01ED91FC910484F585E02D60E0B2
:101A6000199581E090E00895DC011496ED91FC91C8
:101A700080E0309711F085A1817090E00895CF93B8
:101A8000DF93EC016CE87BE287EB9FE00E94EAE1E8
:101A90006C817D814AE050E087EB9FE00E948BE102
:101AA00066E87BE287EB9FE00E94EAE187EB9FE03C
:101AB0000E947EE060E08C810F94E50EE881F98160
:101AC0000484F585E02D60E0CE01199581E090E079
:101AD000DF91CF910895CF93DF93EC0166EA79E22D
:101AE00087EB9FE00E94EAE187EB9FE00E947EE0A7
:101AF000E881F9810484F585E02D60E0CE01199537
:101B000081E090E0DF91CF910895CF93DF93EC01D6
:101B10006EE375E287EB9FE00E94EAE1EA81FB81D8
:101B20000280F381E02D6081718187EB9FE00E944C
:101B3000D4E187EB9FE00E947EE0E881F981048494
:101B4000F585E02D60E0CE01199581E090E0DF9110
:101B5000CF910895EF92FF920F931F93CF93DF934E
:101B6000EC018B018091770A9091780A0097A9F097
:101B7000FC0120852F70263081F40E94ADFFFC010E
:101B800090859F70943049F481859285DF91CF9143
:101B90001F910F91FF90EF900895EE88FF88C70185
:101BA00001970D97D0F463E077E0C8010F94C33636
:101BB000892B99F48FE2888F85E08E9DB0018F9DEF
:101BC000700D11246D5E734D46E050E0CE014996D4
:101BD0000F94FC2ACE014896D9CF90E080E0D6CF72
:101BE0000D9425280D9425280D9425280D9425283D
:101BF0000D9425280D9425280D9425280D9425282D
:101C00000D9425280D9425282F923F924F925F9294
